:020000040800F2
:1000000000000220B1FF000801A3000803A30008BC
:1000100005A3000807A3000809A3000800000000CA
:100020000000000000000000000000000BA300081A
:100030000DA30008000000000FA3000811A3000892
:10004000F5FF0008F5FF0008F5FF0008F5FF0008C0
:10005000F5FF0008F5FF0008F5FF0008F5FF0008B0
:10006000F5FF0008F5FF0008F5FF00082D680008FF
:10007000F5FF0008F5FF0008F5FF0008F5FF000890
:10008000F5FF0008F5FF0008F5FF0008F5FF000880
:10009000F5FF0008F5FF0008F5FF0008B1A500080E
:1000A000F5FF0008F5FF0008F5FF0008F5FF000860
:1000B0000DA50008F5FF0008F5FF0008F5FF000892
:1000C000F5FF0008F5FF0008F5FF0008F5FF000840
:1000D000F5FF0008F5FF0008C5A60008F5FF0008B9
:1000E000F5FF0008F5FF000815A30008F5FF00085C
:1000F000F5FF0008F5FF0008F5FF0008F5FF000810
:10010000F5FF0008F5FF0008F5FF0008F5FF0008FF
:10011000F5FF0008F5FF0008F5FF0008F5FF0008EF
:10012000F5FF0008F5FF0008F5FF0008F5FF0008DF
:10013000F5FF0008F5FF0008F5FF0008F5FF0008CF
:10014000F5FF0008F5FF0008F5FF000845A30008CB
:10015000F5FF0008F5FF0008F5FF0008F5FF0008AF
:10016000F5FF0008F5FF0008F5FF0008F5FF00089F
:10017000F5FF0008F5FF0008F5FF0008F5FF00088F
:08018000F5FF0008F5FF00087F
:10018800FCAB050800000020FC0C0020000D00203E
:100198000C520020064B07481A68074B1A60074B99
:1001A80000221A70064B01221A7001F00EBA00BF25
:1001B800A03E00206C0F0020A4440020883E0020B0
:1001C800403E002008B5034801F0FFF9024B002229
:1001D8001A7008BD44130020403E002008B5054BA6
:1001E800012200201A7004F03DFE0348BDE80840D3
:1001F80001F0EBB9B8440020E81300202DE9F041E4
:10020800144C204602F053FF00201349134A02F011
:1002180005FD1349134A0746002002F0FFFC124966
:10022800124A0646002002F0F9FCD22105463A4659
:1002380023460A2002F00AFED22132462346FA203B
:1002480002F004FE5A20D2212A462346BDE8F04196
:1002580002F0FCBDFC110020F69A0508CD0100084B
:10026800FF9A0508E5010008079B05089D0100089D
:1002780008B5054B012200201A7004F0F3FD03486D
:10028800BDE8084001F0A1B9B8440020E8130020F7
:10029800044B054800221A70044B02221A7001F020
:1002A80094B900BF883E0020FC110020403E002089
:1002B80008B5034801F089F9024B00221A7008BDFD
:1002C80044130020403E00202DE9F041144C204604
:1002D80002F0EDFE00201349134A02F09FFC134977
:1002E800134A0746002002F099FC1249124A0646B2
:1002F800002002F093FCD22105463A4623460A2004
:1003080002F0A4FDD221324623465A2002F09EFD77
:10031800AA20D2212A462346BDE8F04102F096BD24
:100328006C0F0020F69A0508B9020008109B050812
:1003380099020008199B050879020008014801F094
:1003480044B900BF1010002010B5094C204602F037
:10035800AEFE00200749084A02F060FCD22102469E
:1003680023464FF48270BDE8104002F06FBD00BF15
:1003780030150020229B05084503000810B5074CDE
:100388004FF6E071206801F08DFF2068044901F004
:1003980037FFBDE8104003F0C3B800BF000D0020D0
:1003A800299B050810B5074C4FF6E071206801F04D
:1003B80079FF2068044901F023FFBDE8104003F0ED
:1003C800AFB800BF000D00203E9B050810B5074CD4
:1003D8004FF6E071206801F065FF2068044901F0DC
:1003E8000FFFBDE8104003F09BB800BF000D0020D0
:1003F800539B050810B5074C4FF6E071206801F0D3
:1004080051FF2068044901F0FBFEBDE8104003F0ED
:1004180087B800BF000D0020689B050810B51E4C6A
:10042800FFF7C0FF002004F01DFD23790BB9FFF78B
:10043800A5FF63790BB9FFF7C9FFA3790BB9FFF7DC
:10044800D9FF154B5A79E2B11A79D2B199790022BC
:100458001A715A7101B19A71104B0F4C1A7008F049
:10046800F9FE20684FF6E07101F01CFF20680C4986
:1004780001F0C6FE08F053F803F052F8094803F0FB
:1004880093F8FFF78FFF002008F00AF80648BDE848
:10049800104001F09AB800BF000D0020403E002037
:1004A8007D9B0508809698004413002008B500201D
:1004B80007F0F6FF0248BDE8084001F086B800BF23
:1004C8004413002010B586B04FF07E5302930023EA
:1004D800039308F0BAFD8DED000ACDED010A9DE801
:1004E800030006AB03E903009DED020ADDED030AF4
:1004F8009DED041ADDED051A08F059FD104C002099
:1005080084ED040AC4ED050A07F0DAFF20644FF60B
:10051800E07004F07BFCB7206E215E22002304F01B
:1005280091FD084B1A68084B1A60084B02224FF0DD
:10053800804001211A7006B0BDE810400DF06BBF75
:1005480038480020903E0020A4440020190E0020C6
:100558001FB508F07AFD8DED000ACDED010A9DE882
:100568000300104A02AB83E8030082E803004FF659
:10057800E07004F04BFCFFF73DFFB7203C215E2202
:10058800002304F05FFD084B1A68084B1A60084BFB
:1005980001214FF08040197005B05DF804EB0DF0B3
:1005A8003ABF00BF38480020903E0020A4440020F5
:1005B800190E002010B5224B2248234C86B0029316
:1005C8000023039302F0F0FF08F03FFD20460121CD
:1005D80084ED080AC4ED090A08F057FD8DED000AFC
:1005E800CDED010A9DE8030006AB03E903009DED8C
:1005F800020ADDED030A9DED041ADDED051A08F087
:10060800D6FC4FF6E07084ED0C0AC4ED0D0A04F038
:10061800FDFBFFF7B3FEB720A0215E22002304F004
:1006280011FD0A4B1A680A4B1A600A4B03224FF055
:10063800804001211A7006B0BDE810400DF0EBBEF5
:1006480000004842A086010038480020903E002063
:10065800A4440020190E00202DE9F04F434D444ECC
:1006680085B000244FF6FF78284602F020FD414669
:10067800224623463F480094019401F0D7FD042701
:10068800B060224623464FF6E0713B48009701943C
:1006980001F0CCFD2346306041462246374800979A
:1006A800019401F0C3FD3649F060364A204602F055
:1006B800B5FA3549354A0746204602F0AFFA3449BB
:1006C800344A8046204602F0A9FA3349334A814623
:1006D800204602F0A3FA3249324A8246204602F006
:1006E8009DFA3149314A84462046CDF80CC002F0C3
:1006F80095FA21468346B2682B46204602F0A6FBAF
:10070800214632682B467D2002F0A0FB2321F268A7
:100718002B46B42002F09AFB9B213A462B46FA203E
:1007280002F094FB372142462B46FA2002F08EFB5A
:1007380069214A462B46FA2002F088FBC821524616
:100748002B466E2002F082FBC8215A462B46AA206F
:1007580002F07CFBDDF80CC0F0206246C8212B4675
:1007680005B0BDE8F04F02F071BB00BFA012002039
:10077800000D0020919B0508999B0508AC9B050876
:10078800B49B0508BD050008BC9B05085905000871
:10079800C49B0508CD040008CC9B0508610B000824
:1007A800D39B0508B5040008DA9B05082504000852
:1007B8001FB5134802F0F8FE08F047FC8DED000A5B
:1007C800CDED010A9DE803000E4A02AB83E8030061
:1007D80082E803004FF6E07004F018FBFFF70AFE0A
:1007E8005E220023DF203C2104F02CFC064B012272
:1007F8001A71064B1A68064B1A6005B000BD00BF97
:10080800A086010040480020000D0020A03E0020E6
:10081800A444002010B586B04FF07E530293002305
:10082800039308F012FC8DED000ACDED010A9DE856
:10083800030006AB03E903009DED020ADDED030AA0
:100848009DED041ADDED051A08F0B1FB0E4C0020F1
:1008580084ED060AC4ED070A07F03EFE60644FF611
:10086800E07004F0D3FADF206E215E22002304F04A
:10087800E9FB064B01229A71FFF7A8FD044B1A68A1
:10088800044B1A6006B010BD38480020000D002047
:10089800A03E0020A444002008B5FFF76FFDBDE886
:1008A800084002F03DBE70B52DED028B9FED238A06
:1008B80088B00A26F0EE488A03E0B0EE608AF0EECF
:1008C800418A08F0C2FB8DED000ACDED010A9DE8D2
:1008D800030004AB83E80300F0EE680AB0EE480AB0
:1008E8009DED041ADDED051A8DED028ACDED038A22
:1008F80008F042FBCDED010A8DED000A9DE80300EA
:1009080002AD85E80300013E6C46DDED020A9DED6F
:10091800031AD2D19FED0A0A08F08EFB8DED000A6A
:10092800CDED010A9DE8030085E80300DDED030A2B
:100938009DED020A08B0BDEC028B70BD00000000FE
:10094800CDCCCC3D2DE9F74F564D574CDFF864918F
:10095800DFF864814FF6E07004F058FA28680EF06A
:10096800ABFC064668680F460EF0A6FC3246CDE999
:1009780000013B464946204613F0E4F9224600238D
:100988000520372104F07CFB2869484F484E0EF0BB
:1009980093FC824668698B460EF08EFC5246CDE980
:1009A80000015B463946204613F0CCF92246002365
:1009B8000520692104F064FB286B0EF07DFC82465B
:1009C800686B8B460EF078FC5246CDE900015B4619
:1009D8004146204613F0B6F9002305209B21224604
:1009E80004F04EFB31462A6C204613F0ABF9224640
:1009F80000239B21A22004F043FB4FF4FC6004F089
:100A080005FAA8680EF058FC8246E8688B460EF096
:100A180053FC5246CDE900015B464946204613F097
:100A280091F9224605205021002304F029FBA869EA
:100A38000EF042FC8246E8698B460EF03DFC5246B9
:100A4800CDE900015B463946204613F07BF9224682
:100A580000230520822104F013FBA86B0EF02CFC68
:100A68008246E86B8B460EF027FC5246CDE9000122
:100A78005B464146204613F065F900230520B42162
:100A8800224604F0FDFA31466A6C204613F05AF902
:100A9800A220B4212246002303B0BDE8F04F04F0A1
:100AA800EFBA00BF38480020100D0020F39B05085E
:100AB800169C0508E19B0508059C050810B5204B08
:100AC8002048214C86B002930023039302F06CFD6A
:100AD80008F0BBFA2046022184ED0A0AC4ED0B0A8D
:100AE80008F0D3FA8DED000ACDED010A9DE8030068
:100AF80006AB03E903009DED020ADDED030A9DED57
:100B0800041ADDED051A08F052FA4FF6E07084ED8C
:100B18000E0AC4ED0F0A04F079F9DF20A0215E2245
:100B2800002304F08FFAFFF73DFC084B01225A71AD
:100B3800FFF708FF064B1A68064B1A6006B010BD8F
:100B480000004842A086010038480020000D00201F
:100B5800A03E0020A444002008B5FFF723FCBDE810
:100B68000840EFE6002008B504F07CF9064B0022A7
:100B78001A70064B1B78022B0CBF05480548BDE8C8
:100B8800084000F022BD00BFB8440020403E0020CD
:100B9800FC1100206C0F00202DE9F14F2D4C204650
:100BA80002F085FA00202C492C4A02F037F82C492B
:100BB8002C4A8146002002F031F82B492B4A07467F
:100BC800002002F02BF82A492A4A0646002002F0A3
:100BD80025F82949294A0546002002F01FF8284926
:100BE800284A8046002002F019F82749274A8246F9
:100BF800002002F013F8D22183464A462346E62015
:100C080002F024F928203A462346014602F01EF94C
:100C1800462132462346282002F018F964212A4644
:100C28002346282002F012F9822142462346282032
:100C380002F00CF9524623462820A02102F006F9BA
:100C480028205A46BE21234601B0BDE8F04F02F0E5
:100C5800FDB800BFE81300201B9C05086D0B0008B9
:100C6800249C0508811100082F9C05085D110008C7
:100C7800399C050839110008449C0508151100081D
:100C88004F9C0508F1100008599C0508CD10000874
:100C9800023810B5052800F2CE81DFE810F0060012
:100CA8000A005F00C90081011701BDE8104007F084
:100CB800A3BC00204FF6E07107F0A4FD63204FF6B7
:100CC800E07107F09FFDB3204FF4F06107F09AFD43
:100CD800C7204FF6E07107F095FD4FF6FF7004F05E
:100CE80095F8DC2100237D20D34A04F0C9F94EF29F
:100CF8009C7004F08BF8052001210023CF4A04F0F2
:100D0800BFF9052052210023CD4A04F0B9F9B621D4
:100D180000230520CB4A04F0B3F94FF4F06004F047
:100D280075F80121002340F21310C44A04F0A8F911
:100D3800002340F213105221C24A04F0A1F9B6214F
:100D4800C14A40F21310002304F09AF94EF29C7045
:100D580004F05CF80520A221BC4A67E100204FF6A8
:100D6800E07107F04FFD31204FF6E07107F04AFDC2
:100D780063204FF6E07107F045FD95204FF6E071CE
:100D880007F040FDC7204FF6E07107F03BFD4EF23B
:100D98009C7004F03BF8052001210023AC4A04F0C4
:100DA8006FF9052020210023AA4A04F069F90520DB
:100DB80052210023A84A04F063F905208421002366
:100DC800A64A04F05DF9B62105209E4A002304F0E6
:100DD80057F94FF4F06004F019F8012140F21310AC
:100DE80000239B4A04F04CF940F2131020219C4A3E
:100DF800002304F045F940F213105221914A0023D0
:100E080004F03EF940F213108421964A002304F0BE
:100E180037F9B621944A40F21310002304F030F950
:100E28004FF6FF7003F0F2FF7D20DC218F4AFDE0D2
:100E380000204FF6E07107F0E5FC27204FF6E0713F
:100E480007F0E0FC4F204FF6E07107F0DBFC77205D
:100E58004FF6E07107F0D6FC9F204FF6E07107F0DF
:100E6800D1FCC7204FF6E07107F0CCFC4EF29C7025
:100E780003F0CCFF052001210023724A04F000F999
:100E88000520162100237A4A04F0FAF805203E21AD
:100E98000023784A04F0F4F8052066210023764AF6
:100EA80004F0EEF88E2100230520744A04F0E8F8D7
:100EB8000520734AB621002304F0E2F84FF6FF70CC
:100EC80003F0A4FF7D20DC216E4AAFE000204FF63E
:100ED800E07107F097FC31204FF6E07107F092FCC3
:100EE80063204FF6E07107F08DFC95204FF6E07116
:100EF80007F088FCC7204FF6E07107F083FC4EF23C
:100F08009C7003F083FF0520012100235E4A04F052
:100F1800B7F80520202100235C4A04F0B1F8052029
:100F2800522100235A4A04F0ABF8052084210023FB
:100F3800584A04F0A5F8B6210520424A002304F0D7
:100F48009FF84FF4F06003F061FF012140F21310A5
:100F58000023514A04F094F840F2131020214F4A1C
:100F6800002304F08DF840F213105221354A002373
:100F780004F086F840F213108421494A002304F053
:100F88007FF8B621474A40F21310002304F078F89E
:100F98004FF6FF7003F03AFF7D20DC21424A45E01E
:100FA80000204FF6E07107F02DFC31204FF6E0717C
:100FB80007F028FC63204FF6E07107F023FC95202A
:100FC8004FF6E07107F01EFCC7204FF4FC6107F0F4
:100FD80019FC4EF29C7003F019FF05200121002333
:100FE800324A04F04DF8052020210023304A04F04D
:100FF80047F80520522100232E4A04F041F88421A5
:10100800002305202C4A04F03BF84FF4F06003F06D
:10101800FDFEB6210520294A002304F031F84FF6D9
:10102800FF7003F0F3FE264A8720DC210023BDE889
:10103800104004F025B810BD2F9C0508639C0508D6
:101048005E9C050815A10508629C0508909C05088A
:101058007C9C0508679C0508779C05086C9C05081E
:10106800719C0508769C05087B9C0508399C050839
:101078007F9C0508839C0508879C05088B9C0508B0
:101088008F9C0508939C05089F9C0508A39C050850
:1010980073A40508A79C0508B09C0508AC9C050826
:1010A800AB9C0508AF9C0508B49C0508BF9C0508C7
:1010B800889C0508809C050889A405082CA20508B9
:1010C800599C050810B5064C06480623237000F005
:1010D8007CFA2078FFF7DCFDBDE8104007F01CBF64
:1010E800B84400207816002010B5064C064807239F
:1010F800237000F06AFA2078FFF7CAFDBDE81040B7
:1011080007F00ABFB84400207816002010B5064C36
:1011180006480523237000F058FA2078FFF7B8FD39
:10112800BDE8104007F0F8BEB8440020781600204B
:1011380010B5064C06480423237000F046FA2078C0
:10114800FFF7A6FDBDE8104007F0E6BEB844002052
:101158007816002010B5064C06480323237000F0CB
:1011680034FA2078FFF794FDBDE8104007F0D4BEAC
:10117800B84400207816002010B5064C0648022313
:10118800237000F022FA2078FFF782FDBDE81040B6
:1011980007F0C2BEB8440020781600200F4A012389
:1011A80010B513700E4A002414700E4A20461370AE
:1011B80007F076F9204603F055FE0B4B04221A700F
:1011C80007F0F6FD07F094FE084B09481C70094B20
:1011D8001C70BDE8104000F0F8B900BFB84400200A
:1011E800100E00200D0E0020403E00203C4600203E
:1011F800B4100020883E00200F4A38B50123137030
:101208000E4A002414700E4A2046137007F048F95D
:10121800204603F027FE0B4B02251D7007F0C8FD82
:1012280007F066FE084B09481D70094B1C70BDE8A5
:10123800384000F0CAB900BF180E0020100E002078
:10124800B8440020403E00203C460020E81300201F
:10125800883E0020034B01224FF4FC601A7003F013
:10126800D5BD00BF100E00200B4B10B50024204642
:101278001C7003F0F7FD07F029FB06F05FFE074B33
:101288001C70074B01221A7007F01AFB0548BDE8CD
:10129800104000F09AB900BF100E0020B84400209A
:1012A800403E00206C0F00200A4B10B50024204659
:1012B8001C7003F0D7FD07F009FB074B1C70074BA8
:1012C80002221A7007F0FCFA0548BDE8104000F049
:1012D8007CB900BF100E0020B8440020403E00201A
:1012E800FC11002008B5074B0020187003F0BAFD68
:1012F800054B064803221A7000F067F9BDE808405C
:10130800FFF7CABA100E0020403E0020A0120020AD
:101318000C4B10B500220C4C1A7007F0D7FA04F0E9
:101328003BFD07F002F907F0CBFA20684FF6E071B1
:1013380000F0B8FF2068054900F062FFBDE81040E2
:1013480002F0EEB8100E00202C0D0020C39C0508FA
:101358000E4B002210B51A700088C83880B20428D5
:1013680005D90B480B4A0C4B912102F001FB0B4CA1
:10137800C0B204F09BFD20684FF6E07100F092FFC8
:1013880020680749BDE8104000F03ABF100E002061
:10139800D79C050814DC0308F79C05082C0D0020D1
:1013A800289D05082DE9F04F6448654D89B0002453
:1013B80001F07DFE4FF6FF712246234661480094F6
:1013C800019400F033FF042607464FF6E0712246E9
:1013D80023465D480096019400F028FF4FF6E0711F
:1013E80080462246234659480096019400F01EFF85
:1013F8004FF6FF71814622462346554800960194D0
:1014080000F014FF234628604FF6FF71224651482A
:101418000096019400F00AFF4F4968604F4A204641
:1014280001F0FCFB4E494F4A8246204601F0F6FB8C
:101438004D494E4A8346204601F0F0FB4C49039043
:101448004C4A204601F0EAFB4B4904904B4A20469F
:1014580001F0E4FB4A4905904A4A204601F0DEFBC8
:1014680049490690494A204601F0D8FB3A46079078
:101478002146324B204601F0E9FC214642462F4BDB
:10148800C82001F0E3FC0A214A462C4BC82001F091
:10149800DDFC2A68294B5521782001F0D7FC6A68C1
:1014A800264B7820692101F0D1FCC8250526232781
:1014B800E0B204F02BFC364A0146284601F0AEFBA8
:1014C80094FBF6F106FB114179431E31024689B2BD
:1014D80000201A4B0134013501F0B8FC042CADB2E0
:1014E800E6D1D22152460520144B01F0AFFCD2219F
:1014F8005A464C20114B01F0A9FCD221039A0F4BFC
:101508009C2001F0A3FCD221049A0C4BEC2001F0A2
:101518009DFCB421059A094BEC2001F097FCB421FD
:10152800069A064B9C2001F091FC079A034B4C202D
:10153800B42109B0BDE8F04F01F088BC4413002085
:101548002C0D0020389D0508429D05084F9D050873
:101558005A9D05083F9B05086E9D0508191300084C
:10156800769D0508ED1200087F9D0508B112000858
:10157800889D050871120008919D05085D120008F4
:101588009A9D050801120008A39D0508A5110008E9
:101598005913000808B500F04FFBFEF72FFE00F0C6
:1015A80083F8FFF759F8FEF78FFEFFF7F5FA00F01A
:1015B80009FDFFF7F7FEFEF7C7FE00F0EDFB00F0B0
:1015C80047FABDE8084000F015BB10B5044628B935
:1015D8000F48104A104B492102F0CAF90F4B1868FE
:1015E800844213D010B1C36900219847002003F04A
:1015F80039FC002003F020FC4FF6FF7003F006FCD6
:10160800E369204601219847044B1C6010BD00BFC8
:10161800AC9D050823DC0308C89D0508340D00208F
:101628000048D2E74413002008B5124B124A1B7831
:101638000D2B8CBF00210121117014225A430F4930
:1016480088588B184FF47A720D49504308605968CE
:101658004A430C490A609A680B4B1A6006F0DEFE92
:1016680007F02EF9094B0A4800221A70BDE8084015
:10167800FFF7ABBFA63E0020280F00200000002087
:10168800A83E0020C44400209C440020403E002086
:1016980044130020024B034800221A70FFF795BF3D
:1016A800403E0020441300202DE9F347384DDFF871
:1016B800FC80384E0024284601F0F9FC22462346D7
:1016C80047F6FF7134480094019400F0AFFD4FF6DF
:1016D800FF7904278246494622462346404600971A
:1016E800019400F0A3FD4946306022462346404657
:1016F8000097019400F09AFD4946706022462346FF
:1017080040460097019400F091FD2346B060494699
:10171800224640460097019400F088FD1F49F0607A
:101728001F4A204601F07AFA1E491F4A07462046FA
:1017380001F074FA2146804652462B46204601F0B5
:1017480085FB3C2132682B465A2001F07FFB5A204A
:1017580072682B46014601F079FB7821B2682B4666
:101768005A2001F073FB9621F2682B465A2001F0AB
:101778006DFBD2213A462B46EC2001F067FB9C20FA
:10178800D22142462B4602B0BDE8F04701F05EBBCD
:10179800B4100020380D0020D89D0508E59D0508E7
:1017A8009D160008EE9D0508311600083F9B0508A8
:1017B80070B5474E474C327847492DED028B1425BA
:1017C80092B005FB02420C320FA812F0BBFA337834
:1017D8000D2B05FB03F504EB050332D8D3ED016AA5
:1017E8009B6807EE103A6359B8EEE68A06EE903A1F
:1017F800DFED3A7AF8EEC78AB8EEE67A88EE278AFD
:10180800C8EEA78AC7EE277A17EE900A0DF054FDA6
:1018180002460B466846324912F094FA18EE100A4E
:101828000DF04AFD02460B4605A82E4912F08AFA29
:1018380018EE900A0DF040FD02460B460AA82A4908
:1018480029E093ED017A9B6807EE903A635906EE1A
:10185800903AF8EEE78AF8EEE67AB8EEC78A17EE1D
:10186800900A0DF029FD02460B4668461F4912F002
:1018780069FA18EE100A0DF01FFD02460B4605A87E
:101888001B4912F05FFA18EE900A0DF015FD0B4691
:10189800184902460AA8184C12F054FA2068174949
:1018A80000F0AEFC20680FA900F0AAFC6068694649
:1018B80000F0A6FCA06805A900F0A2FCE0680AA94F
:1018C80000F09EFC01F02CFE12B0BDEC028B70BD46
:1018D800A63E002000000020F79D050800007A447D
:1018E800029E0508139E0508249E0508359E0508D6
:1018F800469E0508579E0508380D0020489B050898
:101908004FF6FF7070474FF6FF7070471FB50029FC
:1019180047D04FF2DE7003F0A5FA002003F078FB01
:101928000F2003F073FA1F4C1F4A412101230A209C
:1019380003F0A6FB042003F06BFB23682820962104
:10194800042B24DC0123194A03F09AFB03A90DF1A7
:101958000E02206803F01CFE0F2003F057FABDF8B2
:101968000C00BDF80E1014380F242822002380B272
:10197800009403F07BFABDF80E10BDF80C0000943B
:10198800143989B22822012303F070FA09E0084AC1
:10199800012303F075FB1E20A521064A012303F04D
:1019A8006FFB1FBD480D0020689E05087B9E05083B
:1019B800979E0508AD9E050837B51E4C2368042B75
:1019C80005462BDC01A80DF1060103F0DFFDBDF88B
:1019D8000630BDF80420184904200AF021FD2368C8
:1019E800002B04DA1548164A164B592105E0042B3A
:1019F80005DD1248124A144B5A2101F0B9FF04EBD5
:101A08008302BDF8041001339180BDF806102360ED
:101A1800052BD18008D1201D03F03AFE00230B4886
:101A28002360FFF7D2FD03E028460121FFF76EFF90
:101A38003EBD00BF480D0020C49E0508099F05084B
:101A480035DC03082B9F0508429F05088C140020ED
:101A580037B50B4C204601F02AFB0A4B0A49009384
:101A680000250120094A0A4B019501F0C8F92946C9
:101A780002462346284603B0BDE8304001F0E6B9E7
:101A88005811002015190008091900080F19000835
:101A9800C11900084FF6FF7070474FF6FF70704786
:101AA80030B54FF6E07087B003F0DCF9002003F0A2
:101AB800AFFA0F2003F0AAF900212C4A2C4C01237D
:101AC8000A2003F0DDFA002003F0A0F9042003F057
:101AD8009FFA0A201921274A012303F0D1FA252168
:101AE800254A01230A2003F0CBFA1F2003F08EF9C0
:101AF80001230A203721214A03F0C2FA2378002B58
:101B080031D001231E2096211D4A03F0B9FA6288BC
:101B18001C4902A812F016F901231E20A22102AACC
:101B280003F0AEFAA288184902A812F00BF9AE2108
:101B380002AA01231E2003F0A3FA0F2003F066F97E
:101B48006088A188143880B20F25282200230095C8
:101B580003F08CF9A18860880095143989B228228D
:101B6800012303F083F907B030BD00BF709F05085B
:101B7800600D0020829F0508A29F0508C29F0508E6
:101B8800E59F0508F79F050804A0050801B187E748
:101B9800704713B50DF1060101A803F0ABFC144B17
:101BA80001221A705988BDF80420891A0E311C299F
:101BB80019460AD89C88BDF80600201A0E301C2841
:101BC80003D899680131996001E000238B60084BC4
:101BD8009968012905DD00229A601A70FFF720FD37
:101BE80005E05A80BDF806209A80FFF759FF1CBD12
:101BF800600D002037B50B4C204601F058FA0A4B0F
:101C08000A49009300250120094A0A4B019501F071
:101C1800F6F8294602462346284603B0BDE8304078
:101C280001F014B98C140020951B00089D1A0008B7
:101C3800A31A00089B1B000810B50B4C204601F0A6
:101C480036FA00200146224600F050FB00200749E2
:101C5800074A00F0E3FFD221024623464FF4827080
:101C6800BDE8104001F0F2B87816002011A0050870
:101C7800A11C000870B5C9240AE0A8B200223146A8
:101C8800013502F02DFAF02DF7D10134EF2C02D0F6
:101C98000025A6B2F1E770BD08B5FFF7EBFF0248D3
:101CA800BDE80840FFF791BC1010002010B5064CA5
:101CB8004FF6FF71206800F0F5FA044B20681968A8
:101CC800BDE8104000F09CBA6C0D0020EC0200202A
:101CD80008B5FFF7EBFF0020014606F0C1FABDE8A2
:101CE800084001F01DBC08B5002003F0BBF8054B07
:101CF8001868054B196800F083FA0448BDE80840E5
:101D0800FFF763BC6C0D0020E8020020441300209C
:101D18000088A0F5C87080B2092808B505D9084818
:101D2800084A094B902101F023FE084B1880084B04
:101D3800FF21197006F094FABDE80840B6E700BF25
:101D480016A0050847DC030839A005081C17002061
:101D58001E1700200088A0F5967080B2092808B5E3
:101D680005D90848084A094B842101F001FE084BAF
:101D78001880084B0121197006F072FABDE8084076
:101D880094E700BF16A005085CDC030839A0050825
:101D98001C1700201E170020F7B500243648374DC1
:101DA80001F085F9224623464FF6FF713448009426
:101DB800019400F03BFA04262246234607464FF6D4
:101DC800FF7130480096019400F030FA23462860ED
:101DD80022464FF6FF712B480096019400F026FA30
:101DE80029496860294A204600F018FF20462849FA
:101DF800284A00F013FF214606463A4620461E4B65
:101E080001F024F82A681C4B2046282101F01EF80E
:101E18003246AA20D221184B01F018F80F254FF4AA
:101E2800967440F2351620461B491C4A00F0F6FE0F
:101E380001340246782128460F4BA4B2233501F01D
:101E480005F8B442ADB2EED10F254FF4C87440F294
:101E5800991620461249134A00F0E0FE0134024662
:101E68009B212846044BA4B2233500F0EFFFB4426F
:101E7800ADB2EED1FEBD00BFD41500206C0D002020
:101E88006AA00508509B050876A00508D91C00081B
:101E98007FA00508EF1C000888A005085D1D000844
:101EA8008AA00508191D000808B5FFF7FFFE0020E5
:101EB800014606F0D5F9BDE8084001F031BB00BF86
:101EC80008B506F07DFF164A00230220CA2103F058
:101ED800D7F8144B1A68144B1A60144B1B78023B42
:101EE800052B1CD8DFE803F003070B13170FBDE819
:101EF8000840FFF741B9BDE80840FFF72BB9BDE836
:101F08000840FFF715B9BDE80840FFF7EDB8BDE890
:101F18000840FFF7FBB8BDE80840FFF7D3B808BD95
:101F28003E9B0508A03E0020A4440020B8440020A1
:101F380008B5084B01221A70074B1A68074B002096
:101F48001A6002F08FFF06F033FF0548BDE808402D
:101F5800FFF73BBB180E0020A03E0020A444002041
:101F6800E813002038B50E4B0E4D00241C700E4BA4
:101F78001C700E4B1C700E4B1A680E4B20461A60D4
:101F880002F070FF0C4B1B78022B0CBF0B480C485F
:101F9800FFF71BFB2C70BDE8384006F009BF00BFF7
:101FA800180E00203C460020B8440020883E00203F
:101FB800A03E0020A4440020403E0020FC11002048
:101FC8006C0F00202DE9F041144C204601F06FF809
:101FD80000201349134A00F021FE1349134A07460B
:101FE800002000F01BFE1249124A0646002000F0AD
:101FF80015FED22105463A462346E62000F026FF84
:102008004B2132462346642000F020FF64206921DA
:102018002A462346BDE8F04100F018BF1010002002
:102028001B9C05086D1F00088CA00508391F0008B7
:1020380098A00508C91E000808B508B143682BB95F
:102048000348044A044B9B2101F092FC586908BDDF
:10205800A5A0050870DC0308C7A0050808B5FFF7A8
:10206800EBFF8068123080B208BD08B5FFF7E4FFC7
:102078004068063080B208BD2DE9F84F044688460E
:10208800FFF7DAFF6689E589074606F1030905F1D6
:102098000F0AB8F1000F1FD01F2002F0B7FE20462C
:1020A800FFF7DCFF83462046FFF7DFFF294603469C
:1020B8005FFA8BF2F0B202F0E9FE042002F0A8FF0A
:1020C8000B364FF6FF70033502F0A0FEB0B2A9B28E
:1020D8003A68012302F0D4FF3D69204641464A464A
:1020E8005346A847BDE8F88F13B504460DF106011D
:1020F80001A803F0FFF92046FFF79EFF6389BDF8AA
:102108000410BDF80620C91AE389D21A0339C36836
:102118000F3A204698471CBDF7B5044614200D46D3
:1021280016461F4611F09CFA089BC7600361064BD0
:102138000649074A80E8700000930190054B00208B
:1021480000F05DFEFEBD00BF81200008732000087E
:1021580065200008F1200008704708B508B14368F9
:102168002BB90448044A054BAD2101F001FC58691C
:1021780008BD00BFE6A0050888DC0308C7A005085D
:10218800F8B505460E46FFF7E8FF836B04461BB11A
:1021980028463146984700E018466F8994F83C3045
:1021A800ED890EB9034310D0208E02F02FFE608E09
:1021B80002F042FE94F8350002F02AFF94F8343019
:1021C80038462946224602F05BFF002384F83C305B
:1021D800F8BD08B5FFF7C1FF90F83500BDE8084025
:1021E80002F02BBF38B5FFF7B8FF044611F030FEF8
:1021F800054694F8350002F01BFF684380B238BDED
:1022080038B50D46FFF7A9FF29462E22044611F0DE
:102218004FFE50B1204629462E2211F09BFE002386
:1022280084F82E30012384F83C3038BD2DE9F7437B
:10223800074640200E461546984611F011FA044606
:1022480028B91148114A124B4E2101F091FB114B4C
:10225800114A12498DE818000020114B00F0CFFDFB
:1022680039468146FFF7CCFF9DF82830268684F84A
:1022780035300B9B6586A363002384F8348084F88B
:102288003C304846BDE8FE83E6A00508A0DC03080C
:1022980004A1050889210008DB210008ED210008B8
:1022A8006121000810B50C46FFF757FF012304868B
:1022B80080F83C3010BD00BF4FF4A0707047C820B4
:1022C80070477047074B1B78022B07B508D1064BA0
:1022D8001B78022B04D001A80DF1060103F00AF9BE
:1022E8000EBD00BF3C460020B844002073B50A4B21
:1022F80006460D461446009300200849084A094B33
:10230800019000F07CFD294602462346304602B083
:10231800BDE8704000F09ABDCB220008C122000839
:10232800C7220008CD22000813B502AB03E9060056
:10233800436843B1027C0124082A9C7004D11B69BC
:102348002146984700E01C4620461CBD30B50028B1
:102358002BD0058B002425E0036A1A7C012A05D1BD
:102368005B681A888A421BD1187F30BD052A06D1BE
:102378005B681A888A4213D193F82C0030BD032A6F
:1023880006D15B681A888A420AD193F8250030BDC5
:10239800062A05D15B681A888A4201D1D87A30BDED
:1023A80001340430AC42D7D3002030BD08B1817568
:1023B80001207047F8B504460D46D0B1E175D0F854
:1023C80098309847012D0DD12746002606E0F86978
:1023D80000F10802436906CA98470136238B04377F
:1023E8009E42F4D3D4F898302046294698470120D5
:1023F800F8BDF8BDF8B50546084617460E4611F073
:1024080027FD013FB84234BF04463C463CB128464C
:102418003146224611F09EFD00232B55F8BD2C7045
:10242800F8BDF7B5044600200090019000296CD053
:102438000E8B68E000F1080351F823301D7C042D51
:1024480004D15D682D88954247D0013000F108031A
:1024580051F823301D7C012D04D15D682D889542EB
:102468003BD0013000F1080351F823301D7C052DC5
:1024780004D15D682D8895422FD0013000F1080302
:1024880051F823301D7C032D04D15D682D889542B9
:1024980023D0013000F1080351F823301D7C022DB0
:1024A80004D15D682D88954217D0013000F10803EA
:1024B80051F823301D7C072D04D15D682D8A954283
:1024C8000BD0013000F1080351F823301D7C062D94
:1024D80008D15D682D88954203D103F10801204693
:1024E80015E0013000F1080351F823502B7C082B2C
:1024F80009D16F683F88974204D105F10801204649
:102508001A4605E00130B04294D3204669460822B5
:1025180011F056FB2046FEBDF8B505460F46164697
:10252800002830D04388032B2FD0202011F098F8B2
:10253800044600282BD040F80C5B39460C22FFF7E4
:1025480059FF1820E66111F08BF80646B8B102234E
:102558000374012363760F4B446063600E4BA360E2
:10256800002323766B8805EB830201339BB2012B92
:1025780050606B800CD16A685268137608E0204678
:1025880011F076F804E0064602E0002600E0064670
:102598003046F8BDEC5B04088A58040837B545682E
:1025A80002AB03E906003DB3037C0124042B85F844
:1025B800314022D1688E02F029FC95F8300002F0F3
:1025C80027FD95F8343043B9BDF80200BDF8061070
:1025D800AA1C234602F054FD0FE0012B03D1084842
:1025E80040F2395104E0022B07D1054840F241512D
:1025F800044A054B01F0BCF92C4620463EBD00BFFD
:1026080017A105086027040815A10508F8B50446B0
:102618000F46164610B3838A0A2B20D0202011F0CB
:102628001FF80546E8B14460102200F10800394659
:10263800FFF7E0FE4FF6FF73A08A2B801F236B8005
:1026480000232B76831D013080B20128EE6144F807
:102658002350A08207D1A3691876F8BDF8BD0020E1
:10266800F8BD0120F8BD0120F8BD2DE9F3471D464E
:102678004B1C984282460C461746BDF828600DDD73
:1026880095420BDC01320AF101035B1A521BC8B2F6
:10269800D2B29BB22946009602F0F0FBAAF1020AD8
:1026A8003046C4EB0A0A02F0B1FB4FF000084FF0C5
:1026B80001091FFA8AFA0BE0601C08EB050180B2D9
:1026C80089B252460023009602F0D0FB09F10109B5
:1026D8007B1B08F1010899451FFA88F8ECD3BDE87F
:1026E800FC87F8B5C7B2144638461E460D4602F0B8
:1026F800CFFB621E92B23846294602F0C9FB30462B
:1027080002F084FB022606E0A21B92B23846294654
:1027180002F0BEFB0136A642F6D3F8BD73B50446F7
:102728000E4600F11E001546009200233C2280B29E
:102738001E3E02F09BFBB1B220463C2201230095CD
:1027480002F094FB7CBD73B504460E46013815466D
:1027580000920023032280B2013E02F087FBB1B24F
:10276800204603220123009502F080FB7CBDF7B5CB
:10277800089D2E7BEF7A1C463604AB7A06EB0726BB
:10278800F618431A687B06EB00602D1800200190AC
:10279800121B08462146009501F060FFFEBD30B5CA
:1027A800456885B004AB03E906007DB101242C73AC
:1027B8006D68BDF80800BDF80A109DF80C209DF85A
:1027C8000E300095FFF7D3FF204600E0284605B0FD
:1027D80030BD2DE9F04385B004AB03E90600446839
:1027E800BDF80860BDF80C70002C41D0012384F8B6
:1027F800263094F825300BB9A26800E06268FFB271
:10280800BDF80A109DF80E30009230463A46FFF7A0
:10281800AEFF04F10C08022002F0FAFB404611F06A
:1028280017FB054600B1451E0F3F0024153E1FFA51
:1028380087F90DE002F0F6FB02F0FAFB04FB1061E9
:1028480089B248462022002302F034FC0134E4B265
:10285800AC42EFD3002002F0D9FAB8B2B1B2424686
:10286800012302F027FC002002F0D2FB012000E047
:10287800204605B0BDE8F0832DE9F04385B004ABF0
:1028880003E906004568BDF80860BDF80C70002D26
:102898003CD001236B762B7EBDF80A10012B0CBFB0
:1028A8006A68AA689DF80E300092FFB23A46304630
:1028B800FFF75DFF0C35022002F0AAFB284611F055
:1028C800C7FA0E3F81460024163E1FFA87F80DE02E
:1028D80002F0A8FB02F0ACFB04FB106189B2404691
:1028E8002022002302F0E6FB0134E4B24C45EFD984
:1028F800002002F08BFAB8B2B1B22A46012302F0E6
:10290800D9FB002002F084FB012000E0284605B036
:10291800BDE8F0832DE9F04F85B00546DDF840901D
:10292800029148469046039311F092FADDF838A0D8
:10293800DDF83CB00646294600242F4611E024B1B4
:10294800B4420CBF5B46534600E0039B01F1080507
:10295800ADB200932846029A4346FFF708FF0134B8
:102968002946B442EBDD002002F050FA022002F0C2
:102978004FFB7D1D08F10508A8B21FFA88F14A46E9
:10298800012305B0BDE8F04F02F07ABB70B540688E
:1029980086B006AB03E9060000282ED0012380F894
:1029A8002D308668164BF21A534243EB020390F817
:1029B8002C205AB1002B134D134B144A08BF1D4647
:1029C800134B00F11C0418BF13460AE0002B0D4DF1
:1029D8000D4B0E4A18BF1D460D4B00F10C0408BFE5
:1029E8001346BDF81200BDF81410BDF81620009665
:1029F80001950294FFF78EFF012006B070BD00BF5D
:102A0800D03004080C2D0408B2320408EE2E040855
:102A18009434040870B5446886B006AB03E9060030
:102A280004B301236377A668104B227FF11A4B4247
:102A380043EB01030AB10BB904E01BB966680C4DFE
:102A48000C4B01E00C4D0D4BBDF81200BDF81410F5
:102A5800BDF8162000960C3401950294FFF75AFF32
:102A6800012000E0204606B070BD00BF1C3C0408F1
:102A7800583804083A3A0408F23D0408C83F0408E4
:102A88002DE9F04385B004AB03E906004468BDF8BE
:102A98000860BDF80A90BDF80C50BDF80E80002CF7
:102AA80000F08C800123A3740220676802F0B0FA5A
:102AB8004FF6FF7002F0C0F9002002F0A7F9EDB25E
:102AC8005FFA88F8A6F1160189B230462A464346CD
:102AD8000097FFF74CFE277A002F2ED1A28A2346B3
:102AE80000E00137974204D29969097E043300292E
:102AF800F7D002F097FA02F09BFAA9F116091FFA2B
:102B080089F90E2101FB10914FF6FF7208F10108B7
:102B18005FFA88F389B2009248462A46FFF7A5FD76
:102B2800022002F075FA1F2002F070F9A38A002B28
:102B380038D0103DE8B2303E2CE0E3685C68A28AE9
:102B48002346013A002700E00137974204D29969E9
:102B5800097E04330029F7D002F064FA02F068FA1B
:102B68000E2101FB10914FF6FF7208F101085FFA80
:102B780088F389B2009248462A46FFF776FD02207C
:102B880002F046FA1F2002F041F9A38A53B1103D22
:102B9800E8B21A3E0637B1B254F8272001230832AA
:102BA80002F088FA002002F033FA4FF6FF7002F0C4
:102BB80043F91F2002F02AF9012000E0204605B061
:102BC800BDE8F0832DE9F0410546362088461446D5
:102BD8001F4610F045FD0646E0B120F8025B41466D
:102BE8002E22FFF707FCBDF8183086F834407386AC
:102BF8001820012386F8307086F8313010F030FD47
:102C0800044618B104234660037404E0304610F00B
:102C18002FFD00E004462046BDE8F081F8B50646E1
:102C280024200F46154610F01BFD0446D8B10F4B63
:102C3800068083600E4B39464360102200F10C0079
:102C4800FFF7D8FB01260023182025622377667733
:102C580010F006FD054610B14460067404E02046F5
:102C680010F006FD00E005462846F8BD1C3C0408A7
:102C780076360408F8B506462C200F46154610F09F
:102C8800EFFC0446E8B120F80C6B39461922FFF72F
:102C9800B1FB0D4BA562A3600C4B6360002384F865
:102CA80025301820012384F8263010F0D9FC054679
:102CB80018B103234460037404E0204610F0D8FCE4
:102CC80000E005462846F8BD28550408C651040802
:102CD80010B50446142010F0C3FC20B10023438033
:102CE800014B0480036110BD2125000838B5054655
:102CF800442010F0B5FC0446C0B10E4B0582436079
:102D08000D4B0360012383740023037283820B4BF2
:102D18000364182010F0A4FC054618B1072344608A
:102D2800037404E0204610F0A3FC00E005462846A2
:102D380038BD00BFBC4D0408B24904081526000878
:102D48002DE9F04105463420884614461F4610F008
:102D580087FC064620B3144B05808360134B41461D
:102D68004360102200F10C00FFF744FB214606F1F6
:102D78001C001022FFF73EFB002386F82C30182099
:102D88000123376386F82D3010F06AFC044618B129
:102D980005234660037404E0304610F069FC00E047
:102DA80004462046BDE8F081D03004082A2B0408E8
:102DB8002DE9F041044614200D461646984610F0B9
:102DC8004FFC0746B8B1069B048003610023C37219
:102DD80001234560068180F80A800373182010F0EB
:102DE8003FFC044618B106234760037404E03846E4
:102DF80010F03EFC00E004462046BDE8F0812DE9D5
:102E0800F041044618200D461646984610F028FC56
:102E18000746B8B101238370069B04800361079BB2
:102E280045608660C0F80C804361182010F018FCDB
:102E3800044618B108234760037404E0384610F0CC
:102E480017FC00E004462046BDE8F0812DE9F34177
:102E580098461B8B1D2B05460C4617464FF0000065
:102E680000F2B480B5F5A07F0090019000F2AE802A
:102E7800F02900F2AB80127CADF80610511EADF8B7
:102E88000250072900F28A80DFE801F045595E0404
:102E9800456A14767B684E4A7A611A8893F834300A
:102EA8003A80013BDBB2012B7FD8ADF80240ADF888
:102EB80006507AE005F11602ADF8002004F116027A
:102EC800ADF8042002AE434A16E903007A6107F11F
:102ED800080282E8030003F10802013348F822706F
:102EE800A8F818307B681A8A187A3A8000286CD1BA
:102EF800FFF7FCFE3849436859603849DF6001260E
:102F0800163D196002461E72A8B2E1B24346FFF7A9
:102F18009DFF30465AE0012A0CBF314B314B78688F
:102F28007B6130F80C3B3B8010F092FF431CDB00C8
:102F38001A34ED18ADF80440ADF8005035E07B6860
:102F4800294A1B687A6102E0284A7B687A611B88F3
:102F580014353B80ADF800501434ADF8044024E03B
:102F68007B68234A7A611A883A801A899B7AAD1855
:102F7800ADF80050E418F0E77E681E4B7B6133889B
:102F880038463B8073689847013D4519ADF80050B5
:102F9800B36838469847013C0419DEE71648174AD3
:102FA800174B40F21A3100F0E3FC02AA12E90300C1
:102FB80007F1080383E80300B8F8183003F10802A2
:102FC800013348F82270A8F818300120BDE8FC81C8
:102FD800A5250008892A0008A84504089E41040878
:102FE8001D2A00089529000881280008DB27000809
:102FF800A72700083123000817A10508702704082F
:1030080015A10508F8B51646002834D01378002B0A
:103018002ED0028B002327E0046A257C042D21D1C1
:1030280065682F888F421DD195F8313053B16F8E66
:1030380001F012FF04F1080268866369204606CA97
:1030480098476F86A81C31462E22FFF7D3F995F8CA
:1030580031307BB104F108026369204606CA9847FB
:103068000120F8BD013304309342D5D30020F8BDC8
:103078001846F8BD0120F8BD70B5B8B1068B0446F6
:10308800002310E0256A287C04280AD16D68288866
:10309800884206D11046A91C2E22FFF7ABF9012061
:1030A80070BD01330434B342ECD3002070BD38B591
:1030B800044620B3134BC361134BC0F89830134B2D
:1030C800C0F89C30124B00257822C0F8A0308575D6
:1030D800C5750583294600F1200010F0B3FDD4F82A
:1030E80098302046294698470A4A1388312B07D832
:1030F800094941F8234001331380012038BD38BD08
:10310800284638BDBD230008B5230008552300080C
:103118002B240008740D0020201700202DE9F04111
:103128000446002800F0B380078B02460025A8E07B
:10313800136A1E7C042E00F08780012E23D1586864
:1031480003888B4240F09B8005F1080710F090FA45
:1031580054F827004FF00008C0F8048010F088FAEF
:10316800228B531E9D4208D00732238354F8221025
:1031780044F8271044F8228002E044F82780258389
:103188003046BDE8F081052E5ED0032E5CD0022EBD
:1031980013D15B68186803888B4270D14388013B60
:1031A8009BB243800BB910F063FA05F1080654F896
:1031B8002630586810F05CFA4EE0072E21D15E6880
:1031C800338A8B425BD1002706E0BB1D013756F8D6
:1031D800230010F04DFAFFB2B38ABB42F5D800279E
:1031E800B78205F1080654F82630586810F040FAFE
:1031F80054F8260033E044F8267025830120BDE802
:10320800F081062E1ED1586803888B4237D105F10C
:10321800080610F02DFA54F826000027476010F031
:1032280027FA228B531E9D4209D00833013A54F8DD
:103238002310228344F8261044F82370DEE744F86C
:1032480026701AE0082E1AD1586803888B4216D1C6
:1032580010F00EFA05F1080654F82600002747601A
:1032680010F006FA228B531E9D42C4D0073254F840
:10327800221044F8261044F822702383BEE7013553
:103288000432BD42FFF454AF0020BDE8F081BDE830
:10329800F08170B5044600282AD0068B751E0836C2
:1032A80000EB86061EE056F8043D1A7C042A13D06B
:1032B800012A11D0052A0FD0032A0DD0022A02D1E3
:1032C8005B681B6809E0072A02D15B68198A05E078
:1032D800062A01D0082A04D15B6819882046FFF71E
:1032E8001DFF013D681CDED100232383012070BD32
:1032F80070BDF0B528B30023068B1A461EE0046A99
:10330800257C072D18D16468258A8D4214D1A78A97
:10331800002504EB83040DE004EB050C0435DCF810
:1033280018C09CF818C0BCF1010F03F1010301D1CA
:10333800D8B2F0BDBB42EFD301320430B242DED383
:103348000020F0BD70B508B3048B00231BE0026AAF
:10335800157C072D15D15268158A8D4211D100238D
:10336800958A11461C46012007E013B99669307604
:1033780001E08E69347601330431AB42F5D3012084
:1033880070BD01330430A342E1D3002070BD2DE9A4
:10339800F04128B30023078B1A461EE0046A257CF7
:1033A800072D18D16468258A8D4214D1B4F814C049
:1033B800002504EB83040CE066190435B66996F819
:1033C8001880B8F1010F03D106F10800BDE8F081BB
:1033D80001336345F0D301320430BA42DED3002012
:1033E800BDE8F0812DE9F04700282FD00023B0F880
:1033F80018C01D4627E0046A267C072E21D1646880
:10340800268A8E421DD1B4F81480002604EB830965
:1034180015E009EB0604A7693C7E012C0DD192F852
:1034280000A0BAF1000F08D007F1080011461022D9
:10343800FEF7E0FF2046BDE8F08701330436434538
:10344800E7D3013504306545D5D30020BDE8F087C2
:10345800F0B5B0B1068B002510E0046A277C062F72
:103468000AD1646827888F4206D123819DF81430D9
:103478006260A3720120F0BD01350430B542ECD37F
:103488000020F0BD10B500210446FEF793FF20464A
:103498000121BDE81040FEF78DBF38B598B1048B07
:1034A800024600230CE0106A058804328D4206D1DA
:1034B80000F10802436906CA9847012038BD013364
:1034C800A342F0D3002038BD10B50C460021FEF70A
:1034D80071FF20460121BDE81040FEF76BBF13B510
:1034E80002AC04E90C00BDF80230834206D8BDF8EE
:1034F8000030834234BF0020012000E00020BDF8E6
:1035080006308B4206D8BDF804308B4234BF002108
:10351800012100E00021002818BF0846C0B21CBDE8
:1035280038B5114B114A1988002319E052F8045F85
:10353800A87D012812D100240CE004F1080355F8F5
:103548002300037C082B03D1436800211B6998479B
:103558000134A4B22B8BA342EFD838BD01339BB200
:103568008B42E3D138BD00BF740D00201C1700202A
:10357800704770B5094CA5787DB9094B1E78012EA6
:103588000BD16368013363606268064B9A4204D9C1
:10359800284601F0FFFCA670656070BD740D002020
:1035A8008401002040420F00054A9060134602E063
:1035B80099680139996091680029F9D1704700BF6D
:1035C800740D0020F0B585B001F092FF002800F0DE
:1035D8004981002502A80DF10A01ADF80850ADF89F
:1035E8000A5001F087FF03A80DF10E01ADF80C5049
:1035F800ADF80E5001F0CAFFBDF80C10BDF8082058
:103608000091BDF80E10BDF80A3001912C46964D78
:103618009649082008F004FFA878012803D101F092
:10362800B9FCAC7019E1924B5B78012B40F0158125
:10363800AB78002B40F011816B6029888D4A09E135
:1036480052F8046FB07D012840F002810025FAE0AD
:1036580005F10803BDF8080056F82340BDF80A1024
:1036680004F108030CCBFFF73AFF002800F0E980CB
:10367800237C013B062B00F29F80DFE803F004293E
:10368800159D1F9D4C006668012304F108053377DA
:1036980095E806006369204698470023337720465B
:1036A800636995E8060086E0636893F8252012F1BF
:1036B800FF3218BF012283F8252077E0636893F86A
:1036C8002C2012F1FF3218BF012283F82C206DE064
:1036D8006268137E1568002B6ED16E882F462946C6
:1036E800184606E051F804EFDEF804E001338EF8DE
:1036F8001800B342F6D301231376002607E057F8E3
:10370800040F00F10802436906CA984701366B881E
:103718009E42F4D350E0656820892E68A37B227B03
:103728000096A0F1160189B2FFF721F81420FFF7DF
:103738003BFF2B7AC3B9AF8A29461A461E4609E0D1
:10374800886990F818E00676BEF1010F08BF1346A5
:1037580004310132BA42F3D301220BB9AB6924E038
:10376800053355F8233020E06368DB685A68002386
:10377800908A154619461F4609E0AE6996F818E082
:103788003776BEF1010F08BF0B460435013181427F
:10379800F3D3411E8B4203D1053052F8203003E0A9
:1037A80004D2073352F8233001221A7604F10802B2
:1037B80006CA636920469847237C013B072B4CD8EF
:1037C800DFE803F00410074B0A0D123A63681B6A1E
:1037D80034E063689B6A2DE063681B6B2AE06368CA
:1037E8001B6927E0636824E063681A7A7AB9988AC3
:1037F8001946013800E00132824204D28C69247EE5
:103808000431002CF7D0063253F8223011E0DB687F
:103818005A68908A11460138002300E00133834238
:1038280004D28C69247E0431002CF7D0063352F878
:103838002330DB69984710E06368DB6820469847C7
:103848000BE00135ADB2338BAB423FF601AF04E07C
:1038580001339BB28B427FF4F3AE01F08FFE0F2051
:10386800FFF7A2FE05B0F0BD740D00203DA10508CC
:10387800840100201C170020034B9A6812B19A6833
:10388800013A9A60704700BF740D00202DE9F34794
:103898000120DFF8D080DFF8D09001460AF05AF90D
:1038A800012400254FF48076022740466946009699
:1038B8008DF804708DF805408DF806508DF8074096
:1038C80009F0A0FD40460821224609F01BFE244BC2
:1038D800DFF898801A6844F2A243B2FBF3FA0AF1BF
:1038E800FF3A204621461FFA8AFA0AF063F9C8F817
:1038F80004A048464146A8F80050A8F80250A8F885
:10390800085088F80A500AF0F1FC7023A8F80C3027
:103918000423A8F810300AF1FF3A6323642203FB5A
:103928000AF3B3FBF2F39BB2C8F8143008F10C01A8
:103938004846A8F80E40A8F81870A8F81A50A8F831
:103948001C60A8F81E500AF0EFFD484621460AF010
:1039580062FD484621460BF068F8BDE8FC8700BFC9
:10396800F00200200000024000000140840D002009
:1039780083B50E460746154910201C46154608F023
:103988004FFD1020124908F04BFD1020114908F096
:1039980047FD10200E4908F043FD002310200E4972
:1039A800019308F03DFD334610200C493A4608F0D3
:1039B80037FD10200A492A4608F032FD102009492F
:1039C800224608F02DFD019B0133E7E777A10508A2
:1039D8007CA105089CA10508ACA10508BCA10508A7
:1039E800D1A10508E2A1050808B5164B1A6A0132EB
:1039F8001A621A6A012A1A4603D0134840F20721AC
:103A08000FE05862194602E04B6A013B4B62506A6C
:103A18000C4B0028F8D11A6A012A06D00A4840F24D
:103A280012210A4A0A4BFFF7A3FF1A6A013A1A62DF
:103A38001B6A2BB10448054A064B4FF40571F2E79F
:103A480008BD00BF840D0020F3A105084E5F0408DF
:103A58001DA205082EA2050810B5084C0221002257
:103A6800204609F044FD44F6FF70FFF7BDFF2046ED
:103A780002210122BDE8104009F039BD00040240CE
:103A88000C4B0D491A6844F2A2436428B2FBF3F3C5
:103A9800D4BF20EAE0706420013B9BB24B60013B3D
:103AA80058436422B0FBF2F080B2486103480C31FD
:103AB8000AF0BDBCF0020020840D00200000014087
:103AC80010B5134B93F828202AB11248124A134B09
:103AD80040F2F2210EE0012283F8282066234FF0FD
:103AE800C042013BDBB2108033B90A480A4A0C4B8A
:103AF8004FF43F71FFF73CFF1488A4B28442F0D121
:103B0800084B1980024B002283F8282010BD00BF03
:103B1800840D0020F3A10508585F04083FA205089A
:103B280015A105080000026010B5FFF7AFFE64207C
:103B3800FFF7A6FF21210720FFF7C2FF3220FFF77A
:103B480053FF01210020FFF7BBFF3220FFF74CFF96
:103B580023210720FFF7B4FF3220FFF745FF00219C
:103B68001020FFF7ADFF41F28830FFF73DFF33210A
:103B78000720FFF7A5FF3220FFF736FF112046F692
:103B88003001FFF79DFF3220FFF72EFF4FF4C06191
:103B98000220FFF795FF3220FFF726FF122046F696
:103BA800EB41FFF78DFF3220FFF71EFF03204AF697
:103BB800A401FFF785FF3220FFF716FF00210C2034
:103BC800FFF77EFF3220FFF70FFF0D2040F60C01B4
:103BD800FFF776FF3220FFF707FF0E204FF42C5136
:103BE800FFF76EFF3220FFF7FFFEB0211E20FFF720
:103BF80067FF3220FFF7F8FE012042F63F31FFF75A
:103C08005FFF3220FFF7F0FE05200021FFF758FF85
:103C18003220FFF7E9FE00210620FFF751FF32208E
:103C2800FFF7E2FE16204EF61C71FFF749FF32201F
:103C3800FFF7DAFE172040F20311FFF741FF3220A9
:103C4800FFF7D2FE00210B20FFF73AFF3220FFF7E3
:103C5800CBFE00210F20FFF733FF3220FFF7C4FE11
:103C680041200021FFF72CFF3220FFF7BDFE422044
:103C78000021FFF725FF3220FFF7B6FE002148207C
:103C8800FFF71EFF40F23F143220FFF7ADFE21463A
:103C98004920FFF715FF3220FFF7A6FE00214A2032
:103CA800FFF70EFF3220FFF79FFE00214B20FFF7A2
:103CB80007FF3220FFF798FE44204FF46F41FFF7CB
:103CC800FFFE3220FFF790FE00214520FFF7F8FEA7
:103CD8003220FFF789FE21464620FFF7F1FE322009
:103CE800FFF782FE302040F20771FFF7E9FE32202D
:103CF800FFF77AFE31204FF40171FFF7E1FE322021
:103D0800FFF772FE32204FF40171FFF7D9FE40F23F
:103D180002543220FFF768FE21463320FFF7D0FE19
:103D28003220FFF761FE342040F20751FFF7C8FE4A
:103D38003220FFF759FE35204FF40171FFF7C0FE1E
:103D48003220FFF751FE36204FF40171FFF7B8FE1D
:103D58003220FFF749FE21463720FFF7B1FEA4F5D0
:103D680000743220FFF740FE21463A20FFF7A8FEF4
:103D78003220FFF739FE2F2041F2BE21FFF7A0FEC7
:103D88003220FFF731FE21463B20FFF799FE322013
:103D9800FFF72AFE00212320FFF792FE3220FFF7CB
:103DA80023FE00212420FFF78BFE3220FFF71CFEA4
:103DB80025204FF40041FFF783FE3220FFF714FE61
:103DC80000214F20FFF77CFE3220FFF70DFE4E202A
:103DD8000021FFF775FE3220BDE8104004E608B563
:103DE800124B93F829202AB11148124A124B4FF46A
:103DF80043710FE0012283F82920222166234FF026
:103E0800C042013BDBB2118033B90948094A0B4B68
:103E180040F22531FFF7ACFD108880B22228F0D19E
:103E2800024B002283F8292008BD00BF840D002022
:103E3800F3A10508655F04083FA2050815A1050858
:103E480010B51E4B032826D8DFE800F0021A080E2A
:103E58001C8841F2280246F628000AE01C8841F234
:103E6800080246F6080004E01C8841F2300246F6D3
:103E7800300049F241318C4214BF014611460BE033
:103E8800188846F6200249F24131884214BF11468B
:103E98004FF4815100E000211B8848F689129342B3
:103EA80005D049F22032934204D1032000E01120CA
:103EB800FFF706FEBDE8104091E700BF860100202D
:103EC800014B18800A208FE5000002604FF0C043C4
:103ED800188003F500331A881A88188880B270474A
:103EE8004FF0C04322221A8003F5003382B01A88AB
:103EF80092B2ADF806201B889BB2ADF80630BDF82B
:103F0800060080B202B07047072040F27311D7E56F
:103F180007200021D4E582B0044BADF80600BDF8B7
:103F2800062092B25A8502B0704700BF840D002067
:103F380082B0044BADF80600BDF8062092B25A8054
:103F480002B0704786010020014B80B2188070478C
:103F5800000002604FF0C04380B218807047024BE7
:103F680080B21880704700BF000002604FF0C04365
:103F780080B218807047024B80B21880704700BF2B
:103F88000000026082B0044B0190019ADA62DA6A9A
:103F9800002AFCD102B07047840D002070B54FF0A4
:103FA800C0452A242C800A4C060AC0B226802080EC
:103FB800100AD2B2208022802B222A800A0A22806C
:103FC800C9B21A0ADBB221802280238070BD00BFEB
:103FD8000000026010B50B4614460246FFF7DEFFEC
:103FE8004FF0C0432C22A0B21A80BDE8104067E70A
:103FF800114B1B8848F68912934210B504460BD022
:1040080049F22032934212D1C1F1EF01202089B246
:10401800FFF756FD212006E0C1F1EF014E2089B2DD
:10402800FFF74EFD4F202146BDE8104048E5024607
:104038000B46BDE81040B1E78601002008B5FFF740
:10404800D7FF0E4B1B78012B4FF0C0420C4B0FD102
:104058002E2111801A881A881B8892B202F0FC005F
:1040680002F4784242EAC000C3F3C423184308BDEF
:10407800222111801A88188880B208BD944800202F
:104088000000026070B5134B1C78012C05460BD15B
:10409800114E21462846FFF7D1FF0134A4B2C82C9F
:1040A80026F8020FF5D170BD0121FFF7A1FF01200D
:1040B800FFF7C6FE4FF0C04322221A80074A06497E
:1040C800138800231088C8520233B3F5C67FF9D18C
:1040D80070BD00BF944800203E46002000000260EA
:1040E80010B5084B1B78012B144602D1BDE81040CF
:1040F80070E7FFF77DFFFFF772FE2046BDE810402E
:10410800DEE600BF9448002070B50E4B0E4D1C78BB
:10411800012C06460AD12146013435F8022F3046D3
:10412800A4B2FFF7DDFFC82CF5D170BD01242146EC
:10413800013435F8022F3046A4B2FFF7D1FFC72C5F
:10414800F5D170BD944800203E46002070B5054664
:104158000E46FFF797FF0C4B1C78012C09D121461E
:10416800013428463246A4B2FFF734FFC82CF6D1F2
:1041780070BD01242146013428463246A4B2FFF717
:10418800AFFFC72CF6D170BD944800202DE9F0414F
:1041980004460D461646BDF81880032B39D8DFE8CB
:1041A80003F00B351927381980B2294642460137E2
:1041B800FFF796FFBFB200E00027B742F3D1BDE892
:1041C800F081E01B80B2294642460137FFF788FF9D
:1041D800BFB200E00027B742F3D1BDE8F081E91B88
:1041E80089B2204642460137FFF77AFFBFB200E0A6
:1041F8000027B742F3D1BDE8F081791989B220468A
:1042080042460137FFF76CFFBFB200E00027B74214
:10421800F3D1BDE8F08170B5194B1A4A598E92F95D
:10422800004064180025A4B28AB0AC4208BF01243B
:10423800C62C28BFC62415700F264FF6FF721E869F
:104248005C865A8519202B46009221460A22FFF7E0
:104258009DFF21463046FFF7F1FE224603460A49F4
:1042680002A80FF06FFD02AA06A808490FF06AFD20
:104278003220D22106AA2B4600F002FF0AB070BDF8
:10428800840D0020DC2D002054A205085CA205083E
:104298002DE9F341BDF820500C4690461F461A46BA
:1042A800002306460095FFF771FF611E4144304622
:1042B8003A46002389B20095FFF768FF3046214649
:1042C800424601230095013EFFF760FFBF19B8B2CF
:1042D800214642460123089502B0BDE8F04155E762
:1042E8002DE9F0410D46C5F1F008411E5E18C2EBFC
:1042F8000802C5F1EF039BB292B2B6B29A422CBF44
:10430800904698469A4234BF11461946864234BFB1
:104318003746074640F23F13864238BF06469E425C
:1043280028BF1E46174B1B8848F68912B8F1EF0FB5
:1043380028BF4FF0EF089342044610D049F22032CC
:1043480093421AD15020FFF7BBFB51204146FFF79B
:10435800B7FB52203946FFF7B3FB53200AE041EA86
:10436800082189B24420FFF7ABFB45203946FFF707
:10437800A7FB46203146FFF7A3FB20462946BDE8A8
:10438800F04135E68601002000200146F0224FF476
:10439800A073A5E770B580B202FB03F489B292B2AC
:1043A8009BB2FFF79DFF0020FFF74AFD0025064E50
:1043B80004E0708D80B2FFF783FD0135A542F8DB7C
:1043C800BDE87040E0E700BF840D002070B54FF0F5
:1043D800C0452A242C80094C060A26802080080A19
:1043E800208021802B212980110A218022801A0A0D
:1043F800228023802C232B8070BD00BF0000026028
:1044080070B5114B1B78012B044607D1002040F2F0
:104418003F110246EF23FFF7D9FF04E0FFF7B4FF8F
:104428000020FFF70DFDF02509E0013E2046B6B259
:10443800FFF746FD002EF8D1013DADB215B14FF49E
:10444800A076F2E770BD00BF944800202DE9F04F38
:104458001C463E4B87B01B78039183469DF8441059
:1044680010980591012B039B049092461FFA8BF03C
:104478009AB208D1411E531E0919534489B29BB2FE
:10448800FFF7A4FF09E01FFA8AF51146A3B22A46EE
:10449800FFF726FF0020FFF7D3FC0027DDF80C808C
:1044A8003E4640F23F1CA14639E0BBF1000F2EDB2F
:1044B80065452CDC0398002829DBB8F1EF0F26DCD2
:1044C800220702D1002CC8BF01362149214000290A
:1044D80003DA013961F00F010131059A0AB1C1F11E
:1044E8000F01049830F8162003FA01F10A4012B2BD
:1044F8006AB118494A8D029392B2A8B21FFA88F19C
:10450800CDF804C0FFF7ECFDDDF804C0029B0134D0
:1045180001354C45C9DB0136013708F1010857451B
:1045280003DA5D4600240123F3E7084B1B78012BCF
:1045380008D1002040F23F110246EF2307B0BDE842
:10454800F04F43E707B0BDE8F04F1DE7944800205F
:104558000F000080840D00202DE9F74F1F463B4BCC
:10456800DDF830801B7816469DF83420012B044670
:1045780001920D4680B28AB208D1411E531EC91954
:104588009B1989B29BB2FFF721FF09E01FFA86FE4B
:104598001146BBB27246FFF7A3FE0020FFF750FC9E
:1045A8004FF0000BDA463DE0002C30DB09EB04034A
:1045B80040F23F1293422ADC002D28DB0BEB050367
:1045C800EF2B24DC19F00F0F04D1B9F1000FC8BF8D
:1045D8000AF1010A1E4B09EA0303002B03DA013B27
:1045E80063F00F030133019A0AB1C3F10F030122EB
:1045F80002FA03F338F81A2013401BB213B1154B13
:10460800588D01E0144A508880B2FFF759FC09F12F
:10461800010901E04FF00009B945C5DB0AF1010ABB
:104628000BF1010BB345F5DB084B1B78012B08D1C7
:10463800002040F23F110246EF2303B0BDE8F04FDF
:10464800C4E603B0BDE8F04F9EE600BF94480020E2
:104658000F000080840D0020860100202DE9F04124
:104668001C4F069C3F789DF81C60012F02FB03F548
:1046780080B28FB209D1411ECB1899B27B1E9A180D
:1046880093B23A46FFF7A2FE07E092B29BB23946D0
:10469800FFF726FE0020FFF7D3FB002709E034F8D8
:1046A800020B1EB1030A43EA002080B2FFF708FCA0
:1046B8000137AF42F3DB074B1B78012B07D10020F2
:1046C80040F23F110246EF23BDE8F0417EE6BDE827
:1046D800F04159E6944800202DE9F0431F2093B09B
:1046E800FFF78EFE4FF47840FFF78AFE4FF6E0752D
:1046F8004FF4FC60FFF784FE2846FFF781FE002098
:10470800514CFFF77DFE00204FF6FF7901466422E9
:104718000346A4F82A90CDF80090FFF737FD002053
:104728000A2164220346CDF80090FFF72FFD0020F0
:104738000146642201234FF4784765850095FFF709
:1047480025FD7720EF21C82200234FF4FC666785FA
:104758000097FFF71BFDBD213222012340F23F10D5
:1047680066850096FFF712FDA020322200237821EB
:1047780067850097FFF70AFDA020782132220123E0
:104788004FF01F0866850096FFF700FDA0207821EE
:1047980032220223A4F82A80CDF80080FFF7F6FC25
:1047A800A02078213222032365850095FFF7EEFCCF
:1047B800264B2749A3F8028002AD3C2228460FF079
:1047C800FFF9EB20C3210522302300950025A4F82A
:1047D8002A900195FFF7C0FE32210A2096220B4647
:1047E80067850097FFF754FD32213C2096220B463F
:1047F80066850096FFF74CFD32210B4696226E2007
:10480800A4F82A80CDF80080FFF742FDFFF780FB6F
:10481800FFF77AFB3220FFF733F92846FFF730F924
:104828006420FFF72DF90B4B03F110028DE82400EB
:1048380028465A681B682946FFF710FF1195119BF7
:1048480001331193FBE700BF840D0020860100208F
:104858007A5F0408008401082DE9F14FFFF716F884
:104868004FF0C0456420FFF70BF90127FFF7F4F874
:104878004FF028096D48FFF7B7F82F800520A5F8F5
:10488800009002F025FECF232B80694B002683225F
:104898001E801A8030221A80ED222A804FF0640888
:1048A8000322A3F800801A8012221A8081221A801B
:1048B800E8222A8085221A8079221F801A80CB223A
:1048C8002A8039221A804FF0340C02242C21F72236
:1048D80019801E80A3F800C01C802A8020221A801C
:1048E800EA222A80C0221E80C1211E802A80262218
:1048F8001A80298011211980C52129803521198024
:104908003E211980C7212980BE211980362129809E
:104918003A205521A3F8009028801980B1212980D8
:104928004FF0100BF2211E80A3F800B02980082157
:1049380019802A80E0221F804FF01F092A801A223E
:10494800A3F800904FF0180A1A800F210A22A3F842
:1049580000A01A8019800621198045211980872115
:1049680019803221198007211A804FF0E10E198031
:104978001C80052419801C801E80A5F800E04FF0DB
:10498800250E1E80A3F800E04FF0270EA3F800E0E4
:104998001C80A3F800B04FF0090BA3F800B04FF04B
:1049A800780B1880A3F800B04FF04D0BA3F800B0B7
:1049B8001C800D24A3F800A01C8038241C801880BB
:1049C8002A20A3F80090EF2428802B201E801E8028
:1049D8001E801C8028803F201E801E801F8018801B
:1049E800B720A5F800C028801980B62129801A8030
:1049F80082221A801122A3F800E040461E8029274F
:104A08002A8002F065FD40462F8002F061FD0948CA
:104A1800FEF7EAFF2C232F8030462B8040F23F110F
:104A28003246234601B0BDE8F04FCFE4400D030005
:104A38000000026040420F002DE9F041022098B0CA
:104A48000121002409F086F80125022680481696DF
:104A580016A98DF85D408DF85E408DF85F408DF8A1
:104A68005C5008F0CFFC1820294609F073F8284656
:104A7800294609F087F821460C22764808F042FDBD
:104A88000C227448294608F03DFD04210C22714887
:104A980008F038FD05210C226E4808F033FD072187
:104AA8000C226C4808F02EFD08210C22694808F0F9
:104AB80029FD09210C22674808F024FD0A216548D0
:104AC8000C2208F01FFD0B2162480C2208F01AFD89
:104AD8000E210C225F4808F015FD0F210C225D48BD
:104AE80008F010FD07210C225B4808F00BFD082197
:104AF8000C22594808F006FD09210C22564808F0F6
:104B080001FD0A210C22544808F0FCFC0B210C2260
:104B1800514808F0F7FC0C210A464F4808F0F2FC0F
:104B28000D210C224C4808F0EDFC0E210C224A48BD
:104B380008F0E8FC0C2248480F2108F0E3FC4CF68A
:104B4800B3734448169316A98DF85C608DF85E40DF
:104B58008DF85F408DF85D5008F054FC16A94FF6AB
:104B680080733D4816938DF85C608DF85E408DF833
:104B78005F408DF85D5008F045FC40F6B830FEF710
:104B880033FFFEF769FF40F6B830FEF72DFF0F231D
:104B980011934FF4805310270DF13C080993684690
:104BA8004FF40023109412941494159400940194D3
:104BB8000294039704940694079408940A9405941D
:104BC8000B940C93CDF834800F95139508F093F956
:104BD8000523684611930F96109412941494159413
:104BE800CDF83880139508F086F92946204608F054
:104BF80002FA40F6B830FEF7F7FE2046FFF766F9EE
:104C080004461649164E3846224607F009FC41F27A
:104C180089239C4248F68918124F01D044450ED189
:104C2800FEF782FF00233B70A6F8008010200E4993
:104C380048F6891241F2892307F0F2FB05E0FFF7F5
:104C48000BFE49F241333D70338018B0BDE8F08166
:104C580000040240000C02400010024061A2050856
:104C6800860100209448002078A205084FF0C04330
:104C780036221A8003F50033012814BF6820482023
:104C88001880704770B5244B01228CB01A7000242C
:104C98000AE0A9B21F2230460135FFF721FA642D38
:104CA800F7D10134642C02D00025A6B2F1E73220F6
:104CB800014602460346FFF771F94FF0C0432E2222
:104CC8001A8003F5003300201A881C881D88A4B2B6
:104CD80000F09CF8ADB20023224600930F492B4602
:104CE80003A80FF02FF800230A20C82103AA00F018
:104CF800C7F904F0FC0204F4784444EAC20242EA28
:104D0800D522074903A80FF01DF80A20DC2103AAC1
:104D1800002300F0B5F9FEE794480020B7A2050883
:104D2800CFA205082DE9F04F40F23F19484534BF9E
:104D380004464C46EF2B34BF98464FF0EF084A45DF
:104D480038BF9146EF2934BF0D46EF25C4EB090A59
:104D5800C5EB080785B0BAF1000FB8BFCAF1000A61
:104D6800002FB8BF7F424FF6FF734C452CBF1A4641
:104D780001221FFA8AFA454538BF0123BFB20293C0
:104D88000FFA8AF63BB29E42BDF838B0019202DDB6
:104D9800C6F34F0607E0022693FBF6F67642B6B254
:104DA80001E01E4603E00FFA8AF35B420393144ABC
:104DB8001378022B204629465A4602D1FDF7C3FC38
:104DC80001E0FFF78DF94C4501D1454514D0039A10
:104DD80033B2934205DD019AF31BA4189BB2A4B227
:104DE80000E0334636B23AB29642DADA029A5344CF
:104DF800AD189BB2ADB2D4E705B0BDE8F08F00BFE7
:104E0800B844002000487047F417002082B0064BD1
:104E1800ADF80600BDF8062092B21A80188880B254
:104E280002B0FFF778B800BFF0170020014B1888D0
:104E380080B27047F017002082B0064BADF806002C
:104E4800BDF8062092B21A80188880B202B0FFF727
:104E58006FB800BFF2170020014B188880B2704766
:104E6800F2170020FFF7CCBAFFF73ABA10B5BDF831
:104E780008400294BDE81040FFF788B910B5BDF8A6
:104E880008400294BDE81040FFF702BAFFF782BA63
:104E98002DE9F04F4FEA420800253D4C85B0824687
:104EA8008B46C8F1030817462E461FFA87F909EB07
:104EB8000B0C228805EB0A031FFA8CFC9BB2614697
:104EC800184692B2CDF804C00293FFF709F9C9EB6E
:104ED8000B0292B20392029B22880399184692B25F
:104EE800FFF7FEF8DDF804C02288C5EB0A039BB281
:104EF8006146184692B20293FFF7F2F8029B2288A5
:104F08000399184692B2FFF7EBF805EB0B0292B241
:104F1800039209EB0A03228803999BB2184692B2BE
:104F28000293FFF7DDF8029B2288C5EB0B0C1FFAF2
:104F38008CFC1846614692B2CDF804C0C9EB0A0948
:104F4800FFF7CEF8228803991FFA89F992B24846EA
:104F5800FFF7C6F82288DDF804C092B248466146D9
:104F6800FFF7BEF8B8F1000F04DA08EB860808F17D
:104F7800060805E0F31B08F10A0808EB8308013F5F
:104F880001360135BE42ADB28FD905B0BDE8F08F0C
:104F9800F017002008B9FEF7BBBF012801D1FEF7C2
:104FA800B3BF7047704700200146F0224FF4A0734A
:104FB800FFF796B9704708B505280CD8DFE800F068
:104FC800121403050709094808BD094808BD09481E
:104FD80008BD094808BD0948094A0A4B40F2411171
:104FE800FEF7C6FC084808BD084808BD7401002043
:104FF800640100205C01002054010020DAA20508A9
:10500800B65F040815A105087C0100206C0100208A
:1050180010B50446FFF7CFFF014B18601C7110BD97
:105028008C010020014B1879704700BF8C010020CB
:1050380008B5FFF7C0FF808808BD08B5FFF7BBFFBC
:10504800C08808BDF7B51F460B4B0C4E1D681446AB
:10505800EA882B68203C5443A4B2AE1B03EB4404FB
:1050680018BF0126AB888DE8500017B1FFF7EEF99D
:1050780001E0FFF771FAFEBD8C0100207C010020E1
:105088002DE9F0410F46984615460446084E08E0BB
:10509800204643463946FFF7D5FF33689B88E41816
:1050A800A4B215F8012B002AF2D1BDE8F08100BFA7
:1050B8008C01002010B5044608462146BDE8104082
:1050C800DEE7094B70B5044618790E461546FFF71A
:1050D800B4FFC6F1F001091A89B220462A46002316
:1050E800BDE87040CCE700BF8C010020704700BFCE
:1050F800044B1A680AB9044A1A601A68101818602A
:1051080010467047B80D00200C5200204FF0FF30B9
:10511800704708B50248034A034B3721FEF728FCBD
:10512800F9A20508CC5F040815A1050801207047FD
:1051380010B504460A48022108F092FF0028F9D069
:105148000748214608F055FF0548012108F088FF67
:105158000028F9D00248BDE8104008F047BF00BF5A
:105168000038004010B51948022108F079FF0028DE
:10517800F9D01648002108F03CFF1448012108F036
:105188006FFF0028F9D0114808F030FF0402A4B2DC
:10519800002301E001339BB2002BFBD00B48022116
:1051A80008F05EFF0028F9D00848002108F021FF28
:1051B8000648012108F054FF0028F9D0034808F0F8
:1051C80015FF2043C0F3CB0010BD00BF00380040DE
:1051D8002DE9F0478AB00AAF0A20012108F0BAFC8D
:1051E8004FF4604347F8143D474EDFF824A10124EB
:1051F80000254FF00208304639468DF81A508DF8D0
:1052080018808DF819808DF81B4008F0FBF830469F
:105218000D21052208F076F930460E21052208F006
:1052280071F9052230460F2108F06CF921464FF438
:10523800804008F0B3FC504608F08EFD4FF48273AE
:10524800ADF802304FF40073ADF80A303823ADF8EA
:105258000C30504607236946ADF81030ADF80050C1
:10526800ADF80450ADF80650ADF80850ADF80E5042
:1052780008F0A4FD5046214608F03BFEA9468DF8EB
:105288001A5030464FF48055394605958DF8184028
:105298008DF819808DF81B4008F0B4F8304629467F
:1052A80008F021F94025394618488DF818908DF8EE
:1052B80019808DF81A908DF81B40059508F0A2F812
:1052C80021464FF4804008F075FC0621032008F0C1
:1052D800FFFE0C2307A88DF8213007958DF8209044
:1052E8008DF8224007F082FD17238DF8243009A895
:1052F8000F238DF825308DF826308DF8274002F0E1
:105308006BFB0AB0BDE8F08700040240000C0240C5
:1053180000380040014B1878704700BFBC0D0020D2
:10532800024B5A889B8802800B807047BC0D002076
:10533800014B00221A707047BC0D0020F0B593B0E5
:105348006846002148220EF07DFC6D460024644822
:105358004FF4805108F0C9F8002301E001339BB2F3
:10536800002BFBD09020FFF7E3FE002301E0013380
:105378009BB2002BFBD0FFF7F5FE4FF48051074698
:10538800574808F0B0F8002301E001339BB2002B26
:10539800FBD053484FF4805108F0A7F8002301E0F0
:1053A80001339BB2002BFBD0D020FFF7C1FE0023B6
:1053B80001E001339BB2002BFBD0FFF7D3FE4FF483
:1053C80080510646464808F08EF845F8047B0134BB
:1053D8002E6244484021E4B208F073F810B9092C51
:1053E800B5D101E0092C78D19DE80C00D218029BB8
:1053F80003980699D218049BC018059BC018079BF0
:10540800CB180899032490FBF4F092FBF4F25B1894
:1054180093FBF4F3151AC11A9C1A002DB8BF6D42FC
:105428000029B8BF4942002CB8BF6442502D03DDA3
:10543800502909DD502C50DC8D4205DAAC424FF082
:10544800020405DB111806E08C424FF0020401DA71
:10545800D11800E0C1180A9B099A0C980F9DD21820
:105468000B9BD2180D9BC0180E9BC018109BEB18F5
:10547800119D91FBF4F1032492FBF4F290FBF4F0FC
:105488005B1993FBF4F3161AC41A9D1A002EB8BFC1
:105498007642002CB8BF6442002DB8BF6D42502E32
:1054A80089B203DD502C09DD502D16DCA64205DA41
:1054B800B5424FF0020405DB131806E0A5424FF091
:1054C800020401DAD31800E0C318074A93FBF4F387
:1054D8009BB2938001235180137013B0F0BD00BFBD
:1054E80000040240000C0240BC0D00200000000037
:1054F800FFF710BFF7B505460C4601A80DF10601E8
:10550800FFF70EFF1B4BBDF80660BDF8040093E8DB
:105518000600724301FB002299685218164992FB53
:10552800F1F207EE102AF8EEC77A40F23F17FCEEC8
:10553800E77A17EE902A92B2B2F5207F28BF3A4652
:105548002A801D69DA685B696E4302FB0060C01837
:1055580090FBF1F107EE101AF8EEC77AFCEEE77A45
:1055680017EE903A9BB2B3F5F07F28BFEF23238064
:10557800FEBD00BFC40D002040420F00FFF7D8BE9B
:10558800014B187E704700BFC40D0020FFF7C8BE4E
:10559800042808B505D90748074A084B7D21FEF7B6
:1055A800E7F9054B03EB8000038B0B80438B1380DB
:1055B80008BD00BF1AA30508D25F040838A3050870
:1055C80008B5082001F094F942F69643C31A5842E8
:1055D80040EB030008BD10B50A2001F0B1F90C4CEE
:1055E80020600E2001F0ACF96060122001F0A8F9EB
:1055F800A060162001F0A4F9E0601A2001F0A0F9DB
:1056080020611E2001F09CF901236061237610BD02
:10561800C40D002010B5FFF7DBFD01F033FA044696
:1056280001F03CFA074903462246202006F0F8FE1E
:10563800FFF7C6FF28B101F03FFA10B9BDE81040E6
:10564800C9E710BD74A3050810B5104C0A202168DD
:1056580001F05DF961680E2001F059F9A168122086
:1056680001F055F9E168162001F051F921691A2075
:1056780001F04DF961691E2001F049F9082042F650
:105688009641BDE8104001F025B900BFC40D0020C7
:105698002DE9F04F0346A7B0B0F800C01C898688F2
:1056A800DF885D89CDF810C0B249B0F802C0B3F800
:1056B8000C90B3F80E80CDF824C00FFA84FB30B2FA
:1056C80001220FFA87FE0BEB000C0A7629B20FFABB
:1056D80089FACDF888C001EB0E0C0FFA88F2CDF8E4
:1056E80090C00AEB0B0CCDF830C002EB010CCDF8E2
:1056F80058C0B3F810C05B8ACDF800C00FFA8CFC14
:1057080006910CEB00010A9102930CEB0A011BB203
:10571800239103EB0E010E9199182591049900FA33
:1057280081F0584450446044DDF824C006990EFACC
:105738008CFEDDF810C01FFA80FB1CFB0CF08E44B9
:1057480016FB0600964414FB0400009A19FB090096
:105758009E4412FB02001FFA8EFA09F08BFDDDF859
:1057680024C0029ACDE912011CFB0CF017FB0700BC
:1057780015FB050018FB080012FB020009F07AFD72
:10578800DDF824C0029ACDE9140104991CFB01F349
:1057980017FB063615FB0466009B18FB096612FB0F
:1057A800036009F067FDDDE91423CDE90001DDE9B7
:1057B800120109F0D5FD04460D46DDE90001024657
:1057C8000B4609F0CDFD02460B462046294609F056
:1057D80013FCCDE91801584609F05CFDCDE910012C
:1057E800DDE91023DDE9000109F0BAFDCDE9060184
:1057F800504609F04FFD804689464246DDE91201D0
:105808004B4609F0ADFDDDE91023CDE91C01DDE9CA
:10581800140109F0A5FD002206460F46564BDDE9A6
:10582800180109F09DFD424604460D464B46DDE948
:10583800060109F095FD02460B4609F0DFFB02461A
:105848000B462046294609F0D9FB424604460D4638
:105858004B46DDE91C0109F083FD02460B46204654
:10586800294609F0C9FBDDE9102304460D463046F8
:10587800394609F075FD02460B462046294609F0CF
:10588800BBFBDDF828C0CDE902014FEA8C10DDF83A
:1058980030C000EB0C20DDF810C0A0241CFB040075
:1058A80009F0E8FCDDF838C0CDE90A014FEA8C10B0
:1058B800DDF858C000EB0C20DDF824C01CFB040008
:1058C80009F0D8FCCDE90C01504609F0D3FCDDE91C
:1058D8001023CDE91601DDE90C0109F041FD42462E
:1058E800CDE91E014B46DDE90A0109F039FD4246C2
:1058F800CDE920014B46DDE9000109F031FD3246D2
:105908003B4609F079FBCDE90E01584609F0B2FC97
:10591800DDE91C23CDE91A01DDE9060109F06CFB7C
:10592800DDF88CC0C024CDE9060104FB0CF0DDF8DD
:1059380088C0302505FB0C00DDF810C078261CFB5C
:10594800060009F097FCDDF894C0824604FB0CF0D1
:10595800DDF890C005FB0C00DDF824C01CFB060038
:105968008B4609F087FCDDE9102306460F4609F04F
:10597800F7FC03E0C40D0020000014404246CDE9C6
:1059880004014B465046594609F0EAFCDDE9142368
:1059980080468946DDE90A0109F0E2FCDDE90023D9
:1059A80004460D46DDE90C0109F0DAFC02460B4617
:1059B8002046294609F020FB0022A14B09F0D0FC23
:1059C800DDE9202304460D46DDE91E0109F014FB3C
:1059D80002460B46DDE9160109F0C2FC02460B46F9
:1059E8002046294609F00AFB002204460D46954B3D
:1059F800DDE90E0109F0B4FC02460B4620462946B3
:105A080009F0FCFADDE9022309F0D4FD88A3D3E903
:105A1800002309F0A5FC09F03DFF8B490860DDE98A
:105A28001223DDE90C0109F09BFCDDE900230446A3
:105A38000D46DDE90A0109F093FC02460B462046B3
:105A4800294609F0D9FA00227D4B09F089FCDDE9E5
:105A58001E2304460D46DDE9200109F0CDFA024671
:105A68000B46DDE91A0109F07BFC02460B4620468D
:105A7800294609F0C3FA002204460D46714BDDE9B8
:105A8800060109F06DFC02460B462046294609F03E
:105A9800B5FADDE9022309F08DFD65A3D3E90023FA
:105AA80009F05EFC09F0F6FE674A5060DDE90E2356
:105AB800DDE90A0109F054FCDDE9062304460D4638
:105AC800DDE90C0109F04CFC02460B46204629464C
:105AD80009F094FA002204460D465A4BDDE91801F4
:105AE80009F03EFC02460B462046294609F086FA94
:105AF800DDE9022309F05EFD4DA3D3E9002309F097
:105B08002FFC09F0C7FE504B59469860DDE9142375
:105B1800504609F025FCDDE9002304460D463046D1
:105B2800394609F01DFC02460B462046294609F075
:105B380063FA0022424B09F013FC424604460D4624
:105B48004B46DDE9040109F057FA02460B46DDE948
:105B5800160109F005FC02460B462046294609F0C5
:105B68004DFA35A3D3E9002304460D46DDE90E01BD
:105B780009F0F6FB02460B462046294609F03EFA94
:105B8800DDE9022309F016FD29A3D3E9002309F072
:105B9800E7FB09F07FFEDFF8B0C0DDE91223CCF89F
:105BA8000C003946304609F0DBFBDDE900230446EA
:105BB8000D465046594609F0D3FB02460B4620468F
:105BC800294609F019FA00221D4B09F0C9FBDDE945
:105BD800042304460D464046494609F00DFA02469C
:105BE8000B46DDE91A0109F0BBFB02460B462046CD
:105BF800294609F003FA10A3D3E9002304460D4609
:105C0800DDE9060109F0ACFB02460B4620462946B1
:105C180009F0F4F9DDE9022309F0CCFC04A3D3E987
:105C2800002309F09DFB09F035FE074908610DE0E6
:105C38000000000080842E410000000000C0824067
:105C48000000144000008940C40D0020DDE90E2347
:105C58005046594609F084FBDDE9062304460D4603
:105C68003046394609F07CFB02460B462046294659
:105C780009F0C4F911A3D3E9002304460D46DDE970
:105C8800180109F06DFB02460B462046294609F02B
:105C9800B5F9DDE9022309F08DFC0AA3D3E9002355
:105CA80009F05EFB09F0F6FD034A506127B0BDE834
:105CB800F04FC9E4AFF30080C40D002000000000DD
:105CC80000C082400000000080842E41AFF30080B5
:105CD800064B074A596811601969064A1160D96963
:105CE800054A11609A6A054B1A60704794010020B2
:105CF800A83E0020C44400209C440020583E0020B8
:105D0800014B1878704700BFE00D0020032808B544
:105D180005D90548054A064B7321FDF729FE0C23D2
:105D28005843044B185808BDAFA30508FE5F040884
:105D3800C9A3050894010020032808B505D9064819
:105D4800064A074B7821FDF713FE064B0C2202FB8F
:105D58000030406808BD00BFAFA305080E60040806
:105D6800C9A3050894010020034B044A1B780C21A1
:105D780001FB032398687047E00D00209401002080
:105D8800034B044A1B780C2000FB032399607047DF
:105D9800E00D002094010020144B1B78012B10B556
:105DA800134B144C0ED11968C82000F0B0FD2168BF
:105DB800CC2000F0ACFD104BD020196800F0A7FDF6
:105DC800D4200DE01968D82000F0A1FD2168DC205E
:105DD80000F09DFD084BE020196800F098FDE420D4
:105DE800064B1968BDE8104000F091BD280F00204F
:105DF800A83E0020C44400209C440020583E0020B7
:105E0800144B1B78012B10B5134C0FD1C82000F090
:105E180097FD2060CC2000F093FD104B1860D02037
:105E280000F08EFD0E4B1860D4200EE0D82000F054
:105E380087FD2060DC2000F083FD084B1860E0201F
:105E480000F07EFD064B1860E42000F079FD054B5C
:105E5800186010BD280F0020A83E0020C444002070
:105E68009C440020583E002008B502F04DFB10B1BC
:105E7800BDE80840C4E7BDE8084029E70148FBF74A
:105E8800A4BB00BFD41500200148FBF79EBB00BF90
:105E9800D41500200148FBF798BB00BFD41500209B
:105EA8000148FBF792BB00BFD4150020032808B5B2
:105EB80005D91648164A174B4F21FDF759FD164BC1
:105EC8001870164B1870164B012202281A70154BC1
:105ED8000FD0032813D0904205D0134A12681A60D5
:105EE800BDE80840CAE7114A12681A60BDE80840D0
:105EF800CAE70F4A12681A60BDE80840CAE70D4AA7
:105F080012681A60BDE80840CAE700BFAFA30508D9
:105F18001F600408F3A30508E00D00209E3E002042
:105F28000C0E0020EC020020E4020020E002002019
:105F3800DC020020D8020020064B07495960C02126
:105F4800002219721E211A70D9601A745A611A76C1
:105F5800DA6170472018002040787D0110B50321D0
:105F6800FF22C02001F094F81F4C102120608022ED
:105F7800C02001F08DF8112120608022C02001F09E
:105F880087F8122120608022C02001F081F81321B7
:105F980020608022C02001F07BF81421206080223C
:105FA800C02001F075F8152120608022C02001F082
:105FB8006FF8802220601621C02001F069F8206067
:105FC800C0201721802201F063F82060074CC02010
:105FD800227AB72101F05CF80023237463612376E9
:105FE800E3610123237010BD7C3E002020180020AF
:105FF80038B5C0200321FF2201F04AF80B4D0024D8
:106008002B19615D5A78C020023401F041F8C82C80
:10601800F6D1B121AC22C02001F03AF8C02003210A
:10602800002201F035F8002038BD00BF33600408B5
:106038002DE9F34706460F4692461D461AB90C1F2E
:10604800E401914635E005EE902A06EE903AB8EE66
:10605800657AF8EE667AFC01C7EE277AA4F5007433
:106068009FED5C7A67EE877A17EE900A09F024F9BB
:1060780041EC100B0BF05CF959EC108B494640468B
:1060880009F030FC24184FEACA1009F0F3F8CDE9FA
:106098000001284609F0EEF84B46424609F060F93F
:1060A80002460B46DDE9000108F0A6FF09F01AFCDC
:1060B8008146002E14BF4FF022084FF01A08C5F38E
:1060C80007224146C02000F0E3FF08F10101EAB2CF
:1060D800C02000F0DDFFC4F3014208F10201C02036
:1060E80000F0D6FFC4F3072208F10301C02000F036
:1060F800CFFFE2B208F10401C02000F0C9FFC9F3E4
:10610800034305F4702243EA123208F10501C02066
:1061180000F0BEFF08F10601C9F30722C02000F015
:10612800B7FF08F107015FFA89F2C02000F0B0FF5D
:10613800C020B121A02200F0ABFF07EE107A264C58
:10614800F8EEC77A0EBBD4ED015A06EE90AAB8EE67
:10615800657A05EE905AB8EE666AF8EE656A01232C
:10616800C6EE266A237477EEA67A67EE277A17EECC
:10617800900A09F0A1F841EC100B0BF0D9F851EC9A
:10618800100B09F0AFFB606120E005EE90AAD4ED9A
:10619800016AB8EE656A05EE905AB8EE667AF8EECE
:1061A800656A0123C6EE266A237677EEA67A67EE3D
:1061B800277A17EE900A09F07FF841EC100B0BF0E4
:1061C800B7F851EC100B09F08DFBE0610020BDE839
:1061D800FC8700BF00000043201800200022012394
:1061E80026E7012838B50D4604D002280CBF3C2408
:1061F8002C2400E034242146C02000F0C3FF05F021
:10620800070200F00F0040EA02122146C020BDE854
:10621800384000F03DBF2DE9F3470A9C1D4607466C
:106228008A461646524B01E06D0864089C42FBD82A
:106238002DB906F10076043EF601A94634E006EED3
:10624800905AB8EE667A06EE904AF8EE667AF6014B
:10625800C7EE277AA6F500769FED467A67EE877A2D
:1062680017EE900A09F028F841EC100B0BF060F8D3
:1062780059EC108B4946404609F034FB3618E801C2
:1062880008F0F8FFCDE90001204608F0F3FF4B467F
:10629800424609F065F802460B46DDE9000108F0C0
:1062A800ABFE09F01FFB8146022F9BBF324BDB1967
:1062B8004FF0000893F8C880C4F307224146C02075
:1062C80000F0E6FE08F10101E2B2C9B2C02000F018
:1062D800DFFE08F10201C9B2C6F30142C02000F096
:1062E800D7FE08F10301C9B2C6F30722C02000F0A7
:1062F800CFFE08F10401C9B2F2B2C02000F0C8FE16
:1063080004F47024C9F3034308F1050143EA143285
:10631800C9B2C02000F0BCFE08F10601C9B2C9F339
:106328000722C02008F1070800F0B2FE5FFA89F2E0
:106338005FFA88F1C02000F0ABFEBAF1010F0CBF84
:106348002F220F220DB942F04002012F06D002D3AE
:10635800022F0AD105E0C020102104E0C02011213D
:1063680001E0C020122100F093FE0020BDE8FC8768
:10637800FFFF0F00000000433360040807B5012346
:1063880000930023FFF747FF0EBD00280CBFFF2234
:10639800002208B5C020032100F07AFE002008BDC5
:1063A80008B5C020B121AC2200F072FE002008BD63
:1063B80008B50420012107F0CDFB4FF480700121BE
:1063C800BDE8084007F0F6BB07B502230093032396
:1063D8008DF804300348002369468DF8073007F02C
:1063E80011F80EBD0008024030B5124D8BB00024E4
:1063F80006A8069407940894099406F0D1F9009425
:106408008DF804408DF805400294039404942846BE
:10641800012469468DF8144006F093F928460B21AB
:106428002246062306F008FA2846214606F0D2F945
:106438000BB030BD0020014010B5002104460122F8
:10644800302000F025FEC0B9012001F041F8002CF1
:10645800B8BF4034E4B210212246302000F018FEC4
:10646800012001F035F830201121224600F010FEFD
:106478000120BDE8104001F02BB810BD10B5002177
:1064880004460122302000F003FEC0B9012001F0CB
:106498001FF8002CB8BF4034E4B212212246302045
:1064A80000F0F6FD012001F013F8302013212246F8
:1064B80000F0EEFD0120BDE8104001F009B810BD64
:1064C80038B5012205460C463020002100F0E0FDD9
:1064D800F0B9012000F0FCFF25EAE5725F2AA8BFA9
:1064E8005F223B21D2B2302000F0D2FD012000F023
:1064F800EFFF24EAE4725F2AA8BF5F22D2B23020FD
:106508003C2100F0C5FD0120BDE8384000F0E0BFA7
:1065180038BD302810B504460ADC10F17F0F02DBC5
:10652800002802DB05E06FF07E0404F5807400E0CB
:106538003024002130200A4600F0AAFDA8B9012025
:10654800E4B200F0C5FF41212246302000F0A0FD52
:10655800012000F0BDFF30204221224600F098FDC6
:106568000120BDE8104000F0B3BF10BD282810B5C9
:10657800044609DC10F1180F02DB002802DB04E0F6
:106588006FF017047F3400E02824002130200A46E9
:1065980000F07EFDA8B90120E4B200F099FF532174
:1065A8002246302000F074FD012000F091FF3020D9
:1065B8005421224600F06CFD0120BDE8104000F097
:1065C80087BF10BD08B530200021012200F060FD12
:1065D80060B9012000F07CFF30203321402200F018
:1065E80057FD0120BDE8084000F072BF08BD10B596
:1065F80030200021012200F04BFD044660B9012043
:1066080000F066FF30203321224600F041FD0120D2
:10661800BDE8104000F05CBF10BD10B5302000216F
:10662800012200F035FD0446A0B9012000F050FF1A
:1066380034212246302000F02BFD012000F048FFD5
:1066480030203721224600F023FD0120BDE810400C
:1066580000F03EBF10BD4020EEE640200EE708B532
:1066680000210122302000F013FD012000F030FF4E
:1066780030203421024600F00BFD012000F028FFF5
:1066880030203721024600F003FD0120BDE8084014
:1066980000F01EBF08B500210122302000F0F8FCF0
:1066A800012000F015FF302034210C2200F0F0FC0E
:1066B8000120BDE8084000F00BBF0000000000000A
:1066C800184B1949D3ED006A93ED017A00231A4655
:1066D8009FED166A03E0F0EE476AB0EE677A505E07
:1066E80005EE900AF8EEE57A0133C7EE867A9BB29A
:1066F80018B204327F2877EEE67AECDD27EE077AC7
:1067080007EEA77A0A49074A0B80BDEEC77A00232D
:1067180013605360C2ED027A17EE102A054B9200FF
:106728001A607047E40D0020DC2900200000FA45BB
:106738000C3E0020A81A00202DE9F84F2E4B2F4AB6
:1067480019682F4B19B92F4911602F4A02E02F49B8
:1067580011602F4A1A602F4BDFF8BCA0DFF8BC90FD
:10676800DFF8BCB000221A80244A9846176830E047
:1067780007EB84036500B3F9023007EE103AF8EE30
:10678800C77A013617EE900A08F096FD18A3D3E9E8
:10679800002308F0E5FD09F07DF829F815002AF82E
:1067A800140037F9243007EE103AF8EEC77A0135AD
:1067B80017EE900A08F080FD0DA3D3E9002308F036
:1067C800CFFD09F067F82BF8140029F81500A8F890
:1067D8000060B8F8006034B2FF2CC9DD00F05EF844
:1067E80000F06AF801F09CF9BDE8F84F68E700BFCF
:1067F8009A9999999999E93F9C1A0020901A002032
:10680800C8180020DE310020DE2D0020DE390020EF
:10681800DE3500200C3E0020DC250020DC2900208D
:10682800DC27002010B50B4C204606F038FA0A4B3E
:1068380018600A4806F033FA094B1860FFF77CFF26
:10684800084B0949012220469A81BDE8104006F00C
:10685800A7BA00BF106002409C1A0020886002405E
:10686800B81A0020E40D002020800010014B1868A1
:10687800704700BFA81A002008B5054B05481988BD
:106888000022012309F044FD034B187008BD00BF26
:10689800C4010020C4250020E0200020034804494A
:1068A800044A4FF4807309F0ABBD00BFC801002053
:1068B800DC250020C223002003480449044A4FF481
:1068C800807309F09DBD00BFD4010020DC270020A3
:1068D800FC1B002038B505460C460135C1F30721DD
:1068E80000F004FEA8B2E1B200F000FE00B238BD2C
:1068F80038B5044600F00EFD01340546A0B200F09C
:1069080009FDEDB2C0B240EA052000B238BD37B586
:106918000B0E8DF804300B0C8DF805300B0A8DF832
:1069280006308DF80710002400E0284601AB451C0E
:10693800E15C013400F0DAFD042CADB2F5D13EBDC6
:1069480037B5002400E02846451C00F0E3FC01AB05
:10695800ADB2E0540134042CF5D19DF805009DF842
:106968000430000440EA03609DF8073018439DF89E
:10697800063040EA03203EBD38B50446642000F0E6
:10698800A7FD25786068AD00EDB2257006F09FFD83
:10699800237A40FA03F000F003000543104B2570FA
:1069A80005F00F055A5D6378D218D2B2D3B201321E
:1069B800D2B2022A637001D80022A2705BB2012B06
:1069C80003DD0123A3700023637094F901300133C0
:1069D80003DAFF23A3700023637094F9020038BD23
:1069E800FE600408F7B504200121234F07F0B2F830
:1069F80002AD01214FF48040012407F0DBF80026A6
:106A08004FF4B0733846694645F8083D8DF8046080
:106A18008DF8074006F0F6FC1020214607F09AF89A
:106A280078236946154800938DF804608DF807406F
:106A380006F0E8FC0420214607F08CF821464FF4C4
:106A4800804007F0B7F81C233846694600938DF854
:106A580004608DF8074006F0D5FC0220214607F0B7
:106A680079F8B02306488DF8046069468DF8074028
:106A7800009306F0C7FCFEBD00080240001002406B
:106A880000040240802108B5034806F01AFDD0F141
:106A9800010038BF002008BD0004024008B54FF4CB
:106AA8008071044806F00DFDD0F1010038BF0020C8
:106AB80008BD00BF0008024008B5FFF7E3FF08B1B2
:106AC800FFF7ECFFC0B208BD10B5642000F000FD70
:106AD8001D48FFF751FF044610B91C4B187009E018
:106AE800FFF7DCFF30B9002C184B01DD012200E074
:106AF800FF221A701648FFF73FFF164B1B78042B2E
:106B080016D100281FD0144B1A7806DD0132D2B2F4
:106B18000F2A1A7008D9102205E0013AD2B2102AB9
:106B28001A7001D900221A70BDE81040FAF740BE69
:106B380000280A4B01D1187010BD02DD01221A701D
:106B480010BDFF221A7010BD14020020A0440020BE
:106B580020020020403E0020A63E0020DC2D002020
:106B680007B50220012106F0F5FF012300938DF8F7
:106B7800043002238DF805300448002369468DF857
:106B880006308DF8073006F03DFC0EBD00040240CB
:106B980010B5084C01210022204606F0A8FC40F25E
:106BA800FF4000F095FC012120460A46BDE8104050
:106BB80006F09DBC0004024008B5FFF7E9FF00217C
:106BC8000A46302000F064FA012000F081FC01211F
:106BD8000A46302000F05CFA012000F079FC002120
:106BE8000122302000F054FA012000F071FC01214C
:106BF8000822302000F04CFA012000F069FC022144
:106C08000122302000F044FA012000F061FC00214C
:106C18000A46302000F03CFA012000F059FC1B2104
:106C2800CD22302000F034FA012000F051FC04217C
:106C38000322302000F02CFA012000F049FC062144
:106C48000822302000F024FA012000F041FC07213E
:106C58000A46302000F01CFA012000F039FC082117
:106C68008022302000F014FA012000F031FC1E21AF
:106C7800B022302000F00CFA012000F029FC052198
:106C88009122302000F004FA012000F021FC0D21AF
:106C98000322302000F0FCF9012000F019FC0E213D
:106CA8000022302000F0F4F9012000F011FC14213A
:106CB8008022302000F0ECF9012000F009FC0B21C3
:106CC8008822302000F0E4F9012000F001FC302097
:106CD8000C21822200F0DCF9012000F0F9FB1221DE
:106CE8008822302000F0D4F9012000F0F1FB1321B4
:106CF8008C22302000F0CCF9012000F0E9FB0021C3
:106D08000122302000F0C4F9012000F0E1FB0C2141
:106D18000822302000F0BCF9012000F0D9FB0D2139
:106D28000822302000F0B4F9012000F0D1FB0E2138
:106D38000822302000F0ACF9012000F0C9FB0F2137
:106D48000822302000F0A4F9012000F0C1FB002146
:106D58000A46302000F09CF9012000F0B9FB4021E0
:106D68000222302000F094F9012000F0B1FB00224B
:106D78004121302000F08CF9012000F0A9FB3020DF
:106D88003F21D42200F084F9012000F0A1FB00216A
:106D98000122302000F07CF9012000F099FB10213D
:106DA8000F22302000F074F9012000F091FB11212E
:106DB8000F22302000F06CF9012000F089FB12212D
:106DC8000022302000F064F9012000F081FB13213B
:106DD8000022302000F05CF9012000F079FB092145
:106DE8003C22302000F054F9012000F071FB002112
:106DF8000122302000F04CF9012000F069FB30201E
:106E08003421024600F044F9012000F061FB3020F3
:106E18003721024600F03CF9012000F059FB3621E9
:106E28000322302000F034F9012000F051FB392111
:106E38000322302000F02CF9012000F049FB3B210F
:106E48003C22302000F024F9012000F041FB3C21D5
:106E58000A46302000F01CF9012000F039FB00211F
:106E68000A46302000F014F9012000F031FB5121CE
:106E7800C022302000F00CF9012000F029FB30205E
:106E88005221002200F004F90120BDE8084000F07A
:106E98001FBB00BF2DE9F04F454E464D93B0012171
:106EA8004FF4001006F056FE304605F0F9FD4FF09D
:106EB800C0630293404B0393404B002404934FF468
:106EC80000794FF400334FF480684FF400674FF4B3
:106ED800005A4FF4807B304602A90C93019309971E
:106EE800CDF8189005940794CDF82080CDF828A007
:106EF800CDF82CB00D9405F05FFE2246304630499F
:106F080005F0B5FE3046012105F0BBFE01210A4619
:106F18004FF0402007F08CF8284605F0C1FD294ABB
:106F2800019B0392284A0C9304922846402202A906
:106F3800059209970294CDF818900794CDF820800F
:106F4800CDF828A0CDF82CB00D9405F035FE2246DA
:106F580028461E4905F08BFE2846012105F091FEC2
:106F680042F2107701220221194807F061F83846E9
:106F780000F0AEFA3046012105F059FE01212846FD
:106F880005F055FE384600F0A3FA0B238DF844307F
:106F980011A801238DF845408DF846408DF84730FB
:106FA80000F01AFD384600F093FA13B0BDE8F08FF0
:106FB80010600240886002400C400040DE3900202A
:106FC800DE3100200C3C0040DE350020DE2D0020A4
:106FD800003C004002481021012205F09FBE00BF7E
:106FE8001060024013B50220012106F0B3FD4FF4F2
:106FF80010730E4C009302238DF804308DF8053081
:1070080001238DF806302046002369468DF80730A5
:1070180006F0F8F920460621042206F073FA204605
:107028000921042206F06EFA1CBD00BF00040240CC
:1070380030B5154D85B001214FF4001006F0AEFDB6
:10704800284606F075FA0023ADF804304BF6FF73B6
:10705800ADF806303323ADF808304FF48063ADF84F
:107068000A304FF48043ADF80C3004AC074B284687
:10707800012144F8103D06F0FDFA2846694606F05D
:1070880085FA05B030BD00BF00540040801A0600E4
:1070980073B54FF4961306460D461446019304E063
:1070A800019B5A1E0192002B57D031484FF40031F2
:1070B80006F0F8FB0028F3D12D48012106F0E6FA86
:1070C8004FF48053019304E0019B5A1E0192002B58
:1070D80045D02748274906F0D0FB0028F4D024489B
:1070E8003146002206F0EAFA4FF48053019304E097
:1070F800019B5A1E0192002B33D01D481E4906F0F1
:10710800BCFB0028F4D01A48294606F05AFB4FF475
:107118008053019303E0019B5A1E01921BB314484C
:10712800164906F0AAFB0028F5D01148214606F0BA
:1071380048FB4FF49613019303E0019B5A1E0192FA
:107148009BB10B480E4906F0ADFB0028F5D0084866
:10715800012106F0A7FA002008E0012006E002203D
:1071680004E0032002E0042000E005207CBD00BF0D
:10717800005400400100030082000700800007005F
:107188000400001037B54FF4961304460D460193DA
:1071980005E0019B5A1E0192002B00F09B80564887
:1071A8004FF4003106F07EFB0028F2D1524801214D
:1071B80006F06CFA4FF48053019305E0019B5A1EC8
:1071C8000192002B00F088804B484C4906F055FB93
:1071D8000028F3D048482146002206F06FFA4FF401
:1071E8008053019304E0019B5A1E0192002B75D035
:1071F8004148434906F041FB0028F4D03E4829465F
:1072080006F0DFFA4FF48053019304E0019B5A1E05
:107218000192002B64D038483A4906F043FB002815
:10722800F4D03548012106F031FA4FF48053019328
:1072380004E0019B5A1E0192002B53D02E482F497F
:1072480006F01BFB0028F4D02B482146012206F04B
:1072580035FA4FF48053019304E0019B5A1E0192C2
:10726800002B41D0244C2849204606F01BFB00285F
:10727800F3D02046002106F029FA20460121238B6D
:1072880006F010FA4FF48053019304E0019B5A1E54
:107298000192002B2AD018481C4906F003FB00284D
:1072A800F4D0154806F08FFA4FF480530193124A30
:1072B80003E0019B591E0191D3B113889B05F8D4B3
:1072C800012104460C4806F001FA0B48104906F063
:1072D80003FB0EE001240CE002240AE0032408E08A
:1072E800042406E0052404E0062402E0072400E064
:1072F800082420463EBD00BF0054004001000300A2
:107308008200070004000010020000104000001076
:107318000004001013B54FF496130446019305E0DA
:10732800019B5A1E0192002B00F0B08061484FF477
:10733800003106F0B7FA0028F2D15E48012106F0C4
:10734800A5F94FF48053019305E0019B5A1E019261
:10735800002B00F09D805748574906F08EFA002808
:10736800F3D05448A021002206F0A8F94FF4805326
:10737800019305E0019B5A1E0192002B00F08A80C0
:107388004C484E4906F079FA0028F3D0C4F3052199
:10739800484806F016FA4FF48053019304E0019B25
:1073A8005A1E0192002B77D04248454906F07AFAD6
:1073B8000028F4D0E1B23F4806F003FA4FF48053B6
:1073C800019304E0019B5A1E0192002B66D03948B4
:1073D8003B4906F067FA0028F4D03648012106F048
:1073E80055F94FF48053019304E0019B5A1E019212
:1073F800002B55D02F48304906F03FFA0028F4D02A
:107408002C48A121012206F059F94FF48053019329
:1074180004E0019B5A1E0192002B43D0254C2949B8
:10742800204606F03FFA0028F3D02046002106F057
:107438004DF920460121238B06F034F94FF480538F
:10744800019304E0019B5A1E0192002B2CD019488D
:107458001D4906F027FA0028F4D0164806F0B3F9BB
:107468004FF480530193134A03E0019B591E019185
:10747800E3B113889905F8D4012104460D4806F0B4
:1074880025F90C48114906F027FA10E001240EE00E
:1074980002240CE003240AE0042408E0052406E0A2
:1074A800062404E0072402E0082400E0092420461A
:1074B8001CBD00BF0054004001000300820007000B
:1074C800040000100200001040000010000400102A
:1074D80082B0002304E0019B01330193009B013338
:1074E8000093009B8342F6D302B0704737B54FF440
:1074F800805304460D46019304E0019B5A1E0192F5
:10750800002B6ED03D484FF4003106F0CBF900282F
:10751800F3D13A48012106F0B9F84FF480530193AA
:1075280004E0019B5A1E0192002B5CD03348344979
:1075380006F0A3F90028F4D03048A021002206F074
:10754800BDF84FF48053019304E0019B5A1E019249
:10755800002B4AD029482B4906F08FF90028F4D08F
:10756800C4F30521254806F02CF94FF48053019304
:1075780004E0019B5A1E0192002B38D01F48224973
:1075880006F07BF90028F4D0E1B21C4806F019F99E
:107598004FF48053019303E0019B5A1E019243B3B9
:1075A8001648194906F069F90028F5D01348294604
:1075B80006F007F94FF49613019303E0019B5A1E56
:1075C8000192C3B10D48114906F06CF90028F5D0B5
:1075D8000A48012106F066F80D48FFF779FF0020F8
:1075E8000AE0012008E0022006E0032004E004206D
:1075F80002E0052000E006203EBD00BF0054004028
:10760800010003008200070080000700040000104A
:10761800A0860100F7B54FF4805304460D46164680
:10762800019304E0019B5A1E0192002B75D041483A
:107638004FF4003106F036F90028F3D13D48012116
:1076480006F024F84FF48053019304E0019B5A1E7E
:107658000192002B63D03748374906F00EF900280D
:10766800F4D03448A021002206F028F84FF48053C3
:10767800019304E0019B5A1E0192002B51D02D4822
:107688002E4906F0FAF80028F4D0C4F30521294859
:1076980006F097F84FF48053019304E0019B5A1EBB
:1076A8000192002B3FD02348254906F0E6F8002830
:1076B800F4D0E1B21F4806F084F84FF480530193E8
:1076C80004E0019B5A1E0192002B2ED019481C4938
:1076D80006F0D3F80028F4D000244FF4961710E0F1
:1076E800295D144806F06DF8019703E0019B5A1EC6
:1076F8000192E3B10F48134906F0D4F80028F5D0F9
:107708000134E3B2B342EBD30A48012105F0CAFFC2
:107718000D48FFF7DDFE00200AE0012008E0022006
:1077280006E0032004E0042002E0052000E0062033
:10773800FEBD00BF005400400100030082000700A6
:107748008000070004000010A086010013B5052082
:10775800012106F0FFF9184C4FF4E053009302237F
:107768008DF804308DF805302046002369468DF8E1
:1077780006308DF8073005F045FE20460A2106221E
:1077880005F0C0FE20460C21062205F0BBFE0622AD
:1077980020460B21A4F5006405F0B4FE4FF4004325
:1077A80020466946009305F02DFE20460F2106224B
:1077B80005F0A8FE1CBD00BF000802401FB5044626
:1077C800FFF7CEF9FFF734FCFFF7F6F9FFF7BEFF36
:1077D80001214FF4004006F0E1F902940F4C102308
:1077E800ADF80230204600236946ADF80430ADF804
:1077F8000C30ADF80030ADF8063006F0FEFA6946F8
:107808004FF0402006F0CDFB2046012106F07DFB1D
:107818004FF04020012106F078FB1FBD003C0040DE
:10782800014B1860704700BF000E0020704710B56C
:107838000A4A1379262B04D80949C854013313710D
:1078480010BD074A0123591ED45C0133272B545419
:10785800F9D1034B83F8260010BD00BF000E0020AD
:10786800E03D0020704710B504462078FFF7DFFFA1
:1078780014F8013F002BF8D110BD38B504460D4669
:10788800013D14F8010BEDB2FFF7D1FF002DF7D140
:1078980038BD00BF014B1878704700BF080E0020A4
:1078A800014B5878704700BF080E0020024B18782B
:1078B80080F00100704700BF080E0020024B002234
:1078C8001A705A70704700BF080E0020014B012241
:1078D8001A707047080E0020014B01225A70704739
:1078E800080E002082B0002304E0019B01330193BD
:1078F800009B01330093009B8342F6D302B070478C
:1079080007B50420012106F025F901214FF4804034
:1079180006F050F94FF40073009300238DF80430FB
:107928000348012369468DF8073005F06BFD0EBD4D
:10793800000802400D4B07B51A680D484FF47A73DA
:10794800B2FBF3F20B4B013A5A600B4AF02182F872
:10795800231000229A6007221A60084B084A0093F5
:107968000121084B04F07CFA0EBD00BFF002002094
:10797800AC3E002010E000E000ED00E00C04002028
:10798800F003002058030020054B1A6812B11A684A
:10799800013A1A60034B1A6801321A60704700BF37
:1079A800683E0020803E002082B0044B0190019A7E
:1079B8001A601A68002AFCD102B07047683E00209D
:1079C800704700BF40F0BE60024B40F42020D860F2
:1079D800704700BF00ED00E0C37810B503B3164B45
:1079E8004278DB688478DB43C3F30223C3F10401E4
:1079F800C9B202FA01F10F2242FA03F2C9B22240D7
:107A08000A430E4B01781201CB18D2B283F8002337
:107A180003780122590903F01F0302FA03F307E070
:107A280003780122590903F01F0302FA03F32031F6
:107A3800024A42F8213010BD00ED00E000E100E00C
:107A480021F0604121F07F01014B084398607047A5
:107A580000ED00E0044B1A6909B1104301E022EA85
:107A680000001861704700BF00ED00E0044B1A6881
:107A780004280CBF42F0040222F004021A60704786
:107A880010E000E000000000034A044B1A60044ABA
:107A9800044B1A60704700BF0000FA45B01A002076
:107AA800DB0FC93FAC1A0020034B00221A60034ABF
:107AB800034B1A60E8E700BFE04400200000FA45E5
:107AC800A819002007EE100A024BF8EEC77AC3ED9A
:107AD800007A7047A819002038B510EE100A07F090
:107AE800EBFB0DA3D3E9002307F03AFC084B04464F
:107AF80018680D4607F0E0FB0B460246294620466B
:107B080007F058FD07F00EFF024B186038BD00BFA4
:107B1800B01A0020AC1A0020182D4454FB2119403B
:107B28002DE9F04F2DED048B9D4C89B04FF00008E6
:107B3800A1469C4B38F803509B4B258038F80360CE
:107B48009A4B6680186807F0B7FB8DA3D3E900232A
:107B580007F006FC07F09EFE6368954AC0180111FD
:107B680001F580610905090D6060C0F30B1008AFCD
:107B780032F8203032F82120616A238115FB02F0A7
:107B8800628115FB03F516FB02F216FB03F607EB01
:107B98004103E0602561C0F3CF30C5F3CF356261A2
:107BA800A661C2F3CF32C6F3CF3623F8200C23F8F0
:107BB800105C23F8182C23F8086C7E4BA083013145
:107BC8000B40002BE5832284668403DA013B63F0D3
:107BD80003030133C9F82430002B40F0C5807648F0
:107BE800764A774E774D6946042308F0C9FE7648F1
:107BF800764A04A9042308F0C3FE7548754A02A909
:107C0800042308F0BDFE744A744806A9042308F04A
:107C1800B7FEB4F9283007EE903AB4F92A30B8EE36
:107C2800E79A07EE903AB4F92C30B8EEE78A07EEF7
:107C3800903AB4F92E30F8EEE79A07EE903AF8EE5B
:107C4800E78A68EE087A49EE097A17EE900A07F093
:107C580033FB41EC100B09F025FD51EC100B07F03C
:107C680061FE68EEA87A49EEA97A306017EE900AAC
:107C780007F022FB41EC100B09F014FD51EC100B3E
:107C880007F050FE68EE897A58EE297A28EE288A9D
:107C9800286009EE298A17EE900A07F00DFB824644
:107CA80018EE100A8B4607F007FB4BEC10AB41ECC3
:107CB800110B09F06FFC51EC100B07F033FE484B29
:107CC8001860286807F0F8FA2FA3D3E9002307F013
:107CD800B9FD08B1434B2B6096ED000AD5ED007A4B
:107CE80080EE270A404F87ED000A09F025FC00B90D
:107CF800FEE73B4E3D4D306807F0DEFA24A3D3E99A
:107D0800002307F02DFB824628688B4607F0D4FA3B
:107D180021A3D3E9002307F023FB02460B46504674
:107D2800594607F06BF907F0FDFD286030603868A8
:107D38002F4D07F0C1FA16A3D3E9002307F010FB73
:107D4800824628688B4607F0B7FA13A3D3E90023C5
:107D580007F006FB02460B465046594607F04EF917
:107D680007F0E0FD2860386008F10208B8F5007FE8
:107D78007FF4DFAE09B0BDEC048BBDE8F08F00BF27
:107D880039D6C56D305FC4408DEDB5A0F7C6B03E9D
:107D98009A9999999999B93FCDCCCCCCCCCCEC3F58
:107DA8001C0E0020C2230020FC1B0020AC1A00205F
:107DB800186104080300008008020020440E002017
:107DC800E8440020DC440020FC010020460E00208E
:107DD800F0010020480E00204A0E0020E401002097
:107DE800CC440020BD378635D4440020D044002040
:107DF800E4440020014B93ED000A7047D44400206E
:107E0800014B93ED000A7047CC440020014B93EDE1
:107E1800000A7047E4440020014B93ED000A7047C4
:107E2800D0440020014B93ED000A7047E84400203D
:107E3800014B93ED000A7047DC440020AFF300804B
:107E480010B5FEF78BF80020012324210246FEF727
:107E5800EFF8114B1C780020012C05D10146FEF7E4
:107E6800C0F92046002104E00721FEF7BAF90120F5
:107E78000721FEF7B6F963221221C020FFF708F99F
:107E880002200121FEF7ADF9FEF78AFA0120BDE8CC
:107E98001040FEF77ABA00BF280F00200D4B1B7860
:107EA800012B05D10C4B0D4A196812688A181A6003
:107EB8000B4B1B78012B084B196805D1094A9142D5
:107EC80007DD01321A607047074A914201DD01322D
:107ED8001A607047403E0020A44400203C3E002029
:107EE800280F00207FD1F008FF1FA1070E4B1B7839
:107EF800012B05D10D4B0E4A196812688A1A1A60AF
:107F08000C4B1B78012B094B05D10B4A1968914280
:107F180008DC1A6070471A68B2F57A2FDCBF4FF494
:107F28007A221A60704700BF403E0020A444002017
:107F38003C3E0020280F002040420F00024B1A68E8
:107F4800024B1A60704700BFA03E0020A4440020E6
:107F58002DE9F04F824658488BB0B0FBF1F00C4643
:107F680007F088F941EC100B09F0E2F951EC100B1D
:107F780007F0B8FCC307074648BF471E04FB07F0D5
:107F880007F078F946A3D3E9002307F013FB04466A
:107F98000D4645EC104B09F0CBF959EC108B2046F7
:107FA80042464B46294607F027F8CDE904014946E1
:107FB800404607F097FC3CA3D3E900230990DDE98C
:107FC800040107F049FC00283DD1002401234FF0AB
:107FD8001509224698462046DFF8E4B003E0234618
:107FE80042462C46B04600FB04355D452ED800FBC2
:107FF8000826DDE904012EA3D3E9002307F02CFCB1
:1080080030BBDDE9042300202C4907F0D3FA41EC0A
:10801800100B0390029109F08BF90398029953EC25
:10802800102B8DED060B06F0E7FF09F1FF39CDE9BE
:1080380004015FFA89F9DDE9060107F053FCB9F19B
:10804800000FCCD104E00125002601E02546464674
:10805800099BD9B2BAF1000F0BD132462B465046D4
:10806800FDF7E6FF01230093504651463A46534632
:1080780009E032462B460120FDF7DAFF0120009087
:1080880001463A460023FEF7C6F8FEF789F90120B3
:108098000BB0BDE8F04FFEF778B900BFAFF3008032
:1080A8000000000084D77741956479E17FFDA53D04
:1080B800BBBDD7D9DF7CDB3D00E9A4350000F03F2C
:1080C800FFFF0F0038B52B4B1B78022B2A4B03D12F
:1080D8002A4A12681A6038BD1968294B294A1B6850
:1080E800294CCB189342236018DC0020FFF730FF9F
:1080F80001202168FFF72CFF244B1C780020012C5D
:1081080005D10146FEF76DF82046002104E007215D
:10811800FEF767F801200721FEF763F81C4B1B7870
:10812800022B14D11B4B1C4D1A68134C2B68D31807
:1081380022689A420BDA194B1B78012B07D1184B8E
:10814800186800F085F822682B68D3182360094B5B
:108158001A78012A0DD10F4A11680F4A12688A1835
:1081680005490968914204DB02221A700D4B00226E
:108178001A6038BD3C460020A4440020A03E0020E0
:10818800BC44002080D1F008C0440020280F002003
:10819800403E0020903E00203C3E0020883E0020CB
:1081A800583E0020AC0E002008B5FEF76BFC094BCA
:1081B8005A78187002435A701AB19A7801329A7034
:1081C80030B99B78034A012B02D90023537093706E
:1081D80008BD00BF4C0E002007B50420012105F0A2
:1081E800B9FC4FF46043009301238DF80430022357
:1081F8008DF805300448002369468DF806308DF85F
:10820800073005F0FFF80EBD00080240084B1A6859
:108218004FF47A73B2FBF3F2064B013A5A60064AFE
:10822800F02182F8231000229A6007221A60704712
:10823800F002002010E000E000ED00E0034B5A6877
:1082480012B15A68013A5A60704700BF4C0E0020BC
:10825800024B58605A68002AFCD170474C0E002027
:1082680030B585B004460D4601A85C490A220BF0DA
:10827800A7FC5B4B1B78032B10D8DFE803F0020543
:10828800080B01A8574907E001A8574904E001A8CD
:10829800564901E0564901A80BF07CFD04AA1319C0
:1082A80013F80C3C5D19EDB22F2D01D80A3502E008
:1082B800392D01D90A3DEDB204AB1C194FF6FF70F8
:1082C80004F80C5CFCF7A2FD0020FCF7A1FE0DF100
:1082D80003050F24204623345A21002315F8012FC3
:1082E800A4B2FCF7AFFEB4F5A57FF3D164205A2100
:1082F8002C220023FCF7A6FE0023CD205A212C2295
:10830800FCF7A0FE0020FCF781FD354B1B78032B02
:1083180062D8DFE803F002284B5601A931480BF078
:1083280039FD0A2200212F480BF0D8FE314A324B82
:1083380012781860012A06D1304A904201DC0132D5
:108348001A602F4A06E0B0F5FA5FBCBF4FF4FA5244
:108358001A602C4A1B689342C4BF274B1A602A4BE9
:108368001A682A4B20E001A91F480BF013FD0A22C6
:1083780000211D480BF0B2FE1E4A254B12781860EA
:10838800012A06D11D4A904201DC01321A601C4ABA
:1083980006E0B0F5FA5FBCBF4FF4FA521A60194A0A
:1083A8001B68934218DD1A4B1A6015E001A90F48A3
:1083B8000BF0F0FC0D4800210A220BF08FFE154B44
:1083C80009E001A90A480BF0E5FC094800210A2246
:1083D8000BF084FE104B186005B030BDF2A4050800
:1083E8009E3E00206C3E0020943E0020A9440020C0
:1083F8005C3E0020280F0020A83E00203F420F00CE
:1084080080D1F00840420F00A03E0020A444002084
:10841800C44400209C440020583E002010B50D4B59
:108428000D4C1A680D4821460BF08CFC0C4B0D487E
:108438001A6821460BF086FC0B4B0C481A6821463B
:108448000BF080FC0A4B0B481A682146BDE8104027
:108458000BF078BCA83E0020FCA405086C3E002068
:10846800C4440020943E00209C440020A9440020DD
:10847800583E00205C3E00209FED010A704700BF77
:10848800000000009FED010A704700BF00000000D7
:108498009FED010A704700BF000000007047704759
:1084A800044B18B1012801D1034A00E0034A1268BD
:1084B8001A607047A4440020903E0020A03E00208F
:1084C80010B9034B18687047024B1868704700BF13
:1084D800A83E0020A03E002010B9034B1868704742
:1084E800024B1868704700BFC4440020903E00202B
:1084F80008B54FF49570FEF7FBF940F26523C31AEF
:10850800584240EB030008BD08B5C620FEF7F0F955
:1085180040F28D13C21A504240EB020008BD4FF4DE
:10852800957040F26521FEF7D5B9C62040F28D114D
:10853800FEF7D0B9704760EEA00AB7EE007AF0EE09
:10854800606A70EE077A40EE006A47EEA70A36EED8
:10855800C77A08B5C7EE200A10EE900A06F0ACFEFE
:108568000022084B06F0FCFE0022074B06F046FDF1
:1085780007F0D8F907EE900AFDEEE77A17EE900AB1
:108588009F3008BD000059400000E03F38B52DED90
:10859800028BF7EE008AB0EE608A70EE288A10EE41
:1085A800900A28EE088A06F087FE08EEA88A0022BC
:1085B8000F4B06F0D5FE044618EE100A0D4606F0DD
:1085C8007BFE02460B462046294606F0F3FF0022B2
:1085D800084B06F013FD07F0A5F907EE900AFDEE2B
:1085E800E77A17EE900A7730BDEC028B38BD00BFF2
:1085F800000069400000E03FF0B5694D2DED068BA5
:1086080095E80F008DB008AE103586E80F000FCD45
:1086180001AC0FC495E807004FF6FF7384E8070024
:108628009F2077216422FAF75CF8A0207721642242
:108638004FF6FF73FAF755F89E20772164224FF61C
:10864800FF73FAF74EF89F20762164224FF6FF73E6
:10865800FAF747F84FF6FF73782164229F20FAF75C
:1086680040F80020FBF757FC9F2077216522FCF794
:108678000FFC9F2077216422FCF70AFC07AD0C361B
:10868800F7EE009A0435F7EE008A95ED009A4FF45C
:108698009674B0EE68AA18EE900A06F00DFE3EA396
:1086A800D3E9002306F05CFE07F03CF908EE900AD7
:1086B80038EEE98AB0EE490AF0EE480AFFF73BFFC8
:1086C800B0EE490AF0EE480A0746FFF75FFFBFB26F
:1086D80081B20F223846FBF703FD013CDBD14FF492
:1086E8009674F7EE008A18EE900A06F0E5FD2AA3C4
:1086F800D3E9002306F034FE07F014F908EE900AD7
:1087080039EEE88AB0EE490AF0EE480AFFF713FF9F
:10871800B0EE490AF0EE480A0746FFF737FFBFB246
:1087280081B20F223846FBF7DBFC013CDBD1B542B6
:10873800A8D16C4607AE043494ED009A4FF4C8757E
:10874800F7EE008A18EE900A06F0B6FD12A3D3E9F8
:10875800002306F005FE07F0E5F808EE900A38EE6B
:10876800CA8AF0EE490AB0EE480AFFF7E4FEB0EE16
:10877800480AF0EE490A0746FFF708FFBFB281B280
:1087880000223846FBF7ACFC013DDBD1B442D2D124
:108798000DB0BDEC068BF0BD295C8FC2F528F03F0B
:1087A80018A10408121A06EE902A081AB8EEE67AFA
:1087B80006EE900AF8EEE67AC7EE277A9FED047A7D
:1087C80067EE877AFDEEE77A17EE900A704700BFEA
:1087D8000000A0438A1A06EE902A081AB8EEE67A34
:1087E80006EE900AF8EEE67AC7EE277A9FED047A4D
:1087F80067EE877AFDEEE77A17EE900A704700BFBA
:108808000000484370B506460D460024610704D5AC
:10881800A0B231462A46FBF763FC0134B4F5A07FC9
:10882800F4D170BD70B506460D460024600704D526
:10883800A1B230462A46FBF753FC0134C82CF5D1C7
:1088480070BD114B11481B781149124A0068012B61
:10885800114B09D1126808601A60104B1A68104B46
:108868001A60104B1A680CE01268D2011A600B4BA0
:108878001A680B4BD2011A600A4B1A68C0010860CB
:10888800D201094B1A607047280F0020A83E00202B
:10889800A03E0020C4440020903E00209C440020BC
:1088A8003C3E0020783E0020BC440020024B1A6861
:1088B800024B1A60704700BFA03E0020A44400206D
:1088C80008B5FFF7BEFFBDE80840EFE770B5002127
:1088D8000A222748274D284E284C0BF0FFFB002181
:1088E8000A22286026480BF0F9FB00210A22306092
:1088F80024480BF0F3FB00210A22206022480BF0E9
:10890800EDFB224B326818602B68D31A06EE903ABA
:1089180023681F4AB8EEE67A06EE903AF8EEE67A51
:10892800C7EE277AFCEEE77A17EE903A01339BB24E
:1089380007EE903AB8EE677AF4EE007A67EE277A97
:108948001380FCEEE76A134B16EE901A8AB206EE15
:10895800902AB8EEE67A198077EEC77AF5EEC07AF3
:10896800F1EE10FA01DD01321A80BDE87040A7E788
:108978006C3E0020A83E0020C44400209C440020F7
:10898800943E0020A94400205C3E0020583E002070
:1089980004480020844800200022F0B51346202611
:1089A80003254FF02C0C00E02646303EF6B2174661
:1089B8000132092E10F8014B0AD897FBF5F605FB92
:1089C80016772FB9CE1801F803C07470023301E08E
:1089D800CC540133092AE7D12022CA54CB184822A3
:1089E8005A707A229A700022DA70F0BDF0B51F46EC
:1089F800144B1E788DB005460C4606B3A6F1040C40
:108A0800DCF1000646EB0C06CEB90F4908A80BF0BE
:108A180099F908A86946FFF7BFFF0C496A4604A8F8
:108A28000BF090F9BDF84800FCF7F0F93846FCF770
:108A380003FA2846214604AA3346FCF721FB0DB069
:108A4800F0BD00BF403E0020169C05085CA205084A
:108A58002DE9F04F7E4B2DED068B93ED008A78EED5
:108A6800087A7C4B85B017EE900A1C6806F024FC47
:108A780080462046894606F01FFC68EE088A41ECCD
:108A8800100BF7EE009ACDE9020108F0F9FB78EE39
:108A9800A97A57EC106B17EE900A06F00DFC3246D7
:108AA8003B4682468B464046494606F059FC0246FC
:108AB8000B465046594606F09FFA06F033FF79EE0A
:108AC800E88A09EE100AC8EE898ADFED637A9DED1F
:108AD800020B68EEA78A08F0D3FC404653EC102B33
:108AE800494606F03DFC064619EE100A0F4606F008
:108AF800E3FB02460B463046394606F05BFD574B12
:108B0800002206F02DFC06F00DFF09EE100A69EEB2
:108B1800097A48EEA87AB1EE49AA88EEA77A504BAE
:108B28005C60D8608AEE27AA83ED008AC3ED028ACA
:108B380083ED047A83ED05AA4A4B1B78033B042B8B
:108B48006ED8DFE803F00312254E3C0018EE900AB9
:108B580006F0B2FB044619EE100A0D4606F0ACFB0F
:108B6800CDE90001404841490DE017EE100A06F032
:108B7800A3FB04461AEE100A0D4606F09DFBCDE94C
:108B8800000139483A4922462B460BF0DBF847E00A
:108B980018EE100A06F090FB41EC100B08F0FCFCF4
:108BA8000022344B51EC100B06F0DAFB06F0BAFE4B
:108BB80006F082FB02460B462B482F492EE018EEA2
:108BC800100A06F079FB1EA3D3E9002304460D46DC
:108BD800DDE9020106F0C4FBCDE90001224827497E
:108BE800D1E718EE100A06F067FB17A3D3E90023B4
:108BF80006F046FEDFED227A002818BFB0EE678A3D
:108C080078EE297A79EEC89AC7EEA99A19EE900AF1
:108C180006F052FB02460B4613481A490BF092F82D
:108C2800114C00230220CA212246FCF729FA00230E
:108C3800237005B0BDEC068BBDE8F08FAFF3008064
:108C4800F6285C8FC2A54C40AE47E17A14AEEF3FE0
:108C580020450020244500200000484200004940EB
:108C6800E4470020B8440020F244002002A505088B
:108C780012A50508000034C022A5050834A505087A
:108C8800A4707D3F50A505082DE9F0434FF47F708F
:108C98008DB0FDF72DFE00271FFA80F86BE04FEA34
:108CA800C7091FFA89F909F580691FFA89F0FEF7E3
:108CB80031FB60F3070409F1010080B2FEF72AFBDB
:108CC80060F30F2409F1020080B2FEF723FB60F382
:108CD800174409F1030080B2FEF71CFB60F31F6420
:108CE80009F1040080B2FEF715FB60F3070609F1ED
:108CF800050080B2FEF70EFB60F30F2609F10600AF
:108D080080B2FEF707FB09F1070960F307051FFAB0
:108D180089F0FEF7FFFA60F30F25B0B206F0BAFA51
:108D280000221B4B06F01CFB06F0FCFD06F0C4FA03
:108D3800CDE90001A8B206F0ADFA11A3D3E90023EA
:108D480006F05AF910A3D3E9002306F033FC06F025
:108D5800E9FD06F0B1FA2246CDE902010D4905A860
:108D68000AF0F0FFC1B205A802F024FF0120FFF7C6
:108D78006FFA0137BFB2B84591DA0DB0BDE8F0839C
:108D880000000000C0FFDF40E17A14AE47C1664032
:108D98000000F03E5BA5050808B50021C620FDF7D8
:108DA80099FD4FF495700021BDE80840FDF792BD8C
:108DB800024B4FF6FF721A80704700BFF044002044
:108DC80000200146C82240F23F13FBF7E3BA07B57B
:108DD8000DF1070002F0EFFE9DF807000EBD08B583
:108DE800FFF7F5FF0028FBD108BD30B5044687B072
:108DF80010EE100A0D4606F05FFA02460B4601A86F
:108E080005490AF09FFF2046294601AA0023FCF7DE
:108E180037F907B030BD00BF6EA5050808B508488A
:108E280003F052FD0648022103F01FFE0028F9D086
:108E3800034803F075FD07EE900AB8EE670A08BD0F
:108E48000020014010B50C4C00232DED028B23802F
:108E58009FED0A8A06E0FFF7E1FF238838EE008AD3
:108E6800013323802388182BF5D99FED050A28EEB6
:108E7800000ABDEC028B10BD0C3E00200000000073
:108E8800ACC8683910B54FF4C770FDF731FDDB2861
:108E980005D14FF4C870FDF72BFD84B219E041F2FB
:108EA800E104214644F20100FDF714FD44F20100FB
:108EB800FDF71EFDA04214BF80244FF4007421B2B8
:108EC8004FF4C870FDF706FD4FF4C770DB21FDF7BE
:108ED80001FD204610BD024B00221A70704700BFEA
:108EE80024480020014B01221A70704724480020B2
:108EF800014B00221A6070471C450020014B18786E
:108F0800704700BF244800200030024B18BF0120E2
:108F180018707047254800200E4B1A680E4B1A60CF
:108F28000E4A002313700E4A13700E4A0121117065
:108F38000D4A4FF6FF7010800C4A13700C4B1A78CC
:108F48000C4B002A14BF052204224FF080401A70EF
:108F580005F061BAA03E0020A4440020883E00200D
:108F6800244800200E0E0020F04400203C4600203B
:108F7800180E0020190E002070EEA10A88B030EEFD
:108F8800010A08B0704770EEE10A88B030EE410A75
:108F980008B07047F0EE407A20EEA10A60EE810A30
:108FA80047EEA10A88B017EE810A08B07047D0B51D
:108FB80061EEA17A41EE017A2DED048B17EE900A4D
:108FC80088B0B0EE409AF0EE609AF0EE418AB0EECA
:108FD800618A06F071F90022002306460F4606F062
:108FE80027FCE8B969EE887A49EE287A29EE088ADA
:108FF80017EE900A06F060F932463B4606F0DAFAB8
:1090080019EEA88A06F08EFC044618EE100A06F03F
:1090180053F932463B4606F0CDFA06F083FC01E0F0
:109028000448044600EE900A00EE104A08B0BDEC71
:10903800048BD0BD0050C347F0EE407A86B020EED6
:10904800200A67EE810A06B07047064B93E80300D2
:1090580084B004AB03E90300DDED030A9DED020AC9
:1090680004B0704788480020F7EE007A77EEC07A9F
:1090780020EE022A20EE210A07EEA00AF0EE420AAC
:1090880047EE810A88B008B0704770B56D4B2DED7A
:10909800068B1A786C4B94B00E468DED020ACDED16
:1090A800030A22B91A68802392FBF3F200E01A68D7
:1090B800664C012E236C616CDFED659AB7EE00AA51
:1090C80051D002D3022E60D154E0D21A07EE102AF2
:1090D800CB1AB8EEC79A07EE103AF8EEC77AD4ED75
:1090E800000A89EE279A94ED011AD4ED021A94ED3C
:1090F800032AB0EE490AFFF7B7FF8DED000ACDED60
:10910800010A9DE8030006ABD4ED040A94ED051AA4
:10911800D4ED061A94ED072A83E80300B0EE490A55
:10912800FFF7A2FF8DED000ACDED010A9DE80300CF
:1091380008AB83E80300D4ED0C0A94ED0D1AD4EDC6
:109148000E1A94ED0F2AB0EE490AFFF78DFF8DED48
:10915800000ACDED010ADDED068A9DED078A04AB14
:109168009DE803000EE0D4ED008A94ED018A08AB77
:10917800103405E0D4ED028A94ED038A08AB183464
:1091880094E8030083E8030003E0B0EE698AF0EE98
:109198004A8ADDED030A9DED020A30EEC88A70EEB8
:1091A800688A9DED081ADDED091ACDED0C8A8DED62
:1091B8000D8AFFF7EFFE8DED000ACDED010A9DE85F
:1091C800030010AB83E80300DDED111A9DED101AC2
:1091D80079EEE11A3AEE411AB0EE680AF0EE480A62
:1091E8008DED0E1ACDED0F1AFFF7E1FE8DED000A99
:1091F800CDED010A9DE803000AAD6C4685E8030041
:109208008EB99DED040ADDED050A9DED0A1ADDED26
:109218000B1AFFF7BFFE8DED000ACDED010A9DE8A0
:10922800030085E803000AAB93E8030014AB03E9E5
:109238000300DDED130A9DED120A14B0BDEC068B98
:1092480070BD00BF280F0020A4440020384800202B
:109258000000000010B5244C4FF496702168FDF70B
:1092680056FB61684FF49870FDF751FBA1684FF405
:109278009A70FDF74CFBE1684FF49C70FDF747FBD3
:1092880021694FF49E70FDF742FB61694FF4A070AD
:10929800FDF73DFBA1694FF4A270FDF738FBE169CA
:1092A8004FF4A470FDF733FB216B4FF4A670FDF764
:1092B8002EFB616B4FF4A870FDF729FBA16B4FF4EF
:1092C800AA70FDF724FBE16B4FF4AC70FDF71FFBB0
:1092D800216C4FF4AE70FDF71AFB616C4FF4B0705F
:1092E800BDE81040FDF713BB3848002010B54FF417
:1092F8009670FDF725FB224C20604FF49870FDF71F
:109308001FFB60604FF49A70FDF71AFBA0604FF4E2
:109318009C70FDF715FBE0604FF49E70FDF710FBA5
:1093280020614FF4A070FDF70BFB60614FF4A27051
:10933800FDF706FBA0614FF4A470FDF701FBE061A7
:109348004FF4A670FDF7FCFA20634FF4A870FDF700
:10935800F7FA60634FF4AA70FDF7F2FAA0634FF4CE
:10936800AC70FDF7EDFAE0634FF4AE70FDF7E8FA84
:1093780020644FF4B070FDF7E3FA606410BD00BFDD
:109388003848002008B5FFF7B3F810B1BDE8084029
:10939800ACE708BD70B500F58065A8B2FDF7BAFF67
:1093A800294C2070681C80B2FDF7B4FF6070A81CBF
:1093B80080B2FDF7AFFFA070E81C80B2FDF7AAFFEE
:1093C800E070281D80B2FDF7A5FF002660F30706B0
:1093D800681D80B2FDF79EFF60F30F26B6B207EE58
:1093E800906AB8EE677ADFED197A194B67EE277A3B
:1093F800A81DC3ED007A80B2FDF78CFF0026073563
:1094080060F30706A8B2FDF785FF60F30F26B6B232
:10941800A6F5FE46FF3E07EE106AF8EEC77A17EE8D
:10942800900A05F049FF06A3D3E9002306F0C2F825
:1094380006F078FA074B22681860074B9A6170BDEE
:10944800CDCCCCCC0C5FC44028460020000080372F
:109458002045002024450020E447002073B5064637
:10946800002853D02A4B18888619B6B232B2002A7F
:1094780005DB40F23F139A42C8BF1E4600E00026B3
:10948800FAF742FEB0B24EF29C71FAF75FFE214D38
:109498001F4B214A1E8012682B6836B206EE906A6E
:1094A800D21AB8EEE67A06EE902AF8EEE67ADC21D1
:1094B80067EE277A9FED197AC7EE877A0520FDEEC9
:1094C800E77A17EE904A1C194FF6FF73224600936D
:1094D8000023FFF78BFA2B68E41A114B1B6894FBE7
:1094E800F3F407EE104AF8EEC77AFCEEE77A17EEC7
:1094F800900AC00080B2FFF74DFF0A4B0A481A785D
:109508000A4902B0BDE87040FFF7A2BA02B070BDC8
:10951800F0440020A83E0020C444002000809F435F
:109528009C440020B8440020204500202445002009
:10953800104B1B78022B13B51BD00F4C2389ADF8A9
:109548000630BDF806309BB243B1BDF806004EF2B6
:109558009C7180B2FAF7FAFD00232381074B1B7830
:10956800022B06D1064C94F90000FFF777FF002381
:1095780023701CBDB84400204C0E00203C4600203F
:10958800DC2D00202DE9F04F314D2DED088B2B7887
:10959800022BCDB009D12F4B1A682F4B42F2107015
:1095A8001A60FDF795FF00F068BE2C4B1B78B7EEEC
:1095B80000AADFED2BBA002B40D02A4C2068C0004F
:1095C80080B2FFF7E7FE284B28491A782848FFF7AA
:1095D8003FFA284B2849D3F81880D3F80490098813
:1095E80093ED009A79EE0A8A7AEE497A93ED038A26
:1095F800C8EEA78A002293ED04BAD3ED05AAD3EDED
:10960800029A1E4BF4EE6B8ADA601A610022F1EEC0
:1096180010FAC8BFF0EE6B8AF4EE4A8A5A612368E2
:10962800F1EE10FA48BFF0EE4A8A01338B4223600C
:1096380040F31B8202232B70226016E2104B1A782B
:10964800054BFAB91A68802392FBF3F81CE000BFB7
:109658003C460020A03E0020A4440020180E002014
:10966800003C1C461C450020B8440020244500202E
:1096780020450020E4470020044800204C0E00202C
:10968800280F0020D3F80080FEF7B4FBCC4D85ED01
:10969800060AFEF7B5FBA86985ED070A10EE104A21
:1096A80005F00AFE064620460F4605F005FE41EC89
:1096B800100B41EC180B07F0E3FD5BEC10ABB0EEC0
:1096C800480AF0EE680A07F0DBFE52465B46304671
:1096D80039468DED040B05F043FE06F023F9DFED66
:1096E800B98A07EE900A9FEDB88A17EEA88AB74C98
:1096F800DDE9042384ED008A3046394605F030FE62
:1097080006F010F900EE900A60EEA80AB0EE480ADA
:109718000021AF48C4ED010AFFF7B7FC8DED0E0A32
:10972800CDED0F0A0EAA92E80300AA4B83E80300C6
:1097380093ED018ADFEDA87AB4EE6B8AF1EE10FAA8
:10974800C8BFB0EE678ADFEDA57AB4EE678AF1EE9E
:1097580010FA48BFB0EE678AFDEE007AB4EEE78AE9
:10976800F1EE10FAD3ED009A08DDB5EE408ADFED90
:109778009C7AF1EE10FA48BFB0EE678A68EE088A64
:10978800DFED987AB0EE68BA09EEA9BA19EE900A38
:10979800B5EE40BAF1EE10FA08BFB0EE67BA05F0C0
:1097A8008BFD0022904B06460F4605F025FC04462B
:1097B80018EE900A0D4605F07FFD224682468B463C
:1097C8002B462046294605F0CBFD52465B4605F060
:1097D80015FC41EC100B07F065FF002230463946B6
:1097E800814B8DED040B05F009FC02460B4605F094
:1097F800B7FD52465B4605F001FC41EC100B07F043
:1098080051FFDDE9040155EC104B06F08BF82946B1
:1098180008EE900A204606F085F809EE100A88EE50
:10982800899A724CF1EE48AACAEE8BAA89EE8BBAD5
:1098380019EE100A05F040FD5BA3D3E9002306F0FA
:1098480001F8DFED6B7A002818BFB0EE679ADFEDFC
:10985800697A6AEEA77AB4EE4A9ADFED678AF1EE82
:1098680010FA17EE900AC8BFB0EE689A05F024FD0A
:10987800DFED627A4BEE4B7A4AEEEA7A06460F46FD
:1098880017EE900AC4E9026705F016FD47EC106B65
:1098980041EC110BC4E9000107F07CFE51EC100B00
:1098A80006F040F8B4EE4A9AF1EE10FAA8BFB0EE0E
:1098B800689A7AEE497A79EE0A8A514BC8EEA78AF5
:1098C8001B78DFED457AF4EE6B8AF1EE10FAC8BF2B
:1098D800F0EE678AF4EE4A8AF1EE10FAF7EE007AB3
:1098E80048BFF0EE678A022B80F0004940F0B18053
:1098F800444B1B78002B00F0AC80434B434C1B6857
:109908001C40002C03DA013C64F0070401340826EB
:1099180019EE100A93FBF6F605F0CEFC00223C4B3C
:1099280005F01EFD05F0DEFF05460746484605F032
:10993800C3FC1FA3D3E9002305F012FD1EA3D3E93E
:10994800002305F05BFB05F0CDFF324B1C49C3F843
:10995800008001EBC403C8F3072283F82120C8F371
:109968000742B60183F8222083F824504FEA186290
:10997800C5F3072583F82600072CC0F30720B6B2E5
:1099880083F8208083F8232083F8255083F8270064
:1099980042D106F5806080B220314022FDF73AFEC0
:1099A800D0B3FEE7AFF300802D431CEBE2361A3F3D
:1099B800CDCCCCCC0C5FC44000000000C0FFDF4021
:1099C8004C0E00200000F04200008C428848002025
:1099D8003848002034460020003C1C46003C1CC689
:1099E800CDCC4C3D5F7089300000494010480020C4
:1099F80017B7D1380AD7233D72F97F3F17B7D13946
:109A0800403E0020244800201C450020070000801C
:109A18000000F04028460020A14CA24B22681B8879
:109A28009A4212DB06F58066B0B29F494022FDF7E4
:109A3800F1FD054600B1FEE7B4F900104FF47F7060
:109A4800FCF748FF994B25601D70954B1A68013249
:109A58001A60FEF7E7F9964C84ED030AFEF7E8F979
:109A680084ED040AFCF702FF6061914C914942467B
:109A780038A80AF067F9E06805F01EFC02460B46B4
:109A880028A88D490AF05EF9206905F015FC024600
:109A98000B462CA889490AF055F91BEE100A05F067
:109AA8000BFCCDE90401DDE90423854930A80AF05F
:109AB80049F91AEE900A05F0FFFB82468B4652469A
:109AC8005B46804934A80AF03DF919EE900A05F082
:109AD800F3FBCDE90C01DDE90C237B4914A80AF05E
:109AE80031F918EE100A05F0E7FBCDE90801DDE9C8
:109AF8000823764918A80AF025F919EE100A05F086
:109B0800DBFBCDE90A01DDE90A2371491CA80AF04B
:109B180019F9484605F0D0FBCDE90601DDE9062331
:109B28006C4920A80AF00EF918EE900A05F0C4FB5B
:109B380002460B4624A868490AF004F910A86749A8
:109B480062690AF0FFF8B5EEC08AF1EE10FADFEDAF
:109B580064AA37D5404605F09DFB4BA3D3E9002303
:109B680005F0FEFBF1EE487A044617EE900A0D4622
:109B780005F0A2FB02460B462046294605F0F0FBFD
:109B880002460B4642A1D1E9000105F013FD05F09C
:109B9800C9FE9FED547A07EE900AF4EEC77AF1EE0B
:109BA80010FAC6BFC7EEAA7A4F4C504CF4EEEA7AC8
:109BB800F1EE10FA36DD9FED4A7A4D4D4D4CC7EE69
:109BC800877A32E034A3D3E90023DDE9080105F000
:109BD800C7FB044640460D4605F05CFB2AA3D3E9C3
:109BE800002305F0BDFB02460B462046294605F03A
:109BF800E1FC05F097FE07EE900AF4EECA7AF1EE62
:109C080010FA46BF67EEAA7A3B4C3C4CF4EEEA7A6F
:109C1800F1EE10FA08DD9FED327A394D394CC7EE76
:109C2800877A02E0324D00E0354D17EE900A05F0D4
:109C380043FB2A46CDE900013CA8334902940AF0C7
:109C480081F8324B1D68324B1C68194BA045CCBFBC
:109C580000260126A845D8BF00261E662D4B1B7876
:109C6800013BDBB2012B00F2FA822B4B1B78072B4E
:109C780000F2F582DFE813F05200F302E300A001DE
:109C880000025502B60270021F85EB51B81E19403A
:109C9800000000A2941A6D420000000080842E414A
:109CA8001C450020044800206C0E00202448002099
:109CB8004C0E002088A5050892A505089DA5050855
:109CC800A8A50508B2A50508BCA50508C7A50508E7
:109CD800D2A50508DDA50508E8A50508F4A5050829
:109CE80000007A440024744979A5050876A505087A
:109CF800A1A6050882A505087FA505087CA5050875
:109D0800AA9D050885A5050801A60508A83E002006
:109D1800C4440020403E0020B8440020964B1C78E4
:109D2800002C40F09C820220FBF772F94FF6FF707E
:109D3800FBF782F81F20FBF769F819218F4A2346A1
:109D48002D20FBF79DF94FF6FF70FBF775F82046BD
:109D5800FBF75CF80F20B42142464FF6FF730094DE
:109D6800FEF744FE0F206E2128AA2346FBF788F948
:109D7800A0206E212CAA2346FBF782F90F20382158
:109D88001CAA2346FBF77CF9A020382120AA2346E9
:109D9800FBF776F90F205C2130AA2346FBF770F910
:109DA800A0205C2134AA2346FBF76AF90F204A2138
:109DB80014AA2346FBF764F9A0204A2118AA2346CF
:109DC800FBF75EF90F209B21234624AAFBF758F9DD
:109DD8006B4B1B78012B05D10F2084213CAA23460D
:109DE800FBF74EF9674B5B69B3F57A7FCCBF4FF44D
:109DF800FC604FF47840FBF71FF80023A0209B215C
:109E080010AAFBF73DF9604B1B78012B08D14FF4E2
:109E1800FC60FBF711F84FF48C7002215B4A07E0F5
:109E28004FF6E070FBF708F8594A4FF48C7002219E
:109E38000023FBF725F91F20FAF7FEFF0FE2DDE903
:109E48000423544946A809F07DFF534952465B460E
:109E580049A809F077FF5149DDE90C2340A809F02A
:109E680071FFDDE908234E4943A809F06BFFE6209E
:109E78000221002346AAFBF703F9E6201621002356
:109E880049AAFBF7FDF80220C821002340AAFBF7E6
:109E9800F7F8002343AA0220DC21FBF7F1F8DFEDF5
:109EA800417A29EE279A19EE100A05F005FA9DED78
:109EB800060B06460F4607F0E3F9304653EC102B25
:109EC800394605F04DFA28A3D3E9002305F096F8A2
:109ED80005F0E0FC9DED060B044607F0D1FA30468C
:109EE80053EC102B394605F03BFA02460B4620A1ED
:109EF800D1E9000105F080F805F0CCFC054600200A
:109F0800FAF79AFF4FF6E073009305200A214246BC
:109F18000023FEF76BFD1B4B1B6E53B1224B1888B9
:109F2800224B4FF4784619880096A2B2ABB2FAF7E2
:109F3800F9FE1D4B1C601D4B4FF478441D609D209D
:109F48007721052200230094FAF790FF9F207521BE
:109F5800052201230094FAF789FF4FF6E070FAF71B
:109F680055FF7CE1AFF300800000000000E0634093
:109F78000000000000C05D40180E00200EA6050875
:109F8800403E00204C0E0020280F00202DA605087A
:109F980031A6050835A605083FA6050849A60508FF
:109FA80053A605080000C84230460020904800200B
:109FB8000000FA43000000005FED038A21462846AE
:109FC8004246FEF7EFFBF4EE689AF1EE10FAC8BFCE
:109FD800F0EE689AF5EE409A5FED0A7AF1EE10FA23
:109FE80048BFF0EE679AF4EEE89AF1EE10FA0446EC
:109FF8001CD8F4EEE79AF1EE10FA17DBFDEEE99AB9
:10A00800002019EE902A4FF4FA71FEF7E3FB05469B
:10A0180056B1AB4B1888AB4B4FF6FF7619880096B4
:10A02800A2B2ABB2FAF77EFEA64B1D60B4EE688A08
:10A03800DFEDA57AF1EE10FAC8BFB0EE678ADFED62
:10A04800A37AB4EE678AF1EE10FA48BFB0EE678AD9
:10A05800B4EEE88AF1EE10FA00F20181B4EEE78A74
:10A06800F1EE10FAC0F2FB80BDEEC88A984818EEEF
:10A07800102A4FF4FA71A2E0214628464246FEF71C
:10A0880091FBB5EEC0BAF1EE10FA044625DDDDE924
:10A0980004017DA3D3E9002305F0D4FBE8B17CA338
:10A0A800D3E90023DDE9040105F05AF902460B461D
:10A0B8000020884904F0A0FF05F0ECFB054656B1E6
:10A0C8007F4B18887F4B4FF6FF7619880096A2B20F
:10A0D800ABB2FAF727FE7B4B1D60504659466EA37C
:10A0E800D3E9002305F0CCFB002800F0B8805046E7
:10A0F800594665A3D3E9002305F0A4FB002800F026
:10A10800AE8067A3D3E900235046594605F028F9E5
:10A1180002460B460020704904F06EFF05F0BAFBBA
:10A128004FE0214642462846FEF73CFB5EA3D3E9B2
:10A1380000230446DDE90A0105F0A2FB50B19DEDBC
:10A148000A0B07F029FA002251EC100B634B05F0BB
:10A1580007F96FE0C82570E055A3D3E90023DDE9CE
:10A16800060105F0FDF854A3D3E9002305F022FA0F
:10A1780005F0D8FB214608EE100A42462846FEF7AD
:10A1880011FBDFED577A49EE677A0446FDEEE77A70
:10A1980017EE905A56B14A4B18884A4B4FF6FF763D
:10A1A80019880096A2B2ABB2FAF7BCFDBDEEC88A18
:10A1B800444B18EE102A1D606FF0B300B421FEF76F
:10A1C80009FB484B1B6E054653B13D4B1888464B5F
:10A1D8004FF4FC6619880096A2B2ABB2FAF7A2FD5A
:10A1E800414B39E0DFED417AF4EE678AF1EE10FA7F
:10A1F800C8BFF0EE678AF4EEE78AF1EE10FA2ED8BF
:10A20800424621462846FEF7CDFA044618EE900A43
:10A2180005F052F841EC100B07F0BEF900222E4B66
:10A2280051EC100B05F09CF802460B46002029491A
:10A2380004F0E2FE05F02EFB05462A4B1B6E53B1D7
:10A248001F4B18881F4B4FF6FF7619880096A2B24D
:10A25800ABB2FAF767FD1B4B1D60194B1C60244B12
:10A268001B78022B09D043B14FF6FF7300930520EA
:10A27800DC2142460023FEF7B9FB4DB0BDEC088B4C
:10A28800BDE8F08FAFF300809A9999999999B93FF1
:10A298000000000000409F409A9999999999B9BF88
:10A2A8000000000000408F4089B5F81400E3693FC2
:10A2B80000000000008076401F85EB51B81E194051
:10A2C80030460020904800200000FA430000FAC3FE
:10A2D8000CFEFFFF0000694000005940000054C018
:10A2E800000048434C0E0020104500200000C842E2
:10A2F800B8440020AFF300807047FEE7FEE7FEE7B2
:10A30800FEE7704770477047FDF798BF10B5094CD6
:10A31800A37A4BB1084B1A6822F006021A6000F0C3
:10A3280013F8204600F079FE4FF48020BDE8104075
:10A3380002F0C4BDAC3E002010ED00E0014801F081
:10A348003BB800BFAC3E0020364BD3F8882042F41F
:10A358007002C3F88820344B1A6842F001021A6070
:10A3680000229A60196821F0847121F48031196003
:10A378002E495960196882B021F480211960DA6089
:10A38800009201921A6842F480321A601A6802F444
:10A3980000320192009A01320092019A1AB9009A89
:10A3A800B2F5A06FF2D1204B1B6813F4003318BF2D
:10A3B80001230193019B012B2ED11B4B1A6C42F0F8
:10A3C80080521A641A4A116841F4804111609A68EF
:10A3D8009A609A6842F400429A609A6842F4A052DD
:10A3E8009A60144A5A601A6842F080721A601968B2
:10A3F8000D4A8901FBD5104B40F20561196093683D
:10A4080023F003039360936843F002039360936817
:10A4180003F00C03082BFAD1024B4FF000629A604C
:10A4280002B0704700ED00E0003802401030002410
:10A438000070004008544007003C0240184B194A7D
:10A44800996801F00C01042903D0082903D0164BA0
:10A4580019E0164B17E059685A6811F4800F5968CB
:10A4680014BF124B104B02F03F02B3FBF2F30C4A3D
:10A478005268C2F30142C1F38811013252004B43C2
:10A48800B3FBF2F3074A1360054B9A68054BC2F316
:10A4980003129A181968127921FA02F21A607047A1
:10A4A80000380240F00200200024F40000127A0074
:10A4B80037B51C230124002501A88DF804308DF838
:10A4C80005508DF806408DF80740FDF785FA2046BF
:10A4D800214603F063FB0A494CF24F334B60A3F566
:10A4E80042430B800D814D804FF0804003F0FEFE0B
:10A4F8004FF080402146224604F0BDFA3EBD00BF21
:10A508009848002038B54FF08040012104F0C8FA7F
:10A5180000283ED04FF0804001211E4D04F0CBFAB8
:10A528004FF08040002103F076FF2B78013B042B8D
:10A538002FD8DFE803F003070B102200BDE83840EE
:10A54800F6F736B9BDE83840F6F764B9F6F7B6FA63
:10A5580000232B7038BD104B00242C7001251D7072
:10A56800FEF7C0FCFEF7C4FC0C4B1D700C4B1878B2
:10A57800F6F78EFB0B4B1C7038BD00242C70FEF7D1
:10A58800B7FC064B1C70064B1878F6F781FB054B99
:10A598001C7038BD190E00203C460020883E002063
:10A5A800B84400200E0E002008B5402002F078FCC8
:10A5B80030B1FAF7C3FE4020BDE8084002F07EBC87
:10A5C80008BD0000014608B5044804F033FC034800
:10A5D800402104F0DCFC0028F9D008BD004400400C
:10A5E800F0B589B04FF4E1330120019300232B4CDF
:10A5F800ADF808301E460146ADF80A30ADF80C300B
:10A60800ADF810300C23ADF80E3003F0A3FA4FF478
:10A618000030012103F0C2FA20680221072202F06B
:10A6280071FF07226068032102F06CFF01250227F1
:10A6380004232068059305A98DF81A608DF81B502E
:10A648008DF818708DF8197002F0DCFE0823606828
:10A65800059305A98DF8187002F0D4FEA06801A929
:10A6680004F03EFB2A4640F225510D4804F076FCE2
:10A67800262307A88DF81C308DF81D608DF81E6004
:10A688008DF81F50FDF7A8F9A068294604F0A5FB2E
:10A69800044A054B1A6009B0F0BD00BF040300204E
:10A6A80000440040CDA5000804520020024B9868E1
:10A6B800002104F092BB00BF0403002010B5094C30
:10A6C80040F22551204604F06CFC50B1A288D2B269
:10A6D800112A02D1044B01211970044B19884A40F0
:10A6E8001A8010BD00440040120E0020B40E002055
:10A6F8007047704773B50120014603F02BFA264CCA
:10A708004FF4D8530093022303268DF804302046D3
:10A71800002369468DF806308DF807308DF80560FE
:10A7280002F070FE204608210A2202F0EBFE2046C5
:10A7380009210A2202F0E6FE20460B210A2202F035
:10A74800E1FE0A2220460C2102F0DCFE01254FF42E
:10A7580080632046694600938DF806508DF80750AF
:10A768008DF8056002F04EFE0A210A46204602F0E6
:10A77800C9FE29464FF4804003F01CFA8020294680
:10A7880003F0F4F94FF08050294603F043FA2846C5
:10A7980002F094FB7CBD00BF0000024007B54FF4F7
:10A7A800C060FDF70FF943238DF80430032201231D
:10A7B80001A88DF805308DF806208DF80730FDF7D3
:10A7C8000BF90EBD782358430723B0FBF3F00023A1
:10A7D80001338342FCD970474FF47A735843F1E749
:10A7E80037B50023104C019305460320FFF7EAFF15
:10A7F800EB681A69013C019213D0019A002AF4DA35
:10A80800019A42F001020192019A1A61064A1969F5
:10A81800013A019102D00199C907F8D40320FFF742
:10A82800D1FF00203EBD00BF410D030010B5C47824
:10A8380074B900EB820003339B10D0F8D000224695
:10A8480003E051F8044C0132046004319A42F8D113
:10A85800002010BD033230B59210D0F8D0400B461E
:10A86800002003E02568013043F8045C043390427B
:10A87800F8D101EB800030BD0122F0B500238270D1
:10A8880040220129C37082800CD10823037004235D
:10A8980043704FF4A073C38002230372C1724FF058
:10A8A800A04309E041B90C230370062343704FF419
:10A8B800A063C3801F4BC17203F500620261C360CD
:10A8C8004678044601461A46002508E002F5106C51
:10A8D80002F530620A65C1F814C001353A46043100
:10A8E800B54202F12007F1D303F58062426103F516
:10A8F8008862C0F8CC20067803F5A06501460022DE
:10A9080003E0C1F88C50013220350431B242F8D34B
:10A918001946002202E0C4F8CC1001320434B242D5
:10A9280001F58051F7D303F56063C0F80C310020BE
:10A93800F0BD00BF0000044038B5037AC2680025A6
:10A94800012B044625D1936B417A65F3104309B175
:10A9580043F480139363D36823F4800323F05003F4
:10A9680043F010036FF3C3036FF3C7136FF351433F
:10A978006FF3D343D3602046FFF732FFE378012B10
:10A988003ED1052363F34405E36845F020059D6047
:10A9980036E0D36843F04003D360FFF721FF237A02
:10A9A800627A032B14BF4FF434134FF43C130AB1EB
:10A9B80043F48013E26814209363FFF70DFFE26805
:10A9C800217AD368032908BF43F48033D360237AFC
:10A9D800032B15D1156B012363F39B656FF3D755D3
:10A9E8002D2345F0805563F316451563C820FFF7FE
:10A9F800F3FEE36845F400051D63C820FFF7ECFE8D
:10AA0800E378012B07D1E3689D68052262F34405CA
:10AA180045F020059D60002038BDC3689A6842F063
:10AA280001029A6000207047C3689A6822F0010208
:10AA38009A600020704707B500230193019B43F0FB
:10AA480020030193019B61F38A130193019BC26860
:10AA58001361064B1169013B019102D001998806E7
:10AA6800F8D40320FFF7AEFE00200EBD410D030011
:10AA780007B500230193019B43F010030193019B49
:10AA8800C2681361064B1169013B019102D001991B
:10AA9800C906F8D40320FFF795FE00200EBD00BFBD
:10AAA800410D030008B5C268D36801296FF35D73CF
:10AAB8006FF39E7302D143F0005302E009B943F0EB
:10AAC80080433220D360FFF787FE002008BDC368AB
:10AAD800586900F001007047C3685B6913F0010F03
:10AAE80014BF002001207047C368586900F00100B6
:10AAF8007047C3685A69986910407047C3685868B6
:10AB0800704703691A6861F301021A607047C268E6
:10AB1800002393614FF0FF335361536053610B4B34
:10AB28009361C3789169002B14BF4FF400634FF40D
:10AB3800016343F4701343F4405343F0080321EADC
:10AB480003010B4393610020704700BF0008008099
:10AB5800F8B5D0F80C3100221A60036915461A6856
:10AB680065F3CC221A60C37A012B04461BD103215A
:10AB7800FFF7C7FFE36880214FF4800261F30F02FB
:10AB880059629A62C02262F30F0561F31F454FF4C0
:10AB9800A072C3F8045162F30F056FF31F45C3F8A1
:10ABA8000851C3F80C5110212046FFF744FF2046F6
:10ABB800FFF75EFF226900234FF0FF311361204643
:10ABC80053611E469161FF25D361214610E08269D9
:10ABD8001768C7F3076707F08007FFB2002F14BF95
:10ABE8004FF09047002717600133166104309560D5
:10ABF80062789342EBD300231D46FF2010E04A6D94
:10AC08001668C6F3076606F08006F6B2002E14BF73
:10AC18004FF09046002616600133156104319060AC
:10AC280062789342EBD323691A6942F480721A61FD
:10AC3800E278012A04D1054A402161F359421A6396
:10AC48002046FFF764FF0020F8BD00BF03010100A4
:10AC580003699B68C3F34103013B022B9ABF024A75
:10AC6800D05C0320704700BF60A1040810B50369D9
:10AC780081699C680A68C4F34100022802D06FF316
:10AC88000A0202E0032060F30A020A605A6842F4EA
:10AC980080725A60002010BD30B54D780B780022C4
:10ACA800012D00EB830405D105FA03F3A46963F3CE
:10ACB8000F0205E0012505FA03F3646D63F31F42F3
:10ACC8002368C3F3072505F08005EDB26DB98D68DB
:10ACD80065F30A03CD78C98865F3934361F3995303
:10ACE80043F0805343F4004323600369D9690A435E
:10ACF800DA61002030BD30B54D780B780024012D85
:10AD0800224600EB830105D105FA03F3896963F351
:10AD18000F0205E0012505FA03F3496D63F31F42AD
:10AD280003696FF3CF340C60D96921EA0202DA6152
:10AD3800002030BDF8B54F780B78012F00EB830366
:10AD480049D19E694C69356833692A4664F3120310
:10AD580014B967F3DC430BE08F68E419013CB4FBDA
:10AD6800F7F7CC7867F3DC43012C08BF64F35E7314
:10AD78003361C378012B06D10B780C6900EB830390
:10AD88009B695C610CE0CB78012B09D04B693BB126
:10AD980003690C785E6B012707FA04F434435C639B
:10ADA800CB78012B07D103699B68DB0554BF45F0BD
:10ADB800005245F080520B7800EB830342F00442C6
:10ADC8009B691A60CB78012B38D10A788B8AC968BD
:10ADD800FFF72CFD32E05E6D4F6935688C6833698A
:10ADE8002A462FB964F31203012464F3DC430AE012
:10ADF8003F19013FB7FBF4F7BF05BF0D67F3DC430D
:10AE08007C4364F312033361C378012B05D10B78BB
:10AE18000C6900EB83035B6D5C61CB78012B06D179
:10AE28004B7913B145F0005201E045F080520B78A0
:10AE380000EB830042F00442436D1A600020F8BD25
:10AE480073B54D78012D3DD183694A691E681C6927
:10AE58000094E4B242B962F306048DF800409DF80C
:10AE6800024065F3C4040EE08D68AA4286BF4D61B6
:10AE780065F3060462F306048DF800409DF802406D
:10AE8800012262F3C4048DF80240009A1A61C27864
:10AE9800012A05D10A780C6900EB82029269546193
:10AEA80046F004421A60C378002B34D14B69002B5A
:10AEB80031D003690A78586B012101FA02F2024382
:10AEC8005A6328E00B784E698C6800EB83035B6D4E
:10AED8001A681D690095EDB206B14C6164F3060568
:10AEE8009DF802408DF80050012565F3C4048DF8E3
:10AEF8000240009C1C61C378012B05D10B780C69BA
:10AF080000EB83035B6D5C610B7800EB830042F020
:10AF18000442436D1A6000207CBD4B78012B0B78EE
:10AF280000EB83000AD182691368C3F3076101F05B
:10AF38008001C9B221B143F0804301E0426D13683A
:10AF480043F400131360002070474B78012B0B78F3
:10AF5800C97800EB83000CBF8269426D023913681F
:10AF6800C9B26FF35553012998BF43F0805313605A
:10AF78000020704703699A69D8691040000C70472F
:10AF880000EB810102694B6D9B685069184070475E
:10AF980003699869DB69184080B2704782B0002362
:10AFA8000093C0238DF803300122002362F3C40309
:10AFB8008DF8023018238DF80030009A436D1A611D
:10AFC800C278012A06D100F5B96058611A684FF0B5
:10AFD80080221A6002B07047D0F8143110B50446C8
:10AFE800D3B103699A68D20716D5827A42B1D0F8EC
:10AFF8000C21D0F80C116FF341026FF300020A60C4
:10B008005A6842F001025A600520FFF7E5FB236900
:10B018005A6822F001025A6010BD837A63B103694D
:10B028009B68D90708D5D0F80C31D0F80C216FF3FC
:10B0380041036FF3000313607047012310B500222A
:10B0480080F8123104460346FF2104E05869816004
:10B05800186D01328160607804338242F6D3236927
:10B0680000221A615A61DA614FF0FF329A61204674
:10B07800FFF7FEFC20461021BDE81040DBE44B78CA
:10B08800012B0B7800EB83000FD183691868C0F39C
:10B09800074000F02003DBB2CBB900F00200C0B2D9
:10B0A80000280CBF302020207047436D1868C0F37B
:10B0B800074000F02003DBB25BB900F00200C0B229
:10B0C80000280CBF4FF440504FF400507047102038
:10B0D80070474FF4805070474B78012B0B7810B5B0
:10B0E80000EB83030AD19C69102A236802D1BDE8CA
:10B0F800104012E7202A0CD0302A0FE05C6DB2F520
:10B10800805F236802D143F400131BE0B2F5005FAF
:10B1180002D143F0006315E0B2F5405F0FD1C3F3ED
:10B12800074202F02002D2B222B100234B71BDE8DF
:10B1380010400AE743F0806343F0802302E00AB935
:10B1480062F3CF33236010BDF8B50446FFF794FBD4
:10B158000122002384F8122184F813312827164687
:10B16800194640250CE007FB03F000F58C70221807
:10B178002354D3805670D1709560D16051610133EA
:10B1880062789342EFD300232826194640250CE025
:10B1980006FB03F000F55C7022182354D38051702D
:10B1A800D1709560D1605161013362789342EFD3D9
:10B1B8002046FFF739FC2046FFF7BEFB002120465A
:10B1C800FFF770FC2046FFF7C3FC2046BDE8F840B7
:10B1D800FFF723BC70B5CDB20C464FF0280601F03E
:10B1E8007F0106FB010115F0800F14BF01F58C717A
:10B1F80001F55C7104F07F04ED090C704D708A60F4
:10B20800CB7005B1CC80022B01D100230B71FFF765
:10B2180043FD002070BD10B5CAB201F07F034FF0A6
:10B22800280404FB030312F0800F14BF03F58C738A
:10B2380003F55C7301F07F01D20919705A70194641
:10B24800FFF759FD002010BD38B501F07F0528240F
:10B258006C4304F55C7401194B6100238B614B70DE
:10B26800EBB20355CA60C478012C08BF0A6113B950
:10B27800FFF7E6FD01E0FFF75DFD002038BD70B582
:10B2880001F07F042825654305F58C7541190126D1
:10B29800E4B2CA600A6100224E7044558A614B616B
:10B2A80014B9FFF7CDFD01E0FFF744FD002070BDA4
:10B2B800CAB212F0800F10B54FF0280306D001F083
:10B2C8007F0403FB040303F58C7303E003FB010312
:10B2D80003F55C73D209012401F07F0119709C7099
:10B2E8005A701946FFF719FE002010BDCAB212F0B5
:10B2F800800F10B54FF0280306D001F07F0403FB40
:10B30800040303F58C7303E003FB010303F55C738B
:10B318000024D20901F07F0119709C705A701946F7
:10B32800FFF713FE204610BD08B50B0604D501F043
:10B338007F01FFF780FB01E0FFF79AFB002008BDC3
:10B348000369002261F30A1219680A431A607047F8
:10B3580003695A6803206FF341025A60FFF73CBA49
:10B3680003695A68032042F002025A60FFF734BAB0
:10B3780011F0800F4FF0280306D001F07F0103FB86
:10B38800010101F58C7103E003FB010101F55C711A
:10B39800FFF775BE11F0800F4FF0280306D001F0BB
:10B3A8007F0103FB010101F58C7103E003FB01013F
:10B3B80001F55C71FFF790BE2DE9F74F0446FFF7E2
:10B3C8008BFB002800F03F822046FFF792FB0546E2
:10B3D800002800F03882C0F3074000F00800C0B22F
:10B3E800002861D02046FFF7C5FDA14682462746C2
:10B3F8004FF00008DFF86CB32E4650E01AF0010F4A
:10B4080046D05FFA88F2114620460092FFF7B8FD51
:10B4180010F0010F0546009A20D07B6D01259D6034
:10B42800E178A94207D11B69D9F87813C3F312034D
:10B43800CB1AC9F88833DBF8003020461B68114660
:10B448009847E378012B09D1B8F1000F06D194F899
:10B458001131052B02D12046FFF7A0FD05F00203AC
:10B46800DBB213B17B6D02259D6005F00403DBB2EE
:10B4780013B17B6D04259D6005F00805EDB23DB163
:10B48800DBF8003020469B6898477B6D0820986061
:10B4980008F101084FEA5A0A043709F12809BAF1F4
:10B4A800000FABD135460120C5F3074303F0040371
:10B4B800DBB2002B00F0AF802046FFF769FD26467F
:10B4C80083464FF0000801959FE01BF0010F00F044
:10B4D800978023695FFA88F919695D6B04EB890223
:10B4E80025FA09F59269ED019268EDB20D43154010
:10B4F800EA071CD55A6B012000FA08F122EA01027A
:10B508005A63B369974A9860136805465B68204692
:10B5180049469847E378AB4209D1B8F1000F06D104
:10B5280094F81131042B02D12046FFF737FD05F0BE
:10B538000403DBB213B1B36904259D6005F0080369
:10B54800DBB213B1B36908259D6005F01003DBB2C7
:10B5580013B1B36910259D6005F02003DBB213B168
:10B56800B36920259D6005F04003DBB213B1B369D0
:10B5780040259D6005F00203DBB213B1B3690225D3
:10B588009D6025F07F0515F0FF0F39D0282505FBB4
:10B59800084505F58C75C246AB696A69C3EB020CB0
:10B5A800AB689C4528BF9C460CF1030CB3694FEA75
:10B5B8009C0C9B696746A04614E0AA68E9681C1BB6
:10B5C800944228BF1446A3B240464A46FFF72EF9D4
:10B5D800EB681B19EB60AB69E71C1C19AC61B3691C
:10B5E8009B69BF089BB2BB4205D9AC696B699C4299
:10B5F80001D2002BE1D1B369802544469D60D04635
:10B6080008F101084FEA5B0B0436BBF1000F7FF429
:10B618005CAF019D012005F00203DBB213B1E368C2
:10B6280002225A61C5F3076303F08003DBB2CBB192
:10B63800A37A43B1D4F80C31D4F80C216FF3410349
:10B648006FF30003136023695A6822F001025A60FD
:10B65800444B1B6820469B699847E3684FF00042BB
:10B668005A610120C5F3072303F00803DBB2F3B1E5
:10B678003C4B1B6820465B6998472369E2689B68D6
:10B688004FF400615161A27A82B1DB070ED5D4F87C
:10B698000C311A6842F001021A601A6842F003027B
:10B6A8001A60314B1A6942F006021A61012005F04E
:10B6B8000803DBB243B12B4B1B682046DB68984775
:10B6C800E36808225A61012005F01003DBB2002B61
:10B6D80033D0E3689A6922F010029A611F6A28261B
:10B6E80007F00F0306FB0346C7F34343022B06F597
:10B6F8005C7602D0062B1AD10EE047F6F0733B4079
:10B70800ABB1C7F30A172046F1683A46FFF7A2F82B
:10B71800F368DB19F36007E004F5B96120460822F5
:10B72800FFF798F8C7F30A17B369DF19B761E36839
:10B738009A6942F010029A610120C5F3072303F0C9
:10B748001003DBB2002B39D023695A68002622F097
:10B7580001025A6031462046FFF76DF9234632460A
:10B76800FF2108E0A003002000ED00E05869816097
:10B77800186D01328160607804338242F6D3236900
:10B7880001274FF0FF3267F30F069A6167F31F46F0
:10B798000F22DE615A612F221A611A686FF30A12AA
:10B7A8001A602046FFF7FAFBE3684FF480525A61AB
:10B7B800264B1B6820461B6998473846C5F3072364
:10B7C80003F02003DBB2EBB12046FFF74FFAE36842
:10B7D8002046DE68FFF73CFA032806D10023A37051
:10B7E8004FF40073A380092304E00123A3704023CE
:10B7F800A380052363F38D26E3684FF40052DE60CF
:10B8080001205A61C5F3074303F01003DBB24BB1C3
:10B818000E4B1B682046DB699847E3684FF480129B
:10B828005A610120C5F3074505F02005EDB255B171
:10B83800064B1B6820461B6A9847E3684FF40012C2
:10B848005A610120FFE7BDE8FE8F00BFA00300207A
:10B8580043230B80004870471003002038B51F4B66
:10B868001A68511C052A196035D119790022012955
:10B878001A6030D09968B1F5006F08BF9A60174B0D
:10B888009968DC68A1421A4602D100221A7122E0A6
:10B8980086BFC1F500631361C1EB0404D0F8EC3531
:10B8A80098BF14611569B3F839300C4C9D428AB2BF
:10B8B80004D95918ED1AA160256104E06918A1603E
:10B8C8000021ABB22161054901240C7104498A1891
:10B8D8008121FFF7D4FC002038BD00BFB80E00203E
:10B8E8003749002038B528230A4D03FB01010A4BCC
:10B8F800B1F888131B69044628469847D4F8EC35F4
:10B908002046B3F8403001212A46FFF79DFC00206D
:10B9180038BD00BFEF4800208C03002070B50B78BD
:10B9280013F0600506460C4625D0202D1FD1CD8882
:10B93800B5B113F0800F487808D0214B21499B6896
:10B948002A469847E2881F49304625E01E4B1D4984
:10B9580058641E4B30465D612A4600F022FB1DE00C
:10B96800174B48789B6829462A46984725E000F0F7
:10B9780077FB022521E04B780A2B11D00B2B14D032
:10B98800062B1AD14B881B0A212B03D1CA883A2AC5
:10B9980028BF3A220E49304600F0EAFA00250CE0AA
:10B9A8000C49012200F0E4FA07E08B781BB9074A3A
:10B9B8001D46936101E000F053FB284670BD00BFAF
:10B9C8008C0300202F49002010030020B80E00200F
:10B9D80022030020D00E002010B581210446FFF775
:10B9E8001AFC01212046FFF716FC82212046FFF7AA
:10B9F80012FC024B5B689847002010BD8C030020A6
:10BA080038B5D0F8EC350446B3F839208121022343
:10BA1800FFF7E0FBD4F8EC350121B3F840202046CD
:10BA28000223FFF7D7FB8221082203232046FFF7D2
:10BA3800D1FB094B022200251A715D71074B1B6867
:10BA48009847D4F8EC35064AB3F84030204601212F
:10BA5800FFF7FAFB284638BDD00300208C030020EE
:10BA6800EF48002010B5074C606CFF2807D0064B44
:10BA7800064A9B68064952699847FF236364002079
:10BA880010BD00BF100300208C030020B80E00205A
:10BA98002F49002038B510490B79012B19D10C69B1
:10BAA8000CB90C7115E0D0F8EC358D68B3F8393065
:10BAB8009C42AAB203D95D198D60E41A03E0A3B2CF
:10BAC8002C198C6000240C61044952188121FFF75D
:10BAD800D6FB002038BD00BFB80E00203749002033
:10BAE80000207047002070470023F0B5084A094E2F
:10BAF8001D4609E01468C75C375501340133B4F5B5
:10BB0800006F146008BF15608B42F3D10020F0BDB0
:10BB1800C40E002037490020104B114AD3F800C04A
:10BB280000232DE9F0410F4F16461D460DE014681D
:10BB380010F8038007F804800134802C08BF2C46D5
:10BB480014603468644505D001338B42EFD100207E
:10BB5800BDE8F0810220BDE8F08100BFB8510020A7
:10BB6800CC5100203851002021280FD1084B1A68E9
:10BB78000A701A68120A4A705A888A70DA78CA7083
:10BB88001A790A715A794A719B798B71002070472A
:10BB98008403002007B502AB012103F8010D184604
:10BBA800FFF7A2FF0EBD002100E00131435C002B2E
:10BBB800FBD199E798E70B4B0B491A680968914242
:10BBC8000BD00A498A5C02701A680132802A1A600E
:10BBD80005D100221A60012070470020704701201B
:10BBE800704700BFB8510020CC51002038510020C8
:10BBF800204B1A68204B1B689A42F0B509D135E0F2
:10BC08000133802B08BF00239A4203D11A4B1A60D4
:10BC18002CE01A4CE15C0029F2D00A29F0D00D2959
:10BC2800EED0154C1549134D23600E460023CF184E
:10BC38002268BA5CC254226801339F18802F08BF5B
:10BC480053422F689A18974210D0B25C1AB10A2A48
:10BC580001D00D2AEBD10022C254074A11685918A5
:10BC68007F29116003D98039116000E0002318464C
:10BC7800F0BD00BFCC510020B85100203851002041
:10BC8800704700BFD0F8E43510B51B6904469847E3
:10BC9800032384F81231002010BD08B5042380F86E
:10BCA8001231D0F8E435DB689847002008BD08B5A4
:10BCB800D0F8E035DB6903B19847002008BD08B526
:10BCC800D0F8E0351B6A9847002008BD08B5D0F8C1
:10BCD800E0355B6A9847002008BD002110B5402276
:10BCE80004460B46FFF776FA8021402200232046BF
:10BCF800FFF770FA012384F81231D4F8E435A078FC
:10BD08005B689847002010BD13B56946044600F0EB
:10BD180085F99DF8001001F01F03012B07D0022BB5
:10BD28000AD073B92046694600F026FA0FE020468B
:10BD3800694600F007FA0AE02046694600F0A2F9D1
:10BD480005E021F07F01C9B22046FFF7B1FA0020D3
:10BD58001CBD38B5044600293DD190F81131022B9D
:10BD680042D1D0F83421D0F820319A4211D9C17883
:10BD7800D21A0129C0F8342104D1D0F82411CB18E3
:10BD8800C0F8243192B22046D4F8241100F000F90A
:10BD98002AE0D0F83821B2FBF3F503FB152565B985
:10BDA8009A420AD3D0F83C319A4206D229462A460A
:10BDB80000F0EEF8C4F83C5116E0D4F8E035DB6842
:10BDC8002BB194F81221032A01D120469847204626
:10BDD80000F00FF908E0D0F8E0355B6923B190F87E
:10BDE8001221032A00D19847002038BD10B5044617
:10BDF80059BB90F81131032B30D1D0F88C23D0F8EF
:10BE080078339A4214D9C178D21A0129C0F88C2300
:10BE180004D1D0F87C13C918C0F87C139A4228BF03
:10BE28001A4692B22046D4F87C1300F0CAF815E0FE
:10BE3800D0F8E0351B6923B190F81221032A00D10C
:10BE48009847204600F0C6F808E0D0F8E0359B692E
:10BE580023B190F81221032A00D19847002010BD81
:10BE68002DE9F041069F0446164698460D46FEF712
:10BE780041FC20462946C4F8E085C4F8E475C4F8B6
:10BE8800E865FFF761F9D4F8E4351B689847204660
:10BE9800BDE8F041FEF782BC00207047D0F8E035DD
:10BEA80010B504461B689847D4F8E4359B68984752
:10BEB800002010BD08B5D0F8E0355B689847002031
:10BEC80008BD000012230B8000487047D0030020F3
:10BED80004230B8000487047E203002010B5044C8F
:10BEE80004480A46214600F075FA204610BD00BFF6
:10BEF800D05100205DA605080A4608B50248034946
:10BF080000F068FA014808BD70A60508D051002065
:10BF18000A4608B50248034900F05CFA014808BD22
:10BF28007EA60508D051002008B50A4608B904487D
:10BF380000E00448044900F04DFA034808BD00BF7A
:10BF480089A6050896A60508D051002008B50A4616
:10BF580008B9044800E00448044900F03BFA0348E3
:10BF680008BD00BFA3A60508C4A60508D051002037
:10BF780010B513460C46C0F83821C0F83421022207
:10BF880080F8112100212246FFF779F9002010BD21
:10BF980010B50C46134600212246FFF770F9002021
:10BFA80010BD10B513460C46C0F89023C0F88C237A
:10BFB800032280F8112100212246FFF745F90020CD
:10BFC80010BD10B50C46134600212246FFF73CF978
:10BFD800002010BD0021042310B50A46044680F84D
:10BFE80011310B46FFF74BF92046FEF7D7FF00202B
:10BFF80010BD0021052310B50A46044680F811310A
:10C008000B46FFF721F92046FEF7C8FF002010BDB8
:10C01800282303FB0100B0F88803704790F8C8355F
:10C028000B7090F8C9354B7090F8CB2590F8CA354D
:10C0380003EB02234B8090F8CD2590F8CC3503EB29
:10C0480002238B8090F8CF2590F8CE3503EB02239E
:10C058009BB2CB80C0F83C31012380F81131704786
:10C0680010B591F90030002B044601DBCB880BB9E1
:10C07800802100E00021FFF71BF92046BDE81040B1
:10C08800FEF78CBF38B50D4604466B780979012B4D
:10C0980010D027D3032B51D190F81231022B28D07E
:10C0A800032B47D16B889BB991B1802910D0FFF73A
:10C0B800FFF80DE090F81231022B1AD0032B39D17A
:10C0C8006B88002B3AD149B1802907D0FFF70EF9C8
:10C0D800D4F8E03520469B68294698472046FFF764
:10C0E80079FF2BE090F81231022B02D0032B21D1DB
:10C0F80006E019B3802921D02046FFF7D9F81DE0C2
:10C1080011F0800F4FF0280306D001F07F0103FBE8
:10C11800010393F81A2103E003FB010191F872234C
:10C12800074B02B101221A60204605490222FFF797
:10C138001FFF03E020462946FFF792FF002038BD85
:10C14800D40E002038B590F81231032B04460D4662
:10C158000CD10B79012B09D8D0F8E0359B689847AA
:10C16800EB883BB92046FFF735FF03E02046294618
:10C17800FFF776FF002038BD73B54B7804460D46AF
:10C18800092B00F21C81DFE813F0D10008011A0125
:10C19800E4001A0172000A001A01C00092004B88DC
:10C1A8001A0A013A062A00F20A81DFE812F00700AB
:10C1B8001A0027000801080108010801D4F8E83529
:10C1C800A0781B680DF106019847EB88402B0146C3
:10C1D80003D094F81231012B3AD10823ADF8063078
:10C1E80036E0D4F8E035A0789B6A0DF1060198474F
:10C1F800022343700146C4F8EC0529E0DBB2052BA5
:10C2080000F2DD80DFE803F003080D12171CD4F8F4
:10C21800E835A0785B6817E0D4F8E835A0789B6823
:10C2280012E0D4F8E835A078DB680DE0D4F8E835FA
:10C23800A0781B6908E0D4F8E835A0785B6903E0CA
:10C24800D4F8E835A0789B690DF1060198470146B6
:10C25800BDF80630002B00F0B680EA88002A00F00E
:10C26800B2809A4228BF1A46ADF806205CE08B8857
:10C27800002B40F0A480CB88002B40F0A08094F8DD
:10C2880012214B88032A00F09A8003F07F0520468C
:10C2980084F813512946FFF753F82046FFF79AFE12
:10C2A8000DB1022300E0012384F812318BE0897874
:10C2B800464E0129317100F2828094F81231022B26
:10C2C80002D0032B7BD108E0002962D0012103238F
:10C2D80084F8101184F8123113E041B9022384F86C
:10C2E800123184F810112046FFF7E4FD51E094F86C
:10C2F8001011012920464DD0FFF7DCFD317984F873
:10C3080010112046FFF7CAFD43E0CA88012A56D11A
:10C3180094F81231022B02D0032B50D102E02046B0
:10C328002B4913E004F5887120460FE094F8123188
:10C33800023B012B43D8D4F814312449002B0CBFFD
:10C348000123032341F80C3F20460122FFF710FE8A
:10C3580039E04B88012B29D0022B34D18B8813F07C
:10C36800FF0F30D121691B0A013B4A68042B0FD803
:10C37800DFE803F0030507090B00012306E00223A9
:10C3880004E0032302E0042300E0052363F306121C
:10C398004A602046FFF71EFE15E094F81231023B72
:10C3A800012B0CD84B88012B0DD10023C4F8143174
:10C3B800D4F8E03520469B6829469847E9E72046A7
:10C3C8002946FFF74DFE00207CBD00BFD40E00209B
:10C3D800DC0E002030B5C8B10023DDB20133C4182B
:10C3E80014F8014C002CF8D16B1C5B0013800B7007
:10C3F80003234B70022305E0CA545A1CD2B20233FD
:10C408008C54DBB210F8012B002AF5D130BD00BFE7
:10C418007047704770477047704770477047000013
:10C428000EB403B070470A2810B5044602D10D2097
:10C43800FFF7F9FF064A13681BB103F8014B1360B5
:10C4480010BD044B1B680BB12046984710BD00BFB8
:10C45800E40E00200452002010B5044601E0FFF766
:10C46800E2FF14F8010B0028F9D110BD2DE9F04FB7
:10C47800044685B00D464FF00A0A00E0354620789C
:10C48800002800F0C480252801D0013467E06078D6
:10C49800302803D1A0780123033407E02D2802D0E7
:10C4A8000234002302E0A078022303344FF000088E
:10C4B80005E00AFB080814F8010BA8F13008A0F100
:10C4C8003002D2B2092AF4D96C2801D04C2803D101
:10C4D80014F8010B43F00403002800F0988060284A
:10C4E80086BFA0F12002D2B202464F2A3DD006D81C
:10C4F800432A2DD0442A09D0422A30D133E0552A84
:10C5080004D0582A29D0532A29D101E00A272DE03E
:10C518002E1D2F68002500E001357A5D002AFBD129
:10C5280004E02020FFF77FFF4D4601E0980704D480
:10C53800454505F10109F4D34D463846FFF78CFF10
:10C5480003E02020FFF76FFF01354545F9D395E754
:10C5580028782E1DFFF767FF90E7102706E0FFF702
:10C5680062FF2E468AE7022700E008272E1D442A8C
:10C57800296804D1002902DA494243F0080300225D
:10C5880000E02A46B1FBF7FE07FB1E11CDB2092DCC
:10C59800714607D9782814BF4FF0070C4FF0270CC5
:10C5A8006544EDB230350DF80250551CBEF1000F50
:10C5B80002D0102DE5D10F22190705D504A94D1970
:10C5C8002D2105F8101C951C13F0010F0CBF4FF01E
:10C5D800200B4FF0300B9B072F4604D508E0584638
:10C5E800FFF721FF4F46474507F10109F7D34F46AB
:10C5F800013D1DF80500FFF716FF002DF8D103E0F7
:10C608002020FFF710FF01374745F9D336E705B07B
:10C61800BDE8F08F70B5064D0C462E68286001E025
:10C62800FFF701FF14F8010B0028F9D12E6070BD47
:10C63800045200200FB407B504A951F8040B019166
:10C64800FFF714FFBDE80E4004B070470EB417B5ED
:10C6580005A9084C51F8043B206018460191FFF7E2
:10C6680005FF2268002313702360BDE81E4003B055
:10C67800704700BFE40E00200EB433B505A9074C7F
:10C6880051F8043B2568206018460191FFF7EEFE3B
:10C698002560BDE83C4003B0704700BF045200204D
:10C6A80070B51E4604461C481546FFF7C3FF022E08
:10C6B8001FD0042E25D0012E2AD105E0A15D1748F0
:10C6C800FFF7B8FF013600E00026AE42F6DB202077
:10C6D800FFF7A9FE002609E0A05DA0F12003DBB268
:10C6E8005E2B88BF2E20FFF79EFE0136AE42F3DB9D
:10C6F8000EE034F8021B0A48FFF79CFF013DF8D111
:10C7080006E054F8041B0748FFF794FF013DF8D1F1
:10C718000A20BDE8704086E6E5A60508ECA60508EF
:10C72800F2A60508F8A6050808B501214FF480709F
:10C7380001F07CFA4FF480700021BDE8084001F058
:10C7480075BA43680A6823F0407323F4807313436F
:10C758000A7943EA02234360CA680B6930B51A4371
:10C7680084688D68084B2A43234013434A7943EA77
:10C77800420383600B7DC26A013B22F47002DBB284
:10C7880042EA0353C36230BDFDF7FFC000230360D4
:10C79800037143718360C3600361012303757047AC
:10C7A800074A084B516810B50B4090E81200214326
:10C7B8008468C068214301430B43536010BD00BF28
:10C7C80000230140E030FCFF0023036043608360E6
:10C7D800C3607047836811B143F0010301E023F09F
:10C7E800010383607047436823F4400323F4007314
:10C7F8000B4343607047416282627047436823F08D
:10C808001F030B4343607047044B5A6810B142F44E
:10C81800000201E022F400025A6070470023014040
:10C82800044B5A6810B142F4800201E022F48002FD
:10C838005A60704700230140092970B50CB20CD921
:10C8480004EB44041E3CC6680725A54026EA0505F6
:10C85800A34045EA0304C4600AE0066904EB440403
:10C868000725A54026EA050513FA04F42C430461BC
:10C87800062A0CD80523013A5A43446B1F239340D8
:10C8880024EA0303914043EA0102426370BD0C2A83
:10C8980012B20CD802EB8202233A046B1F23934096
:10C8A80024EA0303914043EA0102026370BD02EBEC
:10C8B8008202413AC46A1F23934024EA0303914049
:10C8C80043EA0102C26270BD836843F0804383601B
:10C8D80070478068C0F380507047836811B143F493
:10C8E800806301E023F4806383607047836811B13B
:10C8F80043F0020301E023F00203836070474368BA
:10C90800013923F4604343EA413343607047436885
:10C9180011B143F4006301E023F4006343607047FE
:10C92800C06C80B27047014B1868704708230140FB
:10C93800836811B143F4807301E023F4807383604A
:10C948007047836811B143F4007301E023F4007366
:10C9580083607047044B5A6810B142F4005201E0FA
:10C9680022F400525A60704700230140092970B52B
:10C978000CB20CD904EB44041E3CC6680725A5403C
:10C9880026EA0505A34045EA0304C4600AE00669EF
:10C9980004EB44040725A54026EA050513FA04F428
:10C9A8002C430461836BC3F30154121B0232D2B2CD
:10C9B80002EB82021F24944023EA040391400B43B4
:10C9C800836370BD836B013923F4401343EA015339
:10C9D8008363704782B0002301930190019BCB18B9
:10C9E8000193019B1A6002B07047836823F4702397
:10C9F8000B4383607047836823F440130B438360C1
:10CA08007047836843F48003836070478068C0F38D
:10CA180080507047436811B143F4806301E023F408
:10CA2800806343607047436811B143F4805301E069
:10CA380023F480534360704782B000230193019030
:10CA4800019B28335B180193019B186880B202B0E0
:10CA580070470123C9B213FA01F143680AB11943B7
:10CA680001E023EA010141607047036819420CBFE5
:10CA7800002001207047C94301607047436800687F
:10CA880010EA112007D00122C9B212FA01F11942A5
:10CA98000CBF0020012070476FEA11210160704728
:10CAA800036823F00103036000230360436083608D
:10CAB800C3600361212343612C4B98421CD02C4B4B
:10CAC800984220D02B4B984225D02B4B98422AD005
:10CAD8002A4B98422FD02A4B984233D0294B984260
:10CAE80037D0294B984204D14FF03D5243F8AC2C33
:10CAF8007047264B984203D13D2243F8082C7047D3
:10CB0800234B984204D14FF4746243F8202C7047A9
:10CB1800204B984204D14FF4741243F8382C7047D4
:10CB28001D4B984204D14FF0746243F8502C704763
:10CB38001A4B984203D11A4A43F8642C7047194B90
:10CB4800984203D1184A43F87C2C7047174B9842F7
:10CB580003D1174A43F8942C7047164B984204BFE8
:10CB68004FF03D5243F8AC2C704700BF10600240B4
:10CB780028600240406002405860024070600240F5
:10CB880088600240A0600240B86002401064024021
:10CB980028640240406402405864024070640240C5
:10CBA8003D00002088640240400F0020A06402403D
:10CBB80000003D20B86402400268134B10B51340D2
:10CBC800CC680A6822434C6922438C692243CC69A9
:10CBD80022430C6A22434C6A22438C6A22434C6BE0
:10CBE80022438C6B22431343036042690C6BCB6A6C
:10CBF80022F007022343134343610B6943604B68E8
:10CC080083608B68C36010BD3F801CF00023036005
:10CC180043608360C360036143618361C3610362EE
:10CC280043628362C3620363436383637047036839
:10CC380011B143F0010301E023F0010303607047E1
:10CC4800036811B143F4004301E023F40043036097
:10CC58007047036811B143F0200301E023F020037B
:10CC68000360704741607047406880B2704703684E
:10CC780012B143F4002301E023F4002303600161AF
:10CC88007047036811B143F4802301E023F4802343
:10CC9800036070470AB101617047C160704700685E
:10CCA800C0F3C0407047006800F001007047406959
:10CCB80000F0380070470A4A0A4B10B50A4CA042E7
:10CCC80088BF13468A004CBF5B681B6821F0F021BF
:10CCD80021F0821119420CBF0020012010BD00BFB5
:10CCE80000640240006002400F64024010B5084B27
:10CCF800084A094CA04288BF134611F0005F21F092
:10CD0800F02121F0821114BFD960996010BD00BFD5
:10CD180000600240006402400F6402400B0607D521
:10CD2800436912B143F0800301E023F080034361BB
:10CD3800802909D001F01E01036812B1194301606E
:10CD4800704723EA010101607047124B124A10B57F
:10CD5800124CA0428CBF14461C4621F0F02323F04D
:10CD6800C3132BB1026802F01E0202EAD12202E0CC
:10CD7800426902F0800288004CBF6368236821F092
:10CD8800F02121F08210184002D0101C18BF012099
:10CD980010BD00BF00600240006402400F64024002
:10CDA80010B5084B084A094CA04288BF134611F039
:10CDB800005F21F0F02121F0821114BFD960996041
:10CDC80010BD00BF00600240006402400F640240D2
:10CDD800044B00221A605A609A60DA60024A5A616B
:10CDE800704700BF003C0140FFFF7F00837910B50A
:10CDF800002B29D01A4B01681C68CA4314401C60D8
:10CE08005C6822405A60027902F1804202F59E3243
:10CE180014682143116002689C68D1430C409C60EF
:10CE2800DC682140D9604179102906D199681143FD
:10CE38009960D9680A43DA6010BD01F1804303F5AF
:10CE48009E3319680A4308E00379016803F18043B7
:10CE580003F59E331A6822EA01021A6010BD00BF6A
:10CE6800003C014000230C2203600371427183716E
:10CE78007047024B1A6902431A617047003C01402F
:10CE8800034B5B6918420CBF00200120704700BFAC
:10CE9800003C0140014B5861704700BF003C014015
:10CEA800054B1A685B69034004D010420CBF002090
:10CEB8000120704718467047003C0140014B5861FB
:10CEC800704700BF003C01404FF0204318B943F2BF
:10CED800DB021A6003E043F2D20243F820204FF04D
:10CEE8002042411C6FF0704342F8213002F58272F3
:10CEF80042F82030704770B584684568C368C16AD5
:10CF0800026825431D4303691D4343691D43836923
:10CF18001D43C3691D43036A1D43436A1D43836A56
:10CF28001D43036B0D431D434FF02043082C43F86A
:10CF3800225005D153F8224044F0400443F82240DF
:10CF4800436B9E691D6835435E6845EA06159E6811
:10CF580045EA0625DE6845EA06451E695B6945EA35
:10CF68000655541C45EA03654FF02043B1F5804F40
:10CF780043F8245010D1836B9869196801435868A5
:10CF880041EA0011986841EA002118695B6941EAA1
:10CF9800005141EA036101E06FF07041014B43F831
:10CFA800221070BD040100A0022242604FF480529A
:10CFB8004262416B4FF4005210B5826200230F2287
:10CFC800FF2403608360C360036143618361C361BD
:10CFD8000362C36203630A604A608C60CA600A61C4
:10CFE8004A618B61816B0A604A608C60CA600A6121
:10CFF8004A618B6110BD4FF0204321B153F82020C6
:10D0080042F0010203E053F82010024A0A4043F8B4
:10D0180020207047FEFF0F0010280CBF064B074B5F
:10D028004FF040024FF0180119605A604FF0FC327F
:10D038009A60DA60704700BF600000A0800000A01E
:10D0480030B5836844681C43C36844F008041C4333
:10D0580003691C43436944EA4324836944EA43342B
:10D06800C36999685A68090441EA02211A68DB68A9
:10D07800114341EA0361036A9A685D68120442EA4F
:10D0880005221D68DB682A4342EA03620368102B05
:10D098000CBF034B034B1C609960DA6030BD00BFC6
:10D0A800600000A0800000A010230360C269002374
:10D0B80043608360C360036143618361FC23136041
:10D0C80053609360D360026A136053609360D360C7
:10D0D800704741B110280CBF074B084B1A6842F043
:10D0E80004021A60704710280CBF034A034A044B15
:10D0F80011680B4013607047600000A0800000A01A
:10D10800FBFF0F0041B110280CBF084B084B1A68F1
:10D1180042F040021A60704710280CBF034A044AC4
:10D12800044B11680B401360704700BF600000A0FB
:10D13800800000A0BFFF0F00102802D1024B5869E1
:10D148007047024B58697047600000A0800000A03B
:10D15800054B18221A6000225A604FF0FC329A6080
:10D16800DA601A61704700BFA00000A00268436837
:10D1780042F0100242EA4322836842EA4332144BE7
:10D1880010B51A60C26891685468090441EA04211C
:10D198001468D268214341EA02629A600269916880
:10D1A8005468090441EA04211468D268214341EA19
:10D1B8000262DA60426991685068090441EA002114
:10D1C8001068D268014341EA02621A6110BD00BFCB
:10D1D800A00000A0C2680023036043608360FC23B2
:10D1E800136053609360D360026913605360936067
:10D1F800D3604269136053609360D3607047054BF6
:10D2080018B11A6842F0040202E01968024A0A409A
:10D218001A607047A00000A0FBFF0F0062B1102841
:10D2280001D10E4B03E0B0F5807F03D10C4B5A6857
:10D23800114311E00B4BFAE7102804D1074B5A6849
:10D2480022EA010108E0B0F5807F0CBF044B054BD2
:10D258005A686FEA0101114059607047600000A0E8
:10D26800800000A0A00000A0102801D1064B04E017
:10D27800B0F5807F0CBF054B054B5B680B420CBFBC
:10D2880000200120704700BF600000A0800000A0BF
:10D29800A00000A0102804D1074B5A6822EA010117
:10D2A80008E0B0F5807F0CBF044B054B5A686FEA65
:10D2B8000101114059607047600000A0800000A083
:10D2C800A00000A0102801D1084B04E0B0F5807F31
:10D2D8000CBF074B074B5B6813EA010004D013EA45
:10D2E800D1010CBF00200120704700BF600000A0E2
:10D2F800800000A0A00000A0102804D1084B5A68A4
:10D3080022EAD10109E0B0F5807F0CBF054B064B3E
:10D318005A684FEAD10122EA01015960704700BFFB
:10D32800600000A0800000A0A00000A008B52C4B61
:10D33800984205D10120014600F048FC012048E050
:10D34800284B984205D10220012100F03FFC022021
:10D358003FE0254B984205D10420012100F036FC1E
:10D36800042036E0214B984205D10820012100F025
:10D378002DFC08202DE01E4B984205D110200121DC
:10D3880000F024FC102024E01A4B984205D12020FC
:10D39800012100F01BFC20201BE0174B984205D10F
:10D3A8004020012100F012FC402012E0134B98426B
:10D3B80005D18020012100F009FC802009E0104BF4
:10D3C80098420BD14FF48070012100F0FFFB4FF41D
:10D3D80080700021BDE8084000F0F8BB08BD00BF20
:10D3E800000002400004024000080240000C024015
:10D3F800001002400014024000180240001C0240C5
:10D40800002002402DE9F0470023D1F800801A4699
:10D418004FF0010C03270CFA02F404EA0805A542B0
:10D428002ED1066817FA03F4E443264006600E7905
:10D43800D0F8009006FA03FA013E4AEA0909012EDB
:10D44800C0F8009014D8866891F805902640866048
:10D45800866809FA03F949EA06068660466826EAF4
:10D46800050545608D7946689540ADB23543456000
:10D47800C5682C40C460CC79C5689C402C43C46006
:10D4880001320233102AC6D1BDE8F0874FF6FF7388
:10D4980003600023037143718371C371704782B0C5
:10D4A8004FF480330193019B0B430193019BC361AC
:10D4B800C161019BC361C3690193C369019302B050
:10D4C8007047036919420CBF0020012070470069AA
:10D4D80080B27047436919420CBF00200120704791
:10D4E800406980B2704701837047418370470AB131
:10D4F80001837047418370474161704743694B40DE
:10D508004361704701F00703C908083130B59B0033
:10D5180050F821500F249C4025EA040440F821408B
:10D5280050F8214012FA03F31C4340F8214030BD63
:10D5380008B5134B984207D14FF40010012100F0B1
:10D5480069FB4FF4001014E00E4B984207D14FF4DA
:10D558008000012100F05EFB4FF4800009E00A4BD7
:10D5680098420BD14FF40000012100F053FB4FF417
:10D5780000000021BDE8084000F04CBB08BD00BF1A
:10D588000054004000580040005C00407FB504464D
:10D59800868868460D4600F06DFA02992C482B687B
:10D5A80026F03F063604B1FBF0F0360C80B2064395
:10D5B800A680228822F001021204120C2280254A39
:10D5C80093420AD85B00B1FBF3F301309BB280B2FF
:10D5D8002084032B98BF042321E0EE884BF6FF72CA
:10D5E800964205D103225343B1FBF3F39BB206E005
:10D5F80019225343B1FBF3F39BB243F480431A055A
:10D608004FF4967208BF43F0010350434FF47A7207
:10D6180090FBF2F0013080B243F400432084A383EE
:10D6280023886989AA889BB243F001032380238851
:10D6380023F4816323F002031B040A431B0C1343E6
:10D648009BB223802A89AB8913439BB223817FBD78
:10D6580040420F00A086010041F288330360002396
:10D6680083804BF6FF72038143814FF48043C2806D
:10D6780083817047038819B19BB243F0010303E02B
:10D6880023F001031B041B0C03807047038819B1A6
:10D698009BB243F4807303E023F480731B041B0CD8
:10D6A80003807047038819B19BB243F4007303E009
:10D6B80023F400731B041B0C0380704712B141F064
:10D6C800010101E001F0FE0101827047038819B1F0
:10D6D8009BB243F4806303E023F480631B041B0CB8
:10D6E8000380704783899BB201F0FE0123F0FE039B
:10D6F8000B4383817047838919B19BB243F00103BF
:10D7080003E023F001031B041B0C8381704703888B
:10D7180019B19BB243F0400303E023F040031B041C
:10D728001B0C03807047038829B16FEA43436FEAF3
:10D7380053439BB201E05B045B0C03807047038892
:10D7480019B99BB243F0800303E023F080031B0464
:10D758001B0C03807047B1F5804F838B04D023F4F2
:10D7680080431B041B0C02E09BB243F48043838379
:10D778007047B1F5006F038803D19BB243F400638F
:10D7880003E023F400631B041B0C03807047B1F50E
:10D79800005F038803D19BB243F4005303E023F4F2
:10D7A80000531B041B0C03807047038819B19BB2FC
:10D7B80043F0100303E023F010031B041B0C038049
:10D7C800704701827047008AC0B27047038819B158
:10D7D8009BB243F4805303E023F480531B041B0CD7
:10D7E80003807047B1F5006F038803D19BB243F4FF
:10D7F800006303E023F400631B041B0C03807047E1
:10D80800038819B19BB243F0200303E023F02003FF
:10D818001B041B0C03807047008BC0F30720704764
:10D82800838819B19BB243F4006303E023F40063D7
:10D838001B041B0C83807047838819B19BB243F487
:10D84800805303E023F480531B041B0C8380704730
:10D8580082B0002301930190019BCB180193019B97
:10D86800188880B202B0704783889BB20AB1194306
:10D8780001E023EA010181807047838A008B9BB213
:10D8880043EA0040084020F07F40431A584240EBEA
:10D8980003007047838A008B9BB243EA004020F064
:10D8A8007F40704782B00023009301930B0F0190D3
:10D8B8000093009B21F07F4113B1019B143302E0D8
:10D8C800019B090C18330193019B1B6819420CBF7B
:10D8D8000020012002B07047C94389B28182704795
:10D8E8008388808A80B208409BB206D001F0E0614C
:10D8F80013EA11410CBF002001207047C94389B2C7
:10D90800818270470A4B1A6842F001021A600022AD
:10D918009A60196821F0847121F4803119600549F1
:10D928005960196821F480211960DA60704700BFD6
:10D938000038024010300024024B00221A70187080
:10D94800704700BF02380240034B1A6822F0F80201
:10D9580042EAC0021A60704700380240014B186062
:10D96800704700BF00004742064B002201281A708A
:10D978001A7002D0042804D101E0187070470522FB
:10D988001A70704770380240014B1860704700BF2A
:10D99800800E4742014341EA821200995B08013B2D
:10D9A80042EA016141EA0341014B5960704700BFF7
:10D9B80000380240014B1860704700BF60004742C2
:10D9C8008001034B40EA0171C3F88410704700BF1F
:10D9D80000380240014B1860704700BF680047429A
:10D9E800014B1860704700BF4C004742034B9A68D0
:10D9F80022F0EC6202430A439A6070470038024002
:10DA0800034B9A6822F0784202430A439A607047AF
:10DA180000380240034B9A6822F0030202439A60DE
:10DA2800704700BF00380240024B986800F00C00B5
:10DA3800704700BF00380240034B9A6822F0F0029A
:10DA480002439A60704700BF00380240034B9A684F
:10DA580022F4E05202439A60704700BF0038024047
:10DA6800034B9A6822F4604242EAC0029A60704707
:10DA7800003802401E4B9A6802F00C02042A10B5C6
:10DA880003D0082A03D01B4B18E01B4B16E059683B
:10DA98005A6811F4800F596814BF174B154B02F0E0
:10DAA8003F02B3FBF2F3124A5268C2F30142C1F3D8
:10DAB800881101324B435200B3FBF2F30C49036067
:10DAC8008B680E4A0468C3F30313D35C34FA03F378
:10DAD80043608C68C4F38224145D33FA04F48460D0
:10DAE8008968C1F34231525CD340C36010BD00BFA6
:10DAF800003802400024F40000127A0028040020B4
:10DB080000F44073B3F5407F084B08D1996820F0C2
:10DB1800704221F4F81122F440720A439A601A6F95
:10DB2800000542EA10501867704700BF00380240ED
:10DB3800014B1860704700BF3C0E4742014B18600C
:10DB4800704700BF400E4742014B1860704700BF46
:10DB58005C014742044B1A6B09B1104301E022EA09
:10DB680000001863704700BF00380240044B5A6B2E
:10DB780009B1104301E022EA00005863704700BF72
:10DB880000380240044B9A6B09B1104301E022EAC5
:10DB980000009863704700BF00380240044B1A6CBD
:10DBA80009B1104301E022EA00001864704700BF81
:10DBB80000380240044B5A6C09B1104301E022EAD4
:10DBC80000005864704700BF00380240044B1A69CF
:10DBD80009B1104301E022EA00001861704700BF54
:10DBE80000380240044B5A6909B1104301E022EAA7
:10DBF80000005861704700BF00380240044B9A6922
:10DC080009B1104301E022EA00009861704700BFA3
:10DC180000380240044B1A6A09B1104301E022EAB5
:10DC280000001862704700BF00380240044B5A6A6F
:10DC380009B1104301E022EA00005862704700BFB2
:10DC480000380240044B1A6D09B1104301E022EA82
:10DC580000001865704700BF00380240044B5A6D39
:10DC680009B1104301E022EA00005865704700BF7F
:10DC780000380240044B9A6D09B1104301E022EAD2
:10DC880000009865704700BF00380240044B1A6EC8
:10DC980009B1104301E022EA00001866704700BF8E
:10DCA80000380240044B5A6E09B1104301E022EAE1
:10DCB80000005866704700BF00380240044B1A78CD
:10DCC80009B1104301E022EA00001870704700BF54
:10DCD8000D3802404309012B074A01D1136803E0BC
:10DCE800022B0CBF136F536F00F01F0033FA00F0C4
:10DCF80000F00100704700BF0038024007B500235C
:10DD080001933120FFF7E6FF019B01330193019B4B
:10DD1800B3F5A06F01D00028F3D03120FFF7DAFF68
:10DD2800003018BF01200EBD024B5A6F42F08072BE
:10DD38005A67704700380240034BDB6818420CBF33
:10DD480000200120704700BF00380240014B1870C6
:10DD5800704700BF0E38024008B5154B98420BD1EA
:10DD680001214FF48050FFF761FF4FF480500021EC
:10DD7800BDE80840FFF75ABF0E4B984207D14FF451
:10DD880080400121FFF746FF4FF4804009E00A4B2D
:10DD980098420BD14FF400400121FFF73BFF4FF4AD
:10DDA80000400021BDE80840FFF734BF08BD00BFB0
:10DDB8000030014000380040003C00400B880288D9
:10DDC80010B54C8823438C882343CC8823430C8983
:10DDD80023434C8923438C892343CC8902F4415241
:10DDE800234313439BB20380838B23F400631B04F8
:10DDF8001B0C83830B8A038210BD838B23F47B6304
:10DE080023F00F031B041B0C8383022303848B68FA
:10DE1800F0B5858B022BADB238D0294A8E8894682C
:10DE2800002E14BF02260126240203D5946824F488
:10DE380000049460D2F88440D2F884705268DFF805
:10DE480084C002F03F02BCFBF2F2C4F388145443CE
:10DE5800C7F30272B4FBF2F4CA88B2F5007F4FF040
:10DE68000A0201D1240A02E07601B4FBF6F4624307
:10DE7800B2FBF3F305330A229BB2B3FBF2F303F0D0
:10DE880001021202C3F34F0392B200E000229C1E6B
:10DE9800A4B2FE2C28BF0022CC8828BF022313433B
:10DEA80023439BB203840B884A882B4343F40063C3
:10DEB80013438A8813438A8913439BB28383F0BD33
:10DEC8000038024000127A000023038043808380D8
:10DED800C380038143818381C38107230382704701
:10DEE80000230222038043808380C3808260838171
:10DEF8007047038819B19BB243F0400303E023F055
:10DF080040031B041B0C03807047838B19B19BB221
:10DF180043F4806303E023F480631B041B0C8383B6
:10DF28007047038823F400631B041B0C03800388D9
:10DF38009BB20B4303807047B1F5804F038803D130
:10DF48009BB243F4804303E023F480431B041B0C7F
:10DF5800038070474FF6FF639942038803D09BB252
:10DF680043F4807303E023F480731B041B0C0380C9
:10DF78007047838819B19BB243F0040303E023F090
:10DF880004031B041B0C83807047838819B19BB260
:10DF980043F0100303E023F010031B041B0C8380E1
:10DFA8007047838B23F47B6323F00F031B041B0C44
:10DFB8008383022303840B88828BB3F5007F10B51B
:10DFC80092B205D0002B0CBF4FF48073002301E000
:10DFD8004FF480734C8822438C88898942F400620C
:10DFE80022430A4392B21343838310BD808980B2CF
:10DFF800704781817047038819B19BB243F400537D
:10E0080003E023F400531B041B0C038070470388B0
:10E018009BB243F4805303807047012902D0008BE0
:10E0280080B27047808A80B27047008A80B2704799
:10E0380083889BB20AB1194301E023EA0101818078
:10E048007047090901238B409BB21AB1828892B2AA
:10E05800134303E0828892B222EA03038380704765
:10E06800038919420CBF002001207047C94389B2B7
:10E078000181704710B584880089012301F00F02DF
:10E0880080B213FA02F21040A4B205D009098B40FD
:10E098001C420CBF0020012010BD01F00F0101231C
:10E0A8008B40DB439BB20381704700BF08B5012159
:10E0B8004FF48040FFF7BAFD4FF480400021BDE8DF
:10E0C8000840FFF7B3BD014B1860704700380140A6
:10E0D80001F0030289080A4B023130B5920053F867
:10E0E80021500F24944025EA040443F8214053F8B2
:10E0F800214010FA02F2144343F8214030BD00BF1A
:10E1080000380140014B1860704700BFDC0027420F
:10E11800014B1860704700BF00042742024B186A81
:10E12800C0F30020704700BF0038014030B5048CB0
:10E1380024F001042404240C0484058B048CADB25F
:10E14800A4B225F0F305154324F00A0445EA0315A3
:10E1580044F00104ADB20C430583048430BD30B5EE
:10E16800048C24F010042404240C0484048B058CEF
:10E1780024F44074ADB22405240D25F0A00544EA2A
:10E18800022445F0100544EA033445EA0115A4B217
:10E19800ADB20483058430BD08B5474B984205D11C
:10E1A80001200146FFF742FD01203DE0B0F1804F1C
:10E1B80005D101200146FFF72DFD012076E03F4BF8
:10E1C800984205D102200121FFF724FD02206DE0CD
:10E1D8003B4B984205D104200121FFF71BFD042089
:10E1E80064E0384B984205D108200121FFF712FD61
:10E1F80008205BE0344B984205D110200121FFF73D
:10E2080009FD102052E0314B984205D12020012110
:10E21800FFF700FD202049E02D4B984209D102204C
:10E228000121FFF703FD02200021BDE80840FFF7A8
:10E23800FDBC284B984207D14FF480300121FFF7ED
:10E24800F5FC4FF48030EFE7234B984207D14FF4A9
:10E2580000300121FFF7EAFC4FF40030E4E71F4BE0
:10E26800984207D14FF480200121FFF7DFFC4FF4DB
:10E278008020D9E71A4B984205D140200121FFF7A9
:10E28800C9FC402012E0174B984205D1802001219B
:10E29800FFF7C0FC802009E0134B98420BD14FF4E4
:10E2A80080700121FFF7B6FC4FF480700021BDE8B3
:10E2B8000840FFF7AFBC08BD000001400004004063
:10E2C80000080040000C004000100040001400400E
:10E2D8000004014000400140004401400048014062
:10E2E80000180040001C0040002000401C4A038821
:10E2F80090429BB212D002F5806290420ED0B0F1EB
:10E30800804F0BD0A2F58032904207D002F5806290
:10E31800904203D002F58062904203D14A8823F0EC
:10E32800700313430F4A904208D002F5806290426E
:10E3380004D023F440730A899BB2134303804B68CB
:10E34800C3620B880385064B984203D003F58063AC
:10E35800984201D18B7A038601238382704700BFDC
:10E3680000000140001000404FF0FF3343600023DD
:10E3780003800381438083727047018582827047DE
:10E38800038823F070031B041B0C0B4303807047A6
:10E3980041627047C1627047406A7047008D80B221
:10E3A8007047038819B19BB243F0020303E023F0DE
:10E3B80002031B041B0C03807047038819B19BB22E
:10E3C80043F0040303E023F004031B041B0C038045
:10E3D8007047038819B19BB243F0800303E023F030
:10E3E80080031B041B0C03807047038823F0080379
:10E3F8001B041B0C038003889BB20B4303807047EC
:10E40800038823F440731B041B0C038003889BB20E
:10E418000B4303807047038819B19BB243F0010393
:10E4280003E023F001031B041B0C03807047038CDB
:10E4380023F001031B041B0C038470B5038C848830
:10E44800028B0D884E8822F073021204120C2A43A4
:10E458008D8923F002031B0435431B0CADB22B43FB
:10E468000E4DA842A4B203D005F58065A8420ED18E
:10E47800CD894E8A23F008032B438D8823F00403AB
:10E488002B430D8A354324F44074ADB22C43848069
:10E4980002838A684263038470BD00BF00000140A4
:10E4A800038C23F010031B041B0C0384038C828849
:10E4B80030B5048B0D8824F4E6442404240C23F09E
:10E4C800200344EA05241B048D891B0C43EA051329
:10E4D8004D8843EA0513134DA84292B2A4B29BB2E9
:10E4E80003D005F58065A84215D1CD8923F08003B6
:10E4F8009BB243EA05134FF6BF751D408B8845EA6A
:10E5080003130D8A22F4406242EA85024D8A42EAE8
:10E5180085029BB292B282808A68048382630384F4
:10E5280030BD00BF00000140038C23F480731B043E
:10E538001B0C0384038C828830B5848B0D8824F0EF
:10E5480073042404240C23F400731B042C438D89C6
:10E558001B0C43EA05234D8843EA0523124DA842C4
:10E5680092B29BB203D005F58065A84215D1CD893A
:10E5780023F400639BB243EA05234FF6FF351D40A1
:10E588008B8845EA03230D8A22F4405242EA051299
:10E598004D8A42EA05129BB292B282808A688483CD
:10E5A800C263038430BD00BF00000140038C23F424
:10E5B80080531B041B0C0384038C30B58488828B26
:10E5C8000D8822F4E6421204120C23F4005342EAA6
:10E5D80005221B048D891B0C43EA05334D8843EA49
:10E5E80005330B4DA842A4B292B29BB203D005F5F5
:10E5F8008065A84205D10D8A24F4804444EA851434
:10E60800A4B2848082838A680264038430BD00BF18
:10E61800000001400023038043808380836083815E
:10E62800C38103824382704730B5058C0124ADB2A3
:10E638008C4025EA040400F11803048409B1082970
:10E6480007D149084FF68F70CC582040C850C85899
:10E658000AE00439C1F34E0148F6FF70CC58204057
:10E66800C8501202C85892B20243CA5030BD416322
:10E67800704781637047C163704701647047038BBB
:10E6880023F070031B041B0C0B4303837047038B9D
:10E6980023F4E0431B041B0C43EA01239BB20383CE
:10E6A8007047838B23F070031B041B0C0B4383837D
:10E6B8007047838B23F4E0431B041B0C43EA0123BC
:10E6C8009BB283837047038B23F008031B041B0C46
:10E6D8000B4303837047038B23F400631B041B0C59
:10E6E80043EA01239BB203837047838B23F008031B
:10E6F8001B041B0C0B4383837047838B23F4006339
:10E708001B041B0C43EA01239BB283837047038BD2
:10E7180023F004031B041B0C0B4303837047038B78
:10E7280023F480631B041B0C43EA01239BB203837D
:10E738007047838B23F004031B041B0C0B43838358
:10E748007047838B23F480631B041B0C43EA01236B
:10E758009BB283837047038B23F080031B041B0C3D
:10E768000B4303837047038B09025B0441EA53435D
:10E778009BB203837047838B23F080031B041B0C1D
:10E788000B4383837047838B09025B0441EA53433D
:10E798009BB283837047038C23F002031B041B0C7A
:10E7A8000B4303847047038C23F008031B041B0CE2
:10E7B8000B4303847047038C23F020031B041B0CBA
:10E7C80043EA01139BB203847047038C23F0800350
:10E7D8001B041B0C43EA01139BB203847047038C90
:10E7E80023F400731B041B0C43EA01239BB203842C
:10E7F8007047038C23F400631B041B0C43EA0123BA
:10E808009BB203847047038C23F400531B041B0C36
:10E8180043EA01339BB20384704710B5048C01238B
:10E828008B40A4B224EA03030384038C12FA01F197
:10E838000B439BB2038410BD10B5048C04238B409A
:10E84800A4B224EA03030384038C12FA01F10B43F4
:10E858009BB2038410BD0023012203804380828081
:10E86800C38003817047406B7047806B7047C06BF3
:10E878007047006C7047038B23F00C031B041B0CC0
:10E888000383038B9BB20B4303837047038B23F4EF
:10E8980040631B041B0C0383038B9BB243EA0123D5
:10E8A8009BB203837047F8B50C464988A288B4F830
:10E8B80000E02389054600290CBF02270027012A0A
:10E8C80014BF01260226BEF1000F10D1FFF72EFC5F
:10E8D8002846E188FFF7CFFF284639463246238984
:10E8E800FFF73DFCE1882846BDE8F840CEE7FFF792
:10E8F80036FC2846E188FFF7C9FF284639463246E4
:10E908002389FFF713FCE1882846BDE8F840B2E701
:10E91800838B23F00C031B041B0C8383838B9BB218
:10E928000B4383837047838B23F440631B041B0CC6
:10E938008383838B9BB243EA01239BB28383704713
:10E94800F8B50D460B88AA88498804463BB92B8937
:10E95800FFF7ECFBE9882046BDE8F8408BE7042B7D
:10E9680007D12B89FFF7FBFBE9882046BDE8F84073
:10E978008CE7082BB5F808C0078C1DD127F48077E1
:10E988003F043F0C0784868B038CB6B29BB226F0FB
:10E99800F30623F4206346EA0C1C43EA01211FFA1C
:10E9A8008CFC89B24CEA020241F4807182830184B2
:10E9B800E988BDE8F840ABE727F480573F043F0CEF
:10E9C8000784868B038C26F4407623F4005336059F
:10E9D8005B04360D5B0C46EA022243EA013342EA45
:10E9E8000C329BB2E98892B243F480538283038449
:10E9F800BDE8F84097E74A880B8813438A88134391
:10EA0800CA8813430A8913434A8913438A891343DB
:10EA18009BB2A0F844307047002303804380838072
:10EA2800C3800381438183817047B0F8443029B1A2
:10EA38006FEA43436FEA53439BB201E05B045B0C0C
:10EA4800A0F844307047838819B19BB243F004039F
:10EA580003E023F004031B041B0C838070478388A6
:10EA680019B19BB243F0010303E023F001031B0437
:10EA78001B0C8380704783899BB20AB1194301E05C
:10EA880023EA01018181704781827047038A194214
:10EA98000CBF002001207047C94389B2018270472A
:10EAA800038A828911EA030092B203D011420CBF93
:10EAB800002001207047C94389B2018270470A4388
:10EAC800A0F84820704783899BB20AB1194301E036
:10EAD80023EA010181817047838819B19BB243F011
:10EAE800080303E023F008031B041B0C8380704712
:10EAF800038923F007031B041B0C03817047038958
:10EB080023F070031B041B0C0B43038103899BB286
:10EB180043F007030381704738B50D4611460122BB
:10EB2800602D044602D1FFF71AFB01E0FFF7FEFA59
:10EB3800238923F070031B041B0C1D4325812389A3
:10EB48009BB243F00703238138BD038923F0700388
:10EB58001B041B0C0B4303817047838823F070034D
:10EB68001B041B0C838083889BB20B4383807047F4
:10EB7800038923F007031B041B0C038103899BB241
:10EB88000B4303817047038923F080031B041B0C8C
:10EB9800038103899BB20B430381704710B5048935
:10EBA800E4B20C43144344EA0324A4B2048110BD24
:10EBB80010B50446FFF7F2FF23899BB243F4804364
:10EBC800238110BD10B50446FFF7E8FF238923F021
:10EBD80077031B041B0C43F07703238110BD70B52A
:10EBE8000489068B058C26F44076ADB226F0030620
:10EBF80024F00704360425F022052404360C1543B6
:10EC0800240C46F4807645EA0315214346F00106B4
:10EC1800ADB201810683058470BD838819B19BB2AA
:10EC280043F0800303E023F080031B041B0C838064
:10EC38007047A0F85010704708B5234B984205D18B
:10EC480010200121FEF7F2FF102037E01F4B9842F9
:10EC580007D14FF400300121FEF7DCFF4FF40030FC
:10EC680009E01B4B98420BD14FF480200121FEF79D
:10EC7800D1FF4FF480200021BDE80840FEF7CABF4D
:10EC8800144B984207D14FF400200121FEF7C2FF30
:10EC98004FF40020EFE7104B984207D14FF4801053
:10ECA8000121FEF7B7FF4FF48010E4E70B4B9842C1
:10ECB80009D120200121FEF7B9FF20200021BDE85D
:10ECC8000840FEF7B3BF08BD0010014000440040F3
:10ECD80000480040004C0040005000400014014033
:10ECE800038ACA889BB223F4405330B513430D46B8
:10ECF800038283890989AA8823F4B0530A4369895E
:10ED080023F00C031B040A431B0C92B213438381A8
:10ED1800838AAA899BB223F44073134385B0838204
:10ED280004466846FEF7A6FE1A4B9C4203D003F53C
:10ED380080639C4201D1039B00E0029BA28912B22E
:10ED4800002A4FF019012A6801FB03F101DA520089
:10ED580000E092006423B1FBF2F1B1FBF3F212017F
:10ED6800100903FB1011A08900B2002806DAC900B7
:10ED78003231B1FBF3F303F0070305E00901323147
:10ED8800B1FBF3F303F00F031A4392B2228105B0EB
:10ED980030BD00BF001001404FF4165303600C2231
:10EDA80000238380C38003814281838170470B885D
:10EDB800028A10B54C8823438C88C988234392B2B1
:10EDC8000B4322F470629BB21343038210BD0023ED
:10EDD800038043808380C3807047838919B19BB2C5
:10EDE80043F4005303E023F400531B041B0C8381FA
:10EDF8007047038B03F47F430383038B9BB20B435E
:10EE080003837047838929B16FEA43436FEA534309
:10EE18009BB201E05B045B0C83817047838A19B164
:10EE28009BB243F4006303E023F400631B041B0C50
:10EE380083827047C905C90D818070478088C005E5
:10EE4800C00D7047038A23F00F031B041B0C0382B9
:10EE5800038A9BB20B4303827047838919B19BB223
:10EE680043F0020303E023F002031B041B0C83811D
:10EE78007047838923F400631B041B0C83818389F7
:10EE88009BB20B4383817047038A23F020031B0442
:10EE98001B0C0382038A9BB20B4303827047038ACD
:10EEA80019B19BB243F4804303E023F480431B046D
:10EEB8001B0C0382704783899BB243F00103838153
:10EEC8007047838A19B19BB243F0080303E023F02B
:10EED80008031B041B0C83827047038BDBB203837C
:10EEE800038B9BB243EA012303837047838A19B1DA
:10EEF8009BB243F0200303E023F020031B041B0C08
:10EF080083827047838A19B19BB243F0100303E0F0
:10EF180023F010031B041B0C83827047838A23F0A1
:10EF280004031B041B0C8382838A9BB20B438382DA
:10EF38007047838A19B19BB243F0020303E023F0C0
:10EF480002031B041B0C83827047838A9BB20AB19D
:10EF5800194301E023EA010181827047C1F342139A
:10EF680010B501F01F01012414FA01F1A34201D1E7
:10EF78000C3004E0022B01D1103000E0143003689B
:10EF88000AB1194301E023EA0101016010BD0388B9
:10EF980019420CBF002001207047C94389B2018083
:10EFA8007047012210B501F01F03C1F342149A40C3
:10EFB800012C01D1838903E0022C0CBF038A838AC8
:10EFC8009BB21340028892B243B1090A012313FA93
:10EFD80001F111420CBF0020012010BD184610BDE0
:10EFE800090A01238B40DB439BB20380704700BFB3
:10EFF80081F0004102E000BF83F0004330B54FEAE2
:10F0080041044FEA430594EA050F08BF90EA020F4E
:10F018001FBF54EA000C55EA020C7FEA645C7FEAE1
:10F02800655C00F0E2804FEA5454D4EB5555B8BF04
:10F038006D420CDD2C4480EA020281EA030382EA75
:10F04800000083EA010180EA020281EA0303362D07
:10F0580088BF30BD11F0004F4FEA01314FF4801CDA
:10F068004CEA113102D0404261EB410113F0004FEC
:10F078004FEA03334CEA133302D0524263EB4303A3
:10F0880094EA050F00F0A780A4F10104D5F1200E41
:10F098000DDB02FA0EFC22FA05F2801841F100019C
:10F0A80003FA0EF2801843FA05F359410EE0A5F170
:10F0B80020050EF1200E012A03FA0EFC28BF4CF0A1
:10F0C800020C43FA05F3C01851EBE37101F0004557
:10F0D80007D54FF0000EDCF1000C7EEB00006EEB64
:10F0E8000101B1F5801F1BD3B1F5001F0CD34908EE
:10F0F8005FEA30004FEA3C0C04F101044FEA445245
:10F1080012F5800F80F09A80BCF1004F08BF5FEACB
:10F11800500C50F1000041EB045141EA050130BDAB
:10F128005FEA4C0C404141EB010111F4801FA4F14E
:10F138000104E9D191F0000F04BF01460020B1FAA3
:10F1480081F308BF2033A3F10B03B3F120020CDADB
:10F158000C3208DD02F1140CC2F10C0201FA0CF0B9
:10F1680021FA02F10CE002F11402D8BFC2F1200C1E
:10F1780001FA02F120FA0CFCDCBF41EA0C019040D4
:10F18800E41AA2BF01EB0451294330BD6FEA04041D
:10F198001F3C1CDA0C340EDC04F11404C4F1200208
:10F1A80020FA04F001FA02F340EA030021FA04F31A
:10F1B80045EA030130BDC4F10C04C4F1200220FA71
:10F1C80002F001FA04F340EA0300294630BD21FAAF
:10F1D80004F0294630BD94F0000F83F4801306BF75
:10F1E80081F480110134013D4EE77FEA645C18BF69
:10F1F8007FEA655C29D094EA050F08BF90EA020F00
:10F2080005D054EA000C04BF1946104630BD91EAF7
:10F21800030F1EBF0021002030BD5FEA545C05D1FA
:10F228004000494128BF41F0004130BD14F5800439
:10F238003CBF01F5801130BD01F0004545F0FE41AD
:10F2480041F470014FF0000030BD7FEA645C1ABFE2
:10F25800194610467FEA655C1CBF0B46024650EA19
:10F26800013406BF52EA033591EA030F41F4002145
:10F2780030BD00BF90F0000F04BF0021704730B5CB
:10F288004FF4806404F132044FF000054FF00001A0
:10F2980050E700BF90F0000F04BF0021704730B561
:10F2A8004FF4806404F1320410F0004548BF404236
:10F2B8004FF000013EE700BF42004FEAE2014FEA8B
:10F2C80031014FEA02701FBF12F07F4393F07F4F66
:10F2D80081F06051704792F0000F14BF93F07F4F98
:10F2E800704730B54FF4607401F0004521F00041DB
:10F2F80020E700BF50EA010208BF704730B54FF061
:10F3080000050AE050EA010208BF704730B511F065
:10F31800004502D5404261EB41014FF4806404F19D
:10F3280032045FEA915C3FF4DCAE4FF003025FEA1F
:10F33800DC0C18BF03325FEADC0C18BF033202EBA7
:10F34800DC02C2F1200300FA03FC20FA02F001FA01
:10F3580003FE40EA0E0021FA02F11444C1E600BFA0
:10F3680070B54FF0FF0C4CF4E06C1CEA11541DBF53
:10F378001CEA135594EA0C0F95EA0C0F00F0DEF81E
:10F388002C4481EA030621EA4C5123EA4C5350EA03
:10F39800013518BF52EA033541F4801143F4801354
:10F3A80038D0A0FB02CE4FF00005E1FB02E506F0E5
:10F3B8000042E0FB03E54FF00006E1FB03569CF03A
:10F3C800000F18BF4EF0010EA4F1FF04B6F5007F40
:10F3D80064F5407404D25FEA4E0E6D4146EB0606B2
:10F3E80042EAC62141EA55514FEAC52040EA5E503B
:10F3F8004FEACE2EB4F1FD0C88BFBCF5E06F1ED8E5
:10F40800BEF1004F08BF5FEA500E50F1000041EB1B
:10F41800045170BD06F0004646EA010140EA0200C8
:10F4280081EA0301B4EB5C04C2BFD4EB0C0541EAEA
:10F43800045170BD41F480114FF0000E013C00F3FF
:10F44800AB8014F1360FDEBF002001F0004170BD23
:10F45800C4F10004203C35DA0C341BDC04F114043C
:10F46800C4F1200500FA05F320FA04F001FA05F2C8
:10F4780040EA020001F0004221F0004110EBD37095
:10F4880021FA04F642EB06015EEA430E08BF20EAC1
:10F49800D37070BDC4F10C04C4F1200500FA04F364
:10F4A80020FA05F001FA04F240EA020001F00041F6
:10F4B80010EBD37041F100015EEA430E08BF20EA69
:10F4C800D37070BDC4F1200500FA05F24EEA020EB1
:10F4D80020FA04F301FA05F243EA020321FA04F0E0
:10F4E80001F0004121FA04F220EA020000EBD37097
:10F4F8005EEA430E08BF20EAD37070BD94F0000F97
:10F508000FD101F00046400041EB010111F4801FCA
:10F5180008BF013CF7D041EA060195F0000F18BF7B
:10F52800704703F00046520043EB030313F4801FB7
:10F5380008BF013DF7D043EA0603704794EA0C0F71
:10F548000CEA135518BF95EA0C0F0CD050EA410687
:10F5580018BF52EA4306D1D181EA030101F0004104
:10F568004FF0000070BD50EA410606BF104619462C
:10F5780052EA430619D094EA0C0F02D150EA013638
:10F5880013D195EA0C0F05D152EA03361CBF104679
:10F5980019460AD181EA030101F0004141F0FE4118
:10F5A80041F470014FF0000070BD41F0FE4141F49C
:10F5B800780170BD70B54FF0FF0C4CF4E06C1CEA9C
:10F5C80011541DBF1CEA135594EA0C0F95EA0C0F51
:10F5D80000F0A7F8A4EB050481EA030E52EA03350C
:10F5E8004FEA013100F088804FEA03334FF080552D
:10F5F80045EA131343EA12634FEA022245EA11155A
:10F6080045EA10654FEA00260EF000419D4208BF0A
:10F61800964244F1FD0404F5407402D25B084FEAB7
:10F628003202B61A65EB03055B084FEA32024FF463
:10F6380080104FF4002CB6EB020E75EB030E22BFC0
:10F64800B61A754640EA0C005B084FEA3202B6EB80
:10F65800020E75EB030E22BFB61A754640EA5C002F
:10F668005B084FEA3202B6EB020E75EB030E22BFBF
:10F67800B61A754640EA9C005B084FEA3202B6EBC0
:10F68800020E75EB030E22BFB61A754640EADC007F
:10F6980055EA060E18D04FEA051545EA16754FEAE1
:10F6A80006164FEAC30343EA52734FEAC2025FEAFF
:10F6B8001C1CC0D111F4801F0BD141EA00014FF08E
:10F6C80000004FF0004CB6E711F4801F04BF01435F
:10F6D8000020B4F1FD0C88BFBCF5E06F3FF6AFAE7B
:10F6E800B5EB030C04BFB6EB020C5FEA500C50F10B
:10F6F800000041EB045170BD0EF0004E4EEA11318E
:10F7080014EB5C04C2BFD4EB0C0541EA045170BD94
:10F7180041F480114FF0000E013C90E645EA060ED8
:10F728008DE60CEA135594EA0C0F08BF95EA0C0F06
:10F738003FF43BAF94EA0C0F0AD150EA01347FF44E
:10F7480034AF95EA0C0F7FF425AF104619462CE725
:10F7580095EA0C0F06D152EA03353FF4FDAE104688
:10F76800194622E750EA410618BF52EA43067FF4D9
:10F77800C5AE50EA41047FF40DAF52EA43057FF469
:10F78800EBAE12E74FF0FF3C06E000BF4FF0010C74
:10F7980002E000BF4FF0010C4DF804CD4FEA410CD8
:10F7A8007FEA6C5C4FEA430C18BF7FEA6C5C1BD0A5
:10F7B80001B050EA410C0CBF52EA430C91EA030F26
:10F7C80002BF90EA020F0020704710F1000F91EA83
:10F7D800030F58BF994208BF90422CBFD8176FEA51
:10F7E800E37040F0010070474FEA410C7FEA6C5C1F
:10F7F80002D150EA013C07D14FEA430C7FEA6C5C26
:10F80800D6D152EA033CD3D05DF8040B704700BF51
:10F818008446104662468C461946634600E000BF9F
:10F8280001B5FFF7B7FF002848BF10F1000F01BD71
:10F838004DF808EDFFF7F4FF0CBF012000205DF83C
:10F8480008FB00BF4DF808EDFFF7EAFF34BF0120C1
:10F8580000205DF808FB00BF4DF808EDFFF7E0FF5A
:10F8680094BF012000205DF808FB00BF4DF808EDAB
:10F87800FFF7CEFF94BF012000205DF808FB00BF12
:10F888004DF808EDFFF7C4FF34BF012000205DF8F4
:10F8980008FB00BF4FEA410212F5001215D211D53C
:10F8A8006FF47873B3EB625212D94FEAC12343F075
:10F8B800004343EA505311F0004F23FA02F018BFF7
:10F8C800404270474FF00000704750EA013005D1C0
:10F8D80011F0004008BF6FF0004070474FF0000083
:10F8E800704700BF4A0011D212F5001211D20DD58F
:10F8F8006FF47873B3EB62520ED44FEAC12343F02E
:10F90800004343EA505323FA02F070474FF00000D7
:10F91800704750EA013002D14FF0FF3070474FF086
:10F92800000070474FEA4102B2F1E04324BFB3F54B
:10F93800001CDCF1FE5C0DD901F0004C4FEAC0025E
:10F948004CEA5070B2F1004F40EB830008BF20F042
:10F958000100704711F0804F21D113F13872BCBFFC
:10F9680001F00040704741F480114FEA5252C2F151
:10F978001802C2F1200C10FA0CF320FA02F018BF9A
:10F9880040F001004FEAC1234FEAD32303FA0CFCED
:10F9980040EA0C0023FA02F34FEA4303CCE77FEA7C
:10F9A800625307D150EA01331EBF4FF0FE4040F4C6
:10F9B8004000704701F0004040F0FE4040F4000075
:10F9C800704700BF4BB942B9002908BF002802D0D0
:10F9D8004FF0FF31084600F037B882B0EC462DE909
:10F9E800005000F01BF8DDF804E002B00CBC7047D2
:10F9F800F8B5144606460F461D4600F027F804FBE6
:10FA080001F300FB0535A4FB0023EB18069CB21A92
:10FA180067EB0303C4E90023F8BD00BFF8B514463B
:10FA280006460F461D4600F075F900FB05F5A0FBDC
:10FA3800042304FB0155EB18069CB21A67EB030379
:10FA4800C4E90023F8BD00BF704700BF00292DE9B5
:10FA5800F0071D46C0F29E800024002DC0F295805C
:10FA680007460D4616469C46002B3ED18A4254D97D
:10FA7800B2FA82F343B1C3F1200620FA06F501FA7F
:10FA880003F19A4029439840160CB1FBF6F597B25A
:10FA980006FB15114FEA104C07FB05F34CEA014130
:10FAA8008B4209D9891805F1FF3C80F015818B42FA
:10FAB80040F21281023D8918C3EB010CBCFBF6F33E
:10FAC80006FB13C180B207FB03F740EA01408742F7
:10FAD80007D9591E821880F00581974240F20281A9
:10FAE800023B43EA0542002303E08B420AD9002384
:10FAF8001A461046194614B1404261EB4101BDE86F
:10FB0800F0077047B3FA83F3002B40F087808C45E9
:10FB180001D38242ECD80122EBE712B90123B3FBEF
:10FB2800F2F2B2FA82F6002E3AD1891A150C1FFAAF
:10FB380082FC0123B1FBF5F705FB17114FEA1048CA
:10FB48000CFB07F648EA01418E4207D9891807F1EC
:10FB5800FF3802D28E4200F2DA804746891BB1FB99
:10FB6800F5F605FB161180B20CFB06FC40EA0140D5
:10FB7800844507D9711E821880F0B080944540F200
:10FB8800AD80023E46EA0742B3E7E443524263EBE4
:10FB9800430365E7404261EB41014FF0FF345CE706
:10FBA800B240C6F1200521FA05F320FA05F701FA5B
:10FBB80006F9150CB3FBF5F847EA09091FFA82FCA8
:10FBC80005FB18374FEA19410CFB08F341EA0747D0
:10FBD800B040BB420AD9BF1808F1FF3180F09580C8
:10FBE800BB4240F29280A8F10208BF18FE1AB6FB89
:10FBF800F5F305FB13611FFA89F90CFB03F649EAD3
:10FC080001418E4206D95F1E891878D28E4276D974
:10FC1800023B8918891B43EA08438BE7C3F1200795
:10FC280026FA07F80CFA03F248EA020C21FA07F15F
:10FC380005FA03FA4FEA1C4920FA07F5B1FBF9F86F
:10FC480045EA0A0509FB18172A0C1FFA8CFA0AFB61
:10FC580008F142EA0747B94206FA03F609D917EB51
:10FC68000C0708F1FF324ED2B9424CD9A8F102086C
:10FC780067447F1AB7FBF9F209FB1271ADB20AFBB0
:10FC880002FA45EA01418A4507D9551E11EB0C01D4
:10FC980037D28A4535D9023A614442EA08424FEAE6
:10FCA800124C1FFA86F808FB0CF7360C95B208FBC5
:10FCB80005F806FB057505EB184506FB0CFCAF427D
:10FCC80088BF0CF5803CCAEB01010CEB1546B1422C
:10FCD80012D309D000230CE76546EDE60E4646EA46
:10FCE800074206E70B46FCE61FFA88F800FA03F31A
:10FCF80008EB0545AB42EDD2013A0023F9E63B4655
:10FD080088E72A46C9E79046B3E788466EE7023F88
:10FD1800891823E72DE9F00F144605460E46002BF7
:10FD28003FD18A424AD9B2FA82F343B1C3F12000E3
:10FD380025FA00F201FA03F69C4016439D40210C77
:10FD4800B6FBF1F22F0CA0B201FB126C00FB02F320
:10FD580047EA0C46B34208D9571E361980F0FF808F
:10FD6800B34240F2FC80023A3619F61AB6FBF1F3B8
:10FD780001FB1361ADB200FB03F045EA0141884283
:10FD880007D95E1E091980F0EC80884240F2E980AC
:10FD9800023B43EA0242002310461946BDE8F00F31
:10FDA80070478B4243D8B3FA83F4002C42D18B427C
:10FDB800234601D382423BD80122EDE712B9012341
:10FDC800B3FBF2F4B4FA84F2002A40F08A80091BEB
:10FDD800260CA7B20123B1FBF6F006FB10114FEA7F
:10FDE800154C07FB00F24CEA01418A4207D9091970
:10FDF80000F1FF3C02D28A4200F2D3806046C2EB97
:10FE0800010CBCFBF6F206FB12C1ADB207FB02F710
:10FE180045EA0145AF4207D9511E2C1980F0A3804D
:10FE2800A74240F2A080023A42EA0042B4E7002327
:10FE38001A46B1E7C4F1200722FA07F603FA04F3D9
:10FE4800334321FA07FA4FEA134C01FA04FB20FA6C
:10FE580007F141EA0B0BBAFBFCF70CFB17A61FFADC
:10FE680083F84FEA1B4508FB07F945EA0645A9450B
:10FE780002FA04FA04D97A1EED18C0F088801746F1
:10FE8800C9EB0505B5FBFCF60CFB16521FFA8BFBFC
:10FE980008FB06F84BEA0241884503D9721EC918C7
:10FEA80070D3164646EA0742170C1FFA8AFC0CFB69
:10FEB80007F695B24FEA1A430CFB05FC03FB0565F0
:10FEC80005EB1C4503FB07F3AE4288BF03F58033FF
:10FED800C8EB010103EB1543994250D347D00023E7
:10FEE8005AE79440C2F12008260C20FA08F721FAB4
:10FEF80008F501FA02F9B5FBF6F847EA090906FB25
:10FF08001855A7B24FEA194C4CEA054C07FB08F301
:10FF1800634500FA02F509D91CEB040C08F1FF321D
:10FF28003DD263453BD9A8F10208A444C3EB0C02B7
:10FF3800B2FBF6F306FB13201FFA89F907FB03F25D
:10FF480049EA00418A4206D9581E091925D28A422F
:10FF580023D9023B0919891A43EA08433BE73A4681
:10FF680003E7334615E70A4642EA004214E71FFA58
:10FF78008CF100FA04F001EB0545A842AFD2013A32
:10FF8800002309E788458CD9023EC9188AE7A945A4
:10FF98007FF675AF023FED1872E70346DBE7904640
:10FFA800C4E7023809192AE7002103E00A4B5B5825
:10FFB8004350043109480A4B42189A42F6D3094A79
:10FFC80002E0002342F8043B074B9A42F9D3FAF7C0
:10FFD800BBF900F00DF87047FCAB050800000020E5
:10FFE800FC0C0020000D00200C520020FEE7000051
:08FFF800A84BF7B54FF4FA66BF
:020000040801F1
:100000001E60A74AA74BA84F1A60A84AA84B1A60BF
:10001000A84B42F210721A60A74B64241C600123A3
:100020003B70F8F75CFFA54B00251D70F8F7F2F860
:10003000F6F7C2F9F6F7CCF9F6F7DAF9F6F7D6FFE4
:100040002046F7F753FCF6F7F7FF2046F7F74EFC8C
:10005000F8F7C6F8F7F7F8FEF7F756FC2046F7F77B
:1000600045FCFAF7C1FA2046F7F740FC4FF4FA5086
:10007000F7F7A8FB2046F7F739FCF6F70FFF204605
:10008000F7F734FC2846F7F713FD8D48F7F72EFCF9
:10009000F4F7D6FC2046F7F729FC8A4B03F110024F
:1000A00029468DE8240028465A681B68F4F7DAFAD6
:1000B0003046F7F71BFC2846F4F7ACFE4FF6FF700E
:1000C000F4F7BEFE032132207F4A2B46F4F7DCFF13
:1000D00096207E4A8C212B46F4F7D6FF9620A0214D
:1000E0007B4A2B46F4F7D0FF7A4A2B469620B42160
:1000F000F4F7CAFFF8F7AAFE5021DC20F8F779FEE2
:100100003046F7F7F3FB744A2B46DC212846F4F718
:10011000BBFF7248F7F7EAFB2046F7F7E7FBF6F775
:1001200065FC2046F7F7E2FB9FED6D0AF7F7D8FC78
:100130002046F7F7DBFBF7F701FCF5F76FFA2046EF
:10014000F7F7D4FB14200146F6F7BEF92846F6F778
:1001500011FA2046F7F7CAFBF6F792FB2046F7F7AD
:10016000C5FBF6F73BFF2046F7F7C0FBF6F78EFC22
:1001700000B13D70F6F796FC08B1F8F711FE594B47
:1001800000241C70F1F70AFAF5F7FEF908B9564891
:1001900002E0564B56481C70F1F71BFAF5F768FE63
:1001A000F8F753FBF8F786FBF9F7F0F8F8F73AF9A8
:1001B000F8F719FEFAF780F9F8F768FE4D4B4E4D47
:1001C0004E4C802814BF4FF480504FF4806018804C
:1001D000374B1A68334B1B68D21A364B1B6892FB9D
:1001E000F3F2474B2E461A80F6F772FC2B7833B1A8
:1001F000012B02D1F7F756FE01E0F7F77BFE00274F
:100200003770F7F7D5FFF3F7E1F9F9F795F92378A8
:1002100013B12770F1F74CFE384B5B781BB100230C
:100220006370F1F7C9FA374B1A8812B2012A13D159
:1002300035484FF40051FDF75EF9A3780BB9F9F793
:10024000A5F9F7F743FF00222F484FF40051FDF7BF
:1002500052F92C4B00221A80E3783BB10020E07069
:10026000F4F7D2F8294B1878F0F716FD237943B14B
:10027000F8F7ECFDF0209621F8F7BBFD2448F7F7DE
:100280002BF9244F3846FBF79AFC0028ACD03B787A
:10029000112BA9D1F8F7FCFCA6E700BF783E00209F
:1002A000E0673500A83E0020280F002080C3C90168
:1002B000C44400209C440020583E00203C460020BE
:1002C00000127A00008401084FA4050869A40508FB
:1002D00076A4050882A405088BA40508002D310129
:1002E0000000FA44883E002058110020403E0020C3
:1002F00044130020A43E0020A04400200C0E002047
:1003000004480020F00D002000080240B8440020FE
:1003100040420F00413E002010B4314C0180B1F545
:10032000807F44608270C37052D00DD9B1F5806F68
:1003300039D017D9B1F5006F2ED0B1F5805F24D038
:10034000FF2040B210BC704720293AD014D9402970
:1003500030D08029F4D123494FF02012C26081604F
:100360000020EEE7B1F5007FEAD11F4B4FF00811F6
:10037000C16083600020E4E71029E1D11B494FF000
:100380000122C26081600020DBE7194B4FF00111B0
:10039000C16083600020D4E7164A4FF00213C360A7
:1003A00082600020CDE714494FF00412C2608160E2
:1003B0000020C6E7114B4FF04011C1608360002060
:1003C000BFE70F4A4FF08013C36082600020B8E798
:1003D0000C4A4FF01013C36082600020B1E700BFE9
:1003E000E4A2040822930508F2920508E2940508A5
:1003F000E4920508E6920508EA920508629305086A
:10040000E2930508029305082DE9F00FB2B02E9093
:1004100030932E9B00882E9C5B68309FA4682D90A3
:10042000451E03EB4506BF08209328942C952F9179
:100430001F921E96319700F03A814FEA900A4FEAD8
:10044000CA0B00F003002F99299003F1080504EB73
:100450000B00CDF884A0CDF8A8B019951A921B977F
:10046000189617912B90179A189E13883380B2F81C
:1004700002C0A6F802C09488B480D788F7800836F6
:100480001896219F199E0832179256F8041C56F8A8
:10049000082C4FF0000A4FF0000B002F00F069828B
:1004A000CDE904ABCDE906ABCDE902ABCDE900ABBC
:1004B000289CBC46029BDDF80C902568C2FBC53920
:1004C0004FF0000848EA030ACB46CDE902AB049B93
:1004D000DDF814B0C1FBC53BCDF824B0CDF82080C9
:1004E000DDE908ABC1EA02004AEA030ACDE904AB40
:1004F000069BDDF81CB03268C0FBD53BCDF82CB0B4
:10050000CDF82880DDE90AABC2EA01074AEA030A0E
:10051000CDE906AB9DE80108C7FBD50BCDF834B09B
:10052000CDF83080DDE90CAB4AEA000A6368029836
:10053000CDE900AB0834DDF80CB0C1FBC30BCDF83E
:100540003CB0CDF83880DDE90EAB4AEA000ACDE9CF
:1005500002AB71680498DDF814B0C2FBC30BCDF890
:1005600044B0CDF84080DDE910AB4AEA000ACDE99D
:1005700004AB0698DDF81CB0C7FBD30BCDF84CB02C
:10058000CDF84880DDE912ABC1EA02054AEA000A6B
:10059000CDE906AB9DE80108C5FBD30BCDF854B0FF
:1005A000CDF85080DDE914AB08364AEA000ABCF108
:1005B000010CCDE900AB7FF47DAF2A9D19982B9BF0
:1005C0002E18299F002F35D01868039F029BC2FB6D
:1005D000C03700241D971C94DDE91C4544EA030440
:1005E000CDE90245049B059DC1FBC035002723953D
:1005F0002297DDE9224544EA0304CDE90445C1EA36
:100600000203079D069AC3FBD02525952497DDE9B3
:10061000244544EA02043368C3EA0101CDE90645F2
:1006200053465D46C1FBD03527952697DDE926ABBD
:100630004AEA030A069A029C0499039D079FD30B7A
:10064000059AE60BC90B46EA454043EA474441EAAE
:10065000424604F30F0500F30F0C199BCCEA054743
:1006600006F30F001A9D1B9E2F604FEADA3A0833FB
:100670004AEA4B4B0BF30F04C0EA04426A600835A8
:10068000711E19931A951B917FF4EDAE319A2F9E2E
:100690001E991F9BDDF880B0D00037180D182F97DA
:1006A0000BEB000A1F181E951F97CDF880A0DDF8F0
:1006B000C0C01CF0030BCDF820B000F086802D9B4D
:1006C000DDF8BC80CDF808B05808DDF880A0DDF872
:1006D000A0B00690CDF81080049A1E9E32F8025BFE
:1006E000069826F8025B0492BAF80270BBF8023052
:1006F000BAF80020BBF800401E9617FB03F112FB6E
:1007000004F6451E4FEAE17711EB06082B4605F08B
:10071000010047EBE6790AF104020BF10401002D18
:100720003BD0A8B1B2F800C0BBF804705488488828
:100730001CFB07F518EB050749EBE57614FB00F900
:1007400017EB090846EBE97904320431013B24D068
:100750000F88B2F800C0568848888C8895881CFBA2
:1007600007FC18EB0C0816FB00F7D088CE8849EB85
:10077000EC7C15FB04F518EB07084CEBE77918EB5C
:10078000050710FB06FC49EBE57417EB0C0844EB7E
:10079000EC7908320831023BDAD11F9A02994FEA0C
:1007A000D83545EA494404F30F0322F8023B4F1EB3
:1007B0000AF1020A1F9202978ED1DDF880A0DDF8BF
:1007C00020B00AEB4B0ACDF880A02C9E2E98B508DD
:1007D00040683FD0209F47EA000212F0030F00F16B
:1007E000080307F1080214BF002101219F4298BFAE
:1007F000904294BF00260126314277D097E842000C
:10080000016001216C1EA942466004EA010419D06E
:1008100044B192E81200196002215C60083208338A
:10082000A9420FD092E850001C605E60966802F109
:10083000080BD2689E600231DA601033A9420BF1D6
:100840000802EFD1DDF880C0ED000CEB050B40197C
:10085000CDF880B02C9C14F0030343D05A08540008
:10086000002A00F08E80209D40EA050717F0030F54
:10087000209F14BF00250125011D3E1D012B94BFA3
:10088000002505F001058F4298BFB04294BF0021BA
:1008900001210D4275D039689200BF18A342016052
:1008A00020971044C4EB03011CD0209B013933F87E
:1008B000024B0A4620F8024B01F0010192B129B126
:1008C00033F8021B013A20F8021B0BD01C460146EC
:1008D00034F802CB21F802CB5D88A31C4580881C2C
:1008E000023AF3D132B0BDE8F00F7047B7F800C05C
:1008F000A0F800C07C884480BE888680691EFE887F
:100900000C46BA4601F00101C680002C9AD089B18C
:10091000B2F800B0A3F800B051885980B2F804C012
:10092000A3F804C0B2F806B00832A3F806B0083342
:10093000013C87D016881E8051885980B2F804B0D7
:10094000A3F804B0B2F806C0A3F806C016891E8149
:1009500003F1080B5189ABF802109389ABF804300E
:10096000D6891032023C0BF10803ABF80660E1D1E6
:1009700068E7289BCDE904ABCDE906ABCDE902AB36
:100980001FE6194691E700BF2DE9F00F9CB00678ED
:100990000F900F9C40880F9DA4686D681990B3FB61
:1009A000F6FA471E4FEA5A0804EB4709AAEB480338
:1009B00040460A940D951A97CDF86C800C911492CC
:1009C000CDF82C901193002800F0B5811746199AA4
:1009D000199CCDF848809108CA00159104F00303D2
:1009E000A9181792169310971891760075084FEA78
:1009F000450C002D00F03B840B9FDDF8308047EA6A
:100A0000080010F0030F14BF0021012108F10404B5
:100A1000381D012E94BF002101F00101804598BFCF
:100A2000A74294BF4FF000094FF0010911EA090FE6
:100A300000F01D84BB46D8F8002001236F1EAB4296
:100A4000CBF8002007EA03072146024614D237B14B
:100A5000246802230431021DAB4204600CD20C4610
:100A6000104654F8047B40F8047B49680233516017
:100A7000211D021DAB42F2D3DDF83080DDF82CB031
:100A80004FEA4C05664508EB05020BEB0503CCEB82
:100A900006001DD0013832F802CB014623F802CB04
:100AA00000F00100A1B128B132F8029B013923F80E
:100AB000029B0DD014461F4634F8029B27F8029B78
:100AC000B2F802A0A21CA3F802A0BB1C0239F1D10B
:100AD0000C9ADDF83CC00B989CF80080710053180C
:100AE0000A9E0C93159BCDF84C80451806EB4802E6
:100AF0000B950E92002B00F0B18300240025CDE968
:100B00000445CDE9024507930D9913460A9AB3F8B7
:100B100004A0B2F806B0CDF804A0B3F806A00E8881
:100B20001588CDF820B0CDF824A0DDE902AB15FB87
:100B300006F51AEB050A4BEBE57BCDE902AB1F8806
:100B40004888B2F802C0B3F80290B2F804808C88EA
:100B5000CDF81880DDE904AB16FB07F61AEB060AA0
:100B60004BEBE67BDDE902671CFB00F5761910FB19
:100B700009F047EBE5771AEB000A4BEBE07BCDE998
:100B800002ABDDF818B0DDF804C0B1F80680099DAD
:100B90001BFB04F016EB000A47EBE07BDDE9026784
:100BA00014FB0CF4361947EBE477089C14FB08F0AF
:100BB0000831083208331AEB000418FB05F84BEB38
:100BC000E075079816EB080A47EBE87B0138CDE99A
:100BD0000245CDE904AB079099D1179E0E9C0A9B64
:100BE0001899A7199A190E97169F002F73D00E9B6C
:100BF00031F8020B32F8024B33F8026BDDE902895F
:100C0000DDE904AB14FB00F47D1E10FB06F618EBC7
:100C1000040849EBE4791AEB060A4BEBE67B2F4616
:100C200005F00100CDE90289CDE904AB002D52D0D9
:100C3000002873D031F8024B32F8020B33F8025B14
:100C400010FB04F614FB05F0DDE90245DDE904893B
:100C5000A41945EBE67518EB000849EBE079013F74
:100C6000CDE90245CDE9048935D0C246CB46DDE960
:100C700002890D4614460497214628461A4630F844
:100C8000026B31F8027B32F802CB6D8864885B8896
:100C900017FB06F718EB070816FB0CF649EBE7798C
:100CA0001AEB060714FB05FA4BEBE67B15FB03FC7E
:100CB0008C1C931C0499851C18EB0A0849EBEA79F3
:100CC00017EB0C0A4BEBEC7B8A1ECDE902890492F0
:100CD000D2D1CDE904AB029D03990498DDF828A098
:100CE000059BEA0B109D42EA4148129908F30F094F
:100CF000A5F80090DDF84C90C70B0AEB8908281D79
:100D00004A1E47EA4346CDF8288006F30F041090A8
:100D10006C8012920AD00F9C267866E6DDE904AB5F
:100D20000D4614460497DDE90289A5E7149F1B9B35
:100D300007EB83061496119F002F00F0A681DDF8C3
:100D400064B0DDF86480DDF834C04FEA9B09CDF86B
:100D50001C904FEAC90908F0030A0CEB090BCDF807
:100D60002090CDF810A0CDF824B0DDF83CC09CF860
:100D7000006075084FEA450C002D00F07E820C994A
:100D80000B980B9F40EA010414F0030F14BF0022DC
:100D900001220C1D0430012E94BF002202F001023A
:100DA000814298BFA74294BF002301231A4200F05A
:100DB0006482BA4601230F68691EAB42CAF800700C
:100DC000024601EA0307214614D237B127680223FD
:100DD000211D021DAB4207600CD20C46104654F890
:100DE000047B40F8047B496802335160211D021DD9
:100DF000AB42F2D3DDF83090DDF82C804FEA4C05A1
:100E0000664509EB050208EB0503CCEB06001DD097
:100E1000013832F802BB014623F802BB00F00100A2
:100E2000A1B128B132F8025B013923F8025B0DD081
:100E300014461F4634F802AB27F802ABB2F802C0E2
:100E4000A21CA3F802C0BB1C0239F1D1DDF82CA012
:100E5000DDF830B0079876000AEB060C0BEB0608BD
:100E6000CDF82CC0CDF83080002800F0F0810A9A2F
:100E7000DDF834805788B2F800A0DDF82890948817
:100E8000B9F80690B8F8062084460D984188058880
:100E9000B8F8040017FB01F61AFB05F3B3461BEB89
:100EA00003014FEAE67714FB00F047EBE3750F18F8
:100EB0000A9B19FB02F145EBE0750CF1FF3617EBCD
:100EC000010AB14606F0010008F1080203F1080327
:100ED00045EBE17B002E00F0858048B3DDF834C09F
:100EE0001E88BCF808405888518897889D88B2F8B9
:100EF0000680B3F806C016FB04F41AEB040A10FBD4
:100F000001F14BEBE4761AEB010415FB07FB46EB12
:100F1000E17014EB0B011CFB08F640EBEB7408329C
:100F2000083311EB060A44EBE67BB9F1010959D00D
:100F3000CDE902ABCB46B3F80080B3F80890168831
:100F4000CDF8389018FB06F6DDE902895D885488F3
:100F500098889188B2F806C0DF88B2F808A015FB1F
:100F600004F418EB060810FB01F149EBE67918EBE5
:100F7000040817FB0CF749EBE47918EB010849EB7F
:100F8000E17918EB070849EBE779CDE90289DDF84B
:100F900038905D89548998899189B2F80EC0DE89AC
:100FA00019FB0AF7DDE9028915FB04F418EB0708C1
:100FB00010FB01F149EBE77918EB040849EBE47900
:100FC00016FB0CF618EB010449EBE17510321033F7
:100FD000A01945EBE671BBF1020BCDE90201AAD1E4
:100FE00082468B460DF1200898E816006318049D90
:100FF0009DB332F802CB33F8026B16FB0CF4013DC3
:101000001AEB040A294605F001004BEBE47B25B3FB
:1010100058B132F8028B33F8020B10FB08F71AEBC9
:10102000070A4BEBE77B691E17D01446184634F8C5
:10103000025B30F8027B52885B8817FB05F81AEBDD
:1010400008064BEBE87713FB02FBA21C831C16EB94
:101050000B0A47EBEB7B0239E7D10F9DDDF850809F
:1010600095F800C00A9A119E4FEADA3343EA4B44DE
:1010700004F30F0028F8020B02EB4C07711E0A97CD
:10108000CDF8508011917FF470AE1A9E0F9CB50878
:10109000A06842D00A9F47EA000616F0030F07F146
:1010A000080200F1080314BF002101219F4298BFEC
:1010B000904294BF4FF0000A4FF0010A11EA0A0F64
:1010C0007FD097E84200016001216C1EA942466072
:1010D00004EA010419D044B192E812001960022117
:1010E0005C6008320833A9420FD092E850001C60BF
:1010F0005E60966802F10804D2689E600231DA6090
:101100001033A94204F10802EFD1DDF828A0ED0068
:101110000AEB05094019CDF82890DDF868A01AF00F
:1011200003034AD05A085400002A00F0A480DDF8D6
:1011300028B040EA0B0515F0030F14BF0025012568
:101140000BF10406011D012B94BF002505F00105DC
:101150008B4598BFB04294BF4FF0000C4FF0010C8C
:1011600015EA0C0F00F08780DBF800109200934422
:10117000A3420160CDF828B01044C4EB03011CD099
:101180000A9B013933F8024B0A4620F8024B01F062
:10119000010192B129B133F8021B013A20F8021B78
:1011A0000BD01C46014634F802CB21F802CB5D88F7
:1011B000A31C4580881C023AF3D11CB0BDE8F00F97
:1011C0007047B7F80090A0F800907C884480BE88F3
:1011D0008680691EFE880C46B84601F00101C68073
:1011E000002C92D091B111881980B2F802C0A3F8F6
:1011F00002C0B2F804A0A3F804A0B2F80690083226
:10120000A3F806900833013C3FF47FAF11881980A2
:10121000B2F802C0A3F802C0B2F80490A3F8049098
:10122000B2F806A0A3F806A016891E8103F1080CE7
:101230005189ACF802109389ACF80430D689103289
:10124000023C0CF10803ACF80660DFD15DE70D9AB3
:101250000A9B4FF0000A4FF0000BC8E6002600275B
:10126000CDE904670A9A0D99CDE90267BCE43046DE
:101270000B9B0C9A0EE4194682E730460B9B0C9AA6
:10128000C6E500BF0000000000B553EC102B42F291
:10129000FB1223F00043C3F6E972934285B026DDCA
:1012A0004FF6FF72C7F6EF7293420BDD51EC100B55
:1012B00002460B46FDF7A4FE02460B4643EC102BFC
:1012C00005B000BD684600F0EBFB00F0030001280C
:1012D0009DED000B9DED021B1AD0022810D0F8B92D
:1012E00000F0FEFE53EC102B10461946E4E79FED8C
:1012F000101B00F0F5FE53EC102B10461946DBE7EF
:1013000000F0EEFE53EC102B104603F10041D3E742
:1013100001F022FC53EC102B104603F10041CBE707
:10132000012001F019FC53EC102B10461946C3E7BD
:1013300000000000000000002DE9F04759EC108B80
:10134000C9F30A56A6F57E74073C132C4D46CA46CF
:10135000474626DC002C4FDB4FF6FF76C0F20F0627
:1013600046FA04F606EA090555EA080517D044A32B
:10137000D3E9002351EC100BFDF744FE00220023BB
:10138000FEF782FA00284AD0B9F1000F6EDB2AEA94
:10139000060A4FF000085346424643EC102BBDE8C6
:1013A000F087332C0CDDB4F5806FF8D151EC100BC5
:1013B0003A460B46FDF726FE41EC100BBDE8F087E0
:1013C000A6F58265033D4FF0FF3323FA05F515EAD4
:1013D000080FE4D02AA3D3E9002351EC100BFDF74A
:1013E00011FE00220023FEF74FFAC0B1B9F1000F41
:1013F0001CDB28EA050813E021A3D3E9002351EC04
:10140000100BFDF7FFFD00220023FEF73DFA38B177
:10141000B9F1000F1BDB4FF00008C24600E0CA46DE
:101420005346424643EC102BBDE8F087142C09D0FC
:10143000C6F5866303334FF0010808FA03F818EB8A
:101440000708D6D30AF1010A28EA0508E8E729F0D7
:10145000004848EA07084FF0000AD045CBF6F07A7A
:1014600008BFCA4618BF4FF00008D9E74FF48013F1
:1014700043FA04F409EB040A89E700BFAFF30080E4
:101480009C7500883CE4377E00B553EC102B42F28B
:10149000FB1223F00043C3F6E972934285B027DDC7
:1014A0004FF6FF72C7F6EF7293420BDD51EC100B53
:1014B00002460B46FDF7A4FD02460B4643EC102BFB
:1014C00005B000BD684600F0EBFA00F0030001280B
:1014D0009DED000B9DED021B1DD0022812D008BB14
:1014E000012001F039FB53EC102B10461946E3E7BD
:1014F00000209FED111B01F02FFB53EC102B104629
:101500001946D9E7012001F027FB53EC102B1046B8
:1015100003F10041D0E700F0E3FD53EC102B10463F
:101520001946C9E700F0DCFD53EC102B104603F11F
:101530000041C1E7AFF300800000000000000000A0
:1015400010EE103A0BB902207047B3F1004FFAD0F9
:10155000A3F500016FF00142914201D804207047C9
:1015600003F1FF419142F9D94FF6FE72591EC0F2C4
:101570007F02914201D80320704703F100410139F5
:101580009142F8D9B3F1FF4F05D013F5000F14BF06
:101590000020012070470120704700BF00F0E4B830
:1015A000D0B52DED048BB0EE408AF0EE608A3C4C55
:1015B0008AB000F0D9F994F90030B0EE409AF0EE1C
:1015C000609A013335D0B0EE480AF0EE680A01F0B7
:1015D0004DFD00282DD051EC180B00220023FEF702
:1015E0003FF930B32F4B24780193002308938DEDFE
:1015F000028B8DED048B002C23D000270026CFF624
:10160000F07751EC180B00220023CDE90667FEF7B6
:1016100013F9002825D002239C42009336D0684657
:1016200001F05CFD002831D0089B002B27D19DEDF7
:10163000069BB0EE490AF0EE690A0AB0BDEC048BD5
:10164000D0BD4FF6FF774FF06046CCF2EF7751EC0C
:10165000180B00220023CDE90667FEF7EDF80028FD
:10166000D9D10123022C009315D0684601F036FD34
:1016700088B10D4801F034FD8DED060BD4E701F083
:10168000EDFF089B9DED069B0360D2E701F0E6FFAE
:1016900022230360C8E701F0E1FF21230360E8E7AC
:1016A0003804002000A7050860A9050810B52DED35
:1016B000048BB0EE408AF0EE608A294C8AB000F0CC
:1016C0002BFC94F90030B0EE409AF0EE609A0133B2
:1016D0002BD0B0EE480AF0EE680A01F0C7FC20B348
:1016E00051EC180B00220023FEF7B0F8E8B11D4BB7
:1016F0002478019301230093002308938DED048B3C
:101700008DED028BCCB10020002102460B46FDF787
:1017100055FF022CCDE9060115D101F09FFF2123D1
:101720000360089BABB99DED069BB0EE490AF0EE55
:10173000690A0AB0BDEC048B10BD0022002343EC03
:10174000172B8DED067B684601F0C8FC0028E8D118
:10175000E3E701F083FF089B9DED069B0360E4E750
:101760003804002008A70508F8B5B0EE407AF0EE7E
:10177000607A53EC112B544210461D46002125F08F
:101780000047044353EC102B47EAD474C7F6F071BA
:101790008C4216463DD85442344323F0004242EA7C
:1017A000D4748C4235D805F1404101F580110143D4
:1017B0004FD0AC1704F00204164344EAD37435D07A
:1017C000384341D00021C7F6F0718F424FD000213D
:1017D000C7F6F0718A4237D0D21B12153C2A42DC80
:1017E000002D7DDB53EC112B51EC170BFDF7E6FEC2
:1017F00041EC100B01F030FC01F06AFA51EC100BD7
:10180000012C68D0022C57D0002C48D141EC170B8A
:1018100007E051EC170B53EC112BFDF7F3FB41ECF8
:10182000170BB0EE470AF0EE670AF8BD032CC7D8D5
:1018300001A151F824F000BF231801082318010862
:10184000611801085B180108002B25DB9FED307B38
:10185000E7E7BDE8F84001F03BBA9FED2F7BE0E7FA
:101860009FED2F7BDDE72AA1D1E90001C8E7BA424D
:101870003CD0032CABD801A151F824F093180108F7
:101880008D180108611801085B1801089FED267B7F
:10189000C7E79FED277BC4E79FED277BC1E730A318
:1018A000D3E90023FDF7ACFB1DA3D3E90023FDF72B
:1018B000A7FB41EC170BB4E729A3D3E90023FDF7FD
:1018C0009FFB02460B4616A1D1E90001FDF798FBEC
:1018D00041EC170BA5E701F1004141EC170BA0E724
:1018E0003C32BFF67FAF0020002189E7032CABD844
:1018F000DFE804F00B0805029FED117B91E79FEDF7
:10190000127B8EE79FED127B8BE79FED137B88E7C1
:10191000182D4454FB21F93F182D4454FB2109C0D4
:10192000182D4454FB2109400000000000000080F5
:101930000000000000000000182D4454FB21F9BFF6
:10194000D221337F7CD902C0D221337F7CD902409F
:10195000182D4454FB21E9BF182D4454FB21E93FC5
:10196000075C143326A6A13C2DE9F84F55EC104B2B
:10197000B5F5801F2F4622DA25F00043234368D0B7
:10198000002D2046294670DB00230022C4F250338C
:10199000FDF7EAFC4FF6FF730F46C7F6EF739F4261
:1019A00004460D466FF0350210DD204629462246DA
:1019B0002B46FDF727FB41EC100BBDE8F88F4FF6E7
:1019C000FF73C7F6EF7300229F42EEDC3B15A3F5D1
:1019D0007E73073B9A18D60F901927F07F47C6F5FC
:1019E0007E76FDF75BFC073627F4700747EA06555D
:1019F00045EC104B8046894601F00AFC40464946BA
:101A000021A3D3E9002355EC104BFDF7ADFC20A337
:101A1000D3E9002382468B4640464946FDF7A4FCA5
:101A20001DA3D3E9002306460F4620462946FDF7AD
:101A30009BFC02460B4630463946FDF7E3FA024668
:101A40000B4650465946FDF7DDFA41EC100BBDE858
:101A5000F88F00210020CCF2503100220023FDF746
:101A6000ADFD41EC100BBDE8F88F22462B46FDF78B
:101A7000C7FA00220023FDF7A1FD41EC100BBDE8E1
:101A8000F88F00BFAFF3008000609F501344D33F36
:101A9000362BF111F3FE593D0EE526157BCBDB3FCE
:101AA0002DE9F04F53EC102B42F2FB1223F00044CF
:101AB000C3F6E97294428FB01E46074640F3AA80EF
:101AC0004DF67B13C4F202039C422ADC002E51EC3B
:101AD000100BDDA3D3E9002340F3CA81FDF790FA90
:101AE00042F2FB13C3F6F9739C428046894600F02C
:101AF000AA80D7A3D3E90023FDF782FA0D46044656
:101B00002B462246C7E9004540464946FDF778FA8C
:101B1000CFA3D3E90023FDF773FA0125C7E902013A
:101B200081E042F2FB13C4F239139C4240F3AA80D5
:101B30004FF6FF73C7F6EF739C4278DC4FEA245AE6
:101B4000AAF5826AAAF1060A51EC100BA4EB0A531B
:101B500019461D460446FDF7A1FEFDF79FFB804692
:101B6000894642464B4620462946CDE90889FDF77D
:101B700047FA00230022C4F27013FDF7F5FB0D466F
:101B80000446FDF78BFEFDF789FB8046894620461B
:101B9000294642464B46CDE90A89FDF731FA002332
:101BA0000022C4F27013FDF7DFFB002204460D464D
:101BB0000023CDE90C45FDF73FFE002800F07B81B6
:101BC0004046494600220023FDF736FE03240AADB5
:101BD000013C40B175E9020100220023FDF72CFE13
:101BE000013C0028F6D12346022400949E4C08A80C
:101BF00039465246019400F0ABFB002E054612DA3E
